:100000000C94671A0C94981A0C94981A0C94981AD9
:100010000C94981A0C94981A0C94981A0C94981A98
:100020000C94981A0C94981A0C94981A0C94981A88
:100030000C94981A0C94981A0C94981A0C94981A78
:100040000C94981A0C945CD10C94981A0C94981AED
:100050000C94981A0C94981A0C9459BE0C94F9A903
:100060000C94981A0C942F560C9425560C94981AAC
:100070000C94981A0C94981A0C94981A0C94981A38
:100080000C9408340C94981A0C94981A0C94981A9E
:100090000C94981A0C94981A0C94981A0C94981A18
:1000A0000C94981A0C94981A0C94DA330C94981AAD
:1000B0000C94981A0C94981A0C94981A0C94981AF8
:1000C0000C94981A0C94981A0C94981A0C94233740
:1000D0000C94ED360C94981A0C94981A0C94981A67
:1000E0000C94981A084AD73B3BCE016E84BCBFFDE6
:1000F000C12F3D6C74319ABD56833DDA3D00C77FF8
:1001000011BED9E4BB4C3E916BAAAABE0000008090
:100110003F05A84CCDB2D44EB93836A9020C50B91F
:10012000918688083CA6AAAA2ABE000000803F004B
:100130000C946CFC0D94560B0C94A1FC0D945F1068
:100140000C9450FC0C94D2FB0C94F0A70C9464FC1F
:100150000C9437440C949C560C94D6A90C9446FCF1
:100160000C94C5370D942B0C0C94ABFC0D945D0FC7
:100170000C9492FC0D94710F0D94280F0D94EE0CBD
:100180000C94BD370C94C9FB0C94EEFB0C94ABFBA8
:100190000D9436090D94D71E0D9486090C94FCFB22
:1001A0000C94C1560C94D5560C94E0560C940CA9A2
:1001B0000D9423050C943CFF0C94C9370D94FB0E51
:1001C0000C94D1560D9470100D947F0B0C94CCFBB5
:1001D0000C9488FC0D946C010C946D560D94BD0725
:1001E0000C94B5FC0C94B9370D943E0C0C94C137AB
:1001F0000D9452090D94B91E0C9439FC0C94C556FB
:100200000C94D6FB0C94BDFB0C94E0FB0C94CFA794
:100210000C94B5370C94F8FB0D94B60B0C94F2FBD0
:100220000D94220F0C94A6FB0C94BFFC0C94634419
:100230000D9413140C94CDA80C94AE370C94C5FBFC
:100240000C946BA40C9441FC0C94C9FC0D94E90B28
:100250000D94930B0C943AA70C94D9560C94AB566E
:100260000D9442010D942B0F0C94DC440C94C1FBB3
:100270000D94E80A0C9474FC0C94D3FC0C941C426E
:100280000C94A4440C9461370C94C9560D94D40278
:100290000D94220A0D94A5030D9403090D947E0F6D
:1002A0000D94B20A0D94CA0B0C9434A80C94E4FB80
:1002B0000C94DF370C947EFC0C94EB560C94EAFB08
:1002C0000C94E7370C94F3560C94EEA40C94CD5692
:1002D0000C94EDA40C94D4370C945AFC0D94440F58
:1002E0000C94DFA80D94530F0C9490370C94BA56CD
:1002F0000D945D000C949F370C946F420C94CD3795
:100300000C94DCFB0C944FA80C946B420C9457A7F4
:100310000D9433114E414E494E495459494E46CDE4
:10032000CCCC3D0AD7233C17B7D13877CC2B3295AC
:1003300095E6241FB14F0A000020410000C842008A
:10034000401C4620BCBE4CCA1B0E5AAEC59D740054
:10035000407A10F35A00A0724E18090010A5D4E894
:100360000000E87648170000E40B54020000CA9A27
:100370003B000000E1F50500008096980000004079
:10038000420F000000A086010000001027000000BE
:1003900000E803000000006400000000000A000004
:1003A0000000000100000000002C76D888DC674FB8
:1003B0000823DFC1DFAE59E1B1B796E5E3E453C6E8
:1003C0003AE651997696E8E6C28426EB898C9B62E0
:1003D000ED407C6FFCEFBC9C9F40F2BAA56FA5F48A
:1003E00090055A2AF75C936B6CF9676DC11BFCE0B2
:1003F000E40D47FEF520E6B500D0ED902E03009405
:100400003577050080841E080000204E0A00000099
:10041000C80C333333330F986E12831141EF8D21A3
:1004200014893BE65516CFFEE6DB18D1844B381B0A
:10043000F77C1D901DA4BBE424203284725E2281CF
:1004400000C9F124ECA1E53D27434F4D4D554E49E0
:10045000434154494F4E0044525952554E00455263
:10046000524F525300494E464F004543484F0045B6
:1004700072726F722077726974696E6720746F2070
:10048000454550524F4D210A0053544F505045445A
:100490002E20005072696E7465722073746F7070D4
:1004A00065642064756520746F206572726F727365
:1004B0002E2046697820746865206572726F7220FC
:1004C000616E6420757365204D39393920746F2051
:1004D000726573746172742E202854656D70657234
:1004E00061747572652069732072657365742E205E
:1004F0005365742069742061667465722072657337
:1005000074617274696E67290A004E6F20436865D2
:10051000636B73756D2077697468206C696E6520F4
:100520006E756D6265722C204C617374204C696E1F
:10053000653A20004E6F20436865636B73756D20CC
:1005400077697468206C696E65206E756D6265727E
:100550002C204C617374204C696E653A20006368EE
:1005600065636B73756D206D69736D617463682C61
:10057000204C617374204C696E653A20004C696EA2
:1005800065204E756D626572206973206E6F7420F0
:100590004C617374204C696E65204E756D62657296
:1005A0002B312C204C617374204C696E653A20000D
:1005B0004D3131300053657269616C207374617420
:1005C0007573206D69736D617463680A0077616982
:1005D000740A0053442072656164206572726F7200
:1005E0000A002121204B494C4C20636175736564DE
:1005F00020627920746F6F206D75636820696E6169
:1006000063746976652074696D65202D2063757249
:1006100072656E7420636F6D6D616E643A20004880
:100620006F74656E642049646C652054696D656FF4
:10063000757400486F74656E642049646C6520545D
:10064000696D656F75740A003D3D6F6E46696C613A
:100650006D656E7452756E6F75743D3D0070617599
:100660007365004D363030002066696C616D656ED3
:10067000745F72756E6F7574200066696C616D656C
:100680006E745F72756E6F757420540046696C618C
:100690006D656E7452756E6F75742054002A2A2A27
:1006A000496E6974696E67206361726420697320A2
:1006B0004F4B2A2A2A004D6564696120496E736593
:1006C00072746564004D656469612052656D6F7672
:1006D0006564004D313030305300627573793A20D3
:1006E00070617573656420666F7220696E707574D1
:1006F0000A00627573793A207061757365642066CB
:100700006F7220757365720A00627573793A207092
:10071000726F63657373696E670A002A2A2A6B69B0
:100720006C6C2A2A2A00706F7765726F6666004BC0
:10073000494C4C45442E20005072696E74657220FD
:1007400068616C7465642E206B696C6C2829206369
:10075000616C6C6564210A0053544F505045442E1F
:1007600020005072696E7465722073746F707065CA
:10077000642064756520746F206572726F72732EC9
:100780002046697820746865206572726F722061F6
:100790006E6420757365204D39393920746F20726D
:1007A0006573746172742E202854656D7065726172
:1007B000747572652069732072657365742E205399
:1007C0006574206974206166746572207265737443
:1007D000617274696E67290A006563686F3A004543
:1007E00072726F723A0042696C696E656172204C78
:1007F0006576656C696E6720477269643A0A002104
:10080000212053544F502063616C6C6564206265F5
:100810006361757365206F6620424C546F75636821
:10082000206572726F72202D20726573746172740C
:100830002077697468204D3939390A002121205305
:10084000544F502063616C6C656420626563617510
:100850007365206F6620424C546F75636820657223
:10086000726F72202D2072657374617274207769C3
:100870007468204D3939390A002F2F616374696F0C
:100880006E3A0070726F6D70745F00656E64005335
:10089000656E64204D31303820746F207265737539
:1008A0006D650A00496E736572742066696C616DCE
:1008B000656E7420616E642073656E64204D313006
:1008C000380A005265686561742066696E697368EC
:1008D00065642E0052656865617420446F6E650022
:1008E000526568656174696E672E2E2E00526568C8
:1008F000656174004865617465722054696D656F47
:1009000075740053656E64204D31303820746F204B
:1009100068656174206E6F7A7A6C650A004E6F7A32
:100920007A6C65205061726B656400486F74656E07
:100930006420746F6F20636F6C640A00706175735C
:1009400065640050617573650044697361626C652C
:1009500052756E6F75740050757267654D6F726574
:10096000005061757365640073686F770062757419
:10097000746F6E00626567696E004C6F616420463B
:10098000696C616D656E74004C6F61642046696CC2
:10099000616D656E74205400496E736572742066D3
:1009A000696C616D656E7420616E642073656E6440
:1009B000204D3130380A00726573756D65640052E0
:1009C0006573756D696E670057616974696E67203C
:1009D000666F72206865617475702E0A004C6561DF
:1009E00076696E6720473236003F537065636966EB
:1009F00069656420582C5920636F6F7264696E6159
:100A00007465206F7574206F6620626F756E6473F5
:100A10002E0A003F28522965706561742076616C4A
:100A20007565206E6F7420706C61757369626C659A
:100A30003B206D757374206265206174206C656164
:100A4000737420312E0A003F285229657065617445
:100A5000206D7573742062652073706563696669C3
:100A60006564207768656E206E6F74207573696E9B
:100A70006720616E204C43442E0A003F537065632B
:100A80006966696564206E6F7A7A6C652074656D3D
:100A90007065726174757265206E6F7420706C6120
:100AA000757369626C652E0A003F537065636966F1
:100AB0006965642066696C616D656E742073697A1E
:100AC00065206E6F7420706C61757369626C652E41
:100AD0000A003F53706563696669656420707269D6
:100AE0006D65206C656E677468206E6F7420706C25
:100AF00061757369626C652E0A003F5072696D659D
:100B0000206C656E677468206D7573742062652053
:100B1000737065636966696564207768656E206EC9
:100B20006F74207573696E6720616E204C43442E8C
:100B30000A003F537065636966696564206E6F7A69
:100B40007A6C652073697A65206E6F7420706C61B1
:100B5000757369626C652E0A003F52657472616339
:100B600074696F6E204D756C7469706C6965722064
:100B70006D7573742062652073706563696669655D
:100B8000642E0A003F53706563696669656420528C
:100B9000657472616374696F6E204D756C746970F1
:100BA0006C696572206E6F7420706C617573696218
:100BB0006C652E0A003F5370656369666965642041
:100BC0006C6179657220686569676874206E6F74FE
:100BD00020706C61757369626C652E0A0043292E62
:100BE0000A003F53706563696669656420626564E5
:100BF0002074656D7065726174757265206E6F74B6
:100C000020706C61757369626C65202834302D002A
:100C1000473236207374617274696E672E2E2E0A05
:100C2000004F46460A00466164652048656967686A
:100C3000742000426564204C6576656C696E67209F
:100C4000004661696C656420746F20656E61626C3A
:100C50006520426564204C6576656C696E670A00A4
:100C6000496E76616C6964206D6573682E0A005068
:100C7000726F62696E6720506F696E740025532031
:100C800025692F2569002E0A002F0050726F6269B6
:100C90006E67206D65736820706F696E7420002028
:100CA0002844525952554E29004732392041757413
:100CB0006F20426564204C6576656C696E67003F05
:100CC00020284C2C522C462C4229206F7574206F02
:100CD0006620626F756E64732E0A003F2856296580
:100CE00072626F7365206C6576656C20696D706CDF
:100CF00061757369626C652028302D34292E0A00D5
:100D0000426164205A2076616C75650A004E6F203E
:100D100062696C696E65617220677269640A004479
:100D20006576696174696F6E0025533A20257300FA
:100D300046696E6973686564210A003A207A3A2030
:100D400000206F662000476F696E6720746F3A203D
:100D5000580043570A00206469723A0020616E67A8
:100D60006C653A00537461727420726164697573C2
:100D70003A004D343820506F696E740025533A2084
:100D800025642F256400506F736974696F6E696EF6
:100D900067207468652070726F62652E2E2E0A00BF
:100DA0003F4C656773206F66206D6F76656D656E6D
:100DB0007420696D706C61757369626C6520283090
:100DC0002D3135292E0A003F2028582C5929206F13
:100DD0007574206F6620626F756E64732E0A005002
:100DE000726F6265206F7574206F6620626F756E1A
:100DF0006473003F53616D706C652073697A652080
:100E00006E6F7420706C61757369626C6520283434
:100E10002D3530292E0A004D3438205A2D50726F4E
:100E20006265205265706561746162696C6974798C
:100E300020546573740A003F2856296572626F73E7
:100E400065206C6576656C20696D706C6175736981
:100E5000626C652028302D34292E0A005374616E8F
:100E60006461726420446576696174696F6E3A20CA
:100E7000002052616E67653A2000204D61783A206B
:100E800000204D696E3A2000205369676D613A2059
:100E9000004D65616E3A20005741524E494E472140
:100EA000204C6F77205A204A65726B206D61792043
:100EB0006C65616420746F20756E77616E74656413
:100EC000207061757365732E0A004F4646004F4EC1
:100ED0000020204D61783A2000200020204D696ECE
:100EE0003A2000536F667420656E6473746F70737C
:100EF0003A20003D3D4F6E506F7765724C6F7373B3
:100F0000526573756D653D3D004D32342053256C3F
:100F1000642054256C64004739322E3920452573EE
:100F200000473120462564004739322E39205A25A2
:100F300073004731205A302046323030004731208C
:100F400058257320592573204633303030004D34F6
:100F5000323020532569205A2573004D3130362018
:100F600050256920532569004D32303020442573C7
:100F70000047323852305859004739322E3920450F
:100F800030205A300A47315A2573004D313039200C
:100F9000532569004D31393020532569004D3432D5
:100FA00030205330205A300020496E76616C6964DD
:100FB000206578747275646572200047322F47335C
:100FC0002062616420706172616D65746572730A7C
:100FD00000536C6565702E2E2E005A2050726F6281
:100FE000652050617374204265640A005A20507273
:100FF0006F62652050617374204265640047323827
:101000004C30004D3131372050726F62652066617F
:10101000696C65642E0A4732380A0070726F626527
:101020005F72657769706500473239205265747266
:1010300079696E670050726F62696E6720466169F8
:101040006C6564004D31313720426564206C6576F3
:10105000656C696E67206661696C65642E0A47304D
:10106000205A31300A4D3330302050323520533839
:1010700038300A4D333030205035302053300A4D4F
:101080003330302050323520533838300A4D333029
:1010900030205035302053300A4D3330302050321C
:1010A0003520533838300A4D333030205035302019
:1010B00053300A47342053310070726F62655F66A7
:1010C00061696C6564004D31313720426564206C84
:1010D0006576656C696E6720646F6E652E00205AB8
:1010E0003A200020593A200042656420583A2000F6
:1010F0004D65736820706F696E74206F7574206F12
:10110000662072616E67650A004D302053746F70FF
:10111000004D312053746F7000436F6E74696E75AB
:101120006500436C69636B20746F20526573756D45
:10113000652E2E2E004E6F204D6F76652E00456E6B
:10114000642066696C65206C6973740A0042656787
:10115000696E2066696C65206C6973740A004E6F55
:10116000206D656469610A00526573756D696E670B
:1011700020534400286E6F2066696C652900437512
:101180007272656E742066696C653A2000507269EF
:101190006E742074696D653A20000A53746174732B
:1011A0003A2046696C616D656E7420757365643AAA
:1011B00020002C204C6F6E67657374206A6F623A52
:1011C0002000546F74616C2074696D653A2000537F
:1011D000746174733A20002C204661696C65643A2E
:1011E00020002C2046696E69736865643A200050BF
:1011F00072696E74733A200053746174733A2000FC
:10120000436F6F6C696E672E2E2E0048656174699E
:101210006E672E2E2E0045202553006F6B006F66E3
:1012200066006A0465045E04570449044445425557
:10123000473A004D31313320530042656420436FFB
:101240006F6C696E672E2E2E0042656420486561C2
:1012500074696E672E2E2E00544D33442045352080
:10126000506C7573204F46462E002F2F00205200E1
:10127000416363656C65726174696F6E3A205000FA
:101280004D32303620580046523A0020466C6F7777
:101290003A20003A200020536572766F2000206FBC
:1012A0007574206F662072616E67650A00536572FF
:1012B000766F200020643A0020693A0020703A00DE
:1012C000496E76616C6964206578747275646572C4
:1012D0000A0020643A0020693A0020703A006469EC
:1012E0007300656E0043290A0061626C6564202802
:1012F0006D696E2074656D702000436F6C642065AD
:101300007874727564657320617265200050494479
:10131000204175746F74756E6500504944204175A5
:10132000746F74756E65206661696C656421204216
:101330006164206865617465722069640A004669A9
:101340006C616D656E742072756E6F757420646962
:101350007374616E636520286D6D293A20004669BB
:101360006C616D656E742072756E6F757420004DC2
:1013700034323120696E636F7272656374207061FC
:1013800072616D657465722075736167650A004DE1
:1013900065736820706F696E74206F7574206F6656
:1013A0002072616E67650A004F666673657473200C
:1013B0004170706C696564004572723A20546F6FB9
:1013C000206661722100546F6F2066617220667220
:1013D0006F6D207265666572656E636520706F69FA
:1013E0006E740A00454550524F4D204F4B0A005035
:1013F0006F7765722D6C6F7373207265636F76659E
:10140000727920004D383400446F6E652070726927
:101410006E74696E672066696C650A004D37370027
:101420004D3331004361703A004D454154504143C2
:101430004B00434F4F4C45525F54454D5045524130
:1014400054555245004348414D4245525F54454D25
:10145000504552415455524500424142595354451A
:101460005050494E470041524353004D4F54494F4D
:101470004E5F4D4F44455300544845524D414C5FDB
:1014800050524F54454354494F4E004C4F4E475FC6
:1014900046494C454E414D45004155544F524550EB
:1014A0004F52545F53445F53544154555300534477
:1014B0005F575249544500524550454154005344EA
:1014C000434152440050524F4D50545F5355505079
:1014D0004F525400454D455247454E43595F504188
:1014E0005253455200434153455F4C494748545F6E
:1014F0004252494748544E45535300544F47474C76
:10150000455F4C494748545300534F465457415246
:10151000455F504F574552004255494C445F504536
:101520005243454E54004C4556454C494E475F4446
:10153000415441005A5F50524F42450052554E4F60
:101540005554004155544F4C4556454C0050524956
:101550004E545F4A4F420050524F4752455353003A
:101560004155544F5245504F52545F54454D5000D1
:10157000564F4C554D455452494300454550524FE6
:101580004D0042494E4152595F46494C455F5452C5
:10159000414E534645520053455249414C5F584FC6
:1015A0004E5F584F4646004649524D574152455F9F
:1015B0004E414D453A4D61726C696E20322E302E8F
:1015C000375F4457372E3320544D33442045355030
:1015D000454D44424220284170722032342032303E
:1015E00032312032313A33323A33322920534F5597
:1015F0005243455F434F44455F55524C3A687474BB
:1016000070733A2F2F6769746875622E636F6D2F40
:10161000496E73616E6974794175746F6D61746937
:101620006F6E2F4D61726C696E2F747265652F43FA
:101630007265616C6974794477696E5F322E30200F
:1016400050524F544F434F4C5F56455253494F4EA3
:101650003A312E30204D414348494E455F54595050
:10166000453A544D334420453520506C7573204520
:10167000585452554445525F434F554E543A3120C9
:10168000555549443A63656465326132662D34319B
:1016900061322D343734382D396231322D6335358E
:1016A0006336326633363766660A0050726F62659B
:1016B000204F6666736574205A0050726F62652011
:1016C0004F6666736574205A00290A0020746F20E3
:1016D000003F5A206F7574206F662072616E6765D7
:1016E000202800290A0020746F20003F59206F75C0
:1016F00074206F662072616E676520282D00290AAC
:101700000020746F20003F58206F7574206F662092
:1017100072616E676520282D0050726F6265204FE0
:10172000666673657420580043616E6E6F74206F37
:1017300070656E207375626469722000256973009C
:1017400025696D20256973002569682025696D204C
:1017500025697300256964202569682025696D2045
:101760002569730025697920256964202569682029
:1017700025696D20256973003D3D4477696E2049D8
:101780006E697420436F6D706C6574653D3D002A11
:101790002A2A4E6F7A7A6C6554656D705374617441
:1017A00075735B325D203D003D3D48656174696E37
:1017B0006720446F6E65204368616E6765204669E7
:1017C0006C616D656E743D3D0020207374617274B0
:1017D00070726F677265737320003D3D7761697445
:1017E00077617920353D3D003D3D776169747761D2
:1017F0007920343D3D003D3D776169747761792002
:10180000333D3D003D3D7761697477617920313D1D
:101810003D003D3D6F6E5072696E7454696D657226
:1018200053746F707065643D3D003D3D6F6E466161
:1018300063746F727952657365743D3D00270A0ABF
:101840000000272027002027002D006E6F74696696
:1018500069636174696F6E200063616E63656C001B
:101860005072696E742041626F72746564004469DD
:10187000736D6973730055492041626F72746564BA
:1018800000726573756D65004D3234002A2A2A4353
:10189000506C617920546F6E652A2A2A003D3D6F95
:1018A0006E5072696E7454696D65725061757365BE
:1018B000643D3D00486F6D696E67204661696C65E7
:1018C00064006F70656E0054524947474552454465
:1018D000003A200066696C616D656E74007A5F6D18
:1018E000696E00795F6D617800785F6D6178005294
:1018F00065706F7274696E6720656E6473746F7063
:10190000207374617475730A0020746F6F206C6F9C
:101910006E6720657874727573696F6E207072657A
:1019200076656E7465640A0020636F6C6420657868
:1019300074727573696F6E2070726576656E74650A
:10194000640A00486F6D6520257325732573204652
:1019500069727374005761726E696E673A20486FDE
:101960006D696E672042756D702044697669736F8A
:1019700072203C20310A000202040000B44300003F
:10198000B443000000000000B4430000B443000072
:10199000C843000000410000004100000040010178
:1019A000FF000000010000000100008000555555B7
:1019B000000000400033333300AAAA2A00499224D1
:1019C0000000002000C7711C0099991900D145172B
:1019D00000555515003BB113002449120011111197
:1019E00000000010000F0F0F00E3380E0043790DC8
:1019F00000CCCC0C00C3300C00E8A20B0064210B1F
:101A000000AAAA0A00703D0A009DD80900427B097D
:101A10000092240900DCD3080088880800104208DE
:101A20000000000800F0C107008787070075500715
:101A300000711C07003EEB0600A1BC060069900681
:101A40000066660600703E06006118060017F40581
:101A50000074D105005BB00500B29005006272050C
:101A6000005555050078390500B81E050005050527
:101A7000004EEC040087D40400A1BD040090A7042C
:101A80000049920400C17D0400EE690400C75604B9
:101A900000444404005C32040008210400411004A6
:101AA00000000004003FF00300F8E0030026D2032A
:101AB00000C3C30300CCB503003AA803000A9B038C
:101AC00000388E0300C08103009F750300D06903B6
:101AD00000505E03001D53030034480300913D0392
:101AE000003333030016290300381F030097150342
:101AF00000300C0300030303000BFA020049F1025B
:101B000000BAE802005CE002002DD802002DD002ED
:101B10000059C80200B0C0020031B90200DAB102B7
:101B200000AAAA0200A0A30200BC9C0200FA95022F
:101B3000005C8F0200DF88020082820200457C0286
:101B4000002776020027700200436A02007C6402CC
:101B500000D05E02003F590200C8530200FFFDFCA6
:101B6000FAF8F6F4F2F0EEECEAE9E7E5E3E1E0DEBC
:101B7000DCDAD9D7D5D4D2D0CFCDCBCAC8C7C5C36C
:101B8000C2C0BFBDBCBAB9B7B6B4B3B2B0AFADACEA
:101B9000AAA9A8A6A5A4A2A1A09E9D9C9A9998973F
:101BA00095949392908F8E8D8B8A89888786848373
:101BB0008281807F7E7D7B7A797877767574737287
:101BC00071706F6E6D6C6B6A69686766656463627D
:101BD00061605F5E5D5C5B5A595858575655545367
:101BE000525150504F4E4D4C4B4A4A494847464639
:101BF000454443424241403F3E3E3D3C3B3B3A39F7
:101C0000383837363535343332323130302F2E2EA6
:101C10002D2C2B2B2A292928272726252524232349
:101C200022212120201F1E1E1D1C1C1B1B1A1919DE
:101C30001818171616151514131312121111100F68
:101C40000F0E0E0D0D0C0C0B0A0A090908080707E8
:101C5000060605050404030302020100003D3D6F72
:101C60006E5072696E7454696D65725374617274EA
:101C700065643D3D000000B4430000B4430000C86B
:101C8000430000000000000000000000003D3D6F28
:101C90006E53746F726553657474696E67733D3DFE
:101CA000003D3D6F6E436F6E666967757261746962
:101CB0006F6E53746F72655772697474656E3D3DD3
:101CC0000053657474696E67732053746F72656432
:101CD000000A20696E6974207A70726F62655F7A9B
:101CE0006F6666736574203D20003D3D6F6E436FE7
:101CF0006E66696775726174696F6E53746F726531
:101D0000526561643D3D00454550524F4D20496E3E
:101D1000697469616C697A65640A003B20003A0A5B
:101D20000020204D363033200020440020204D3448
:101D3000313220530046696C616D656E7420727596
:101D40006E6F75742073656E736F723A0020550064
:101D50004C0046696C616D656E74206C6F61642F18
:101D6000756E6C6F6164206C656E677468733A00A1
:101D700020204D3835312058005A2D50726F626541
:101D8000204F66667365740020204D343133205334
:101D900000506F7765722D4C6F7373205265636FBF
:101DA000766572793A0020440020490020204D33A6
:101DB000303420500020440020490020204D333092
:101DC000312050005049442073657474696E677304
:101DD0003A00204A0020204732392057204900206D
:101DE000204D3432302053004175746F20426564B9
:101DF000204C6576656C696E673A0020204D323064
:101E000036205800486F6D65206F66667365743ABA
:101E10000020580020530020204D32303520420051
:101E2000416476616E6365643A20423C6D696E5F21
:101E30007365676D656E745F74696D655F75733E1C
:101E400020533C6D696E5F66656564726174653EC2
:101E500020543C6D696E5F74726176656C5F666577
:101E60006564726174653E20583C6D61785F785F8F
:101E70006A65726B3E20593C6D61785F795F6A6577
:101E8000726B3E205A3C6D61785F7A5F6A65726B57
:101E90003E20453C6D61785F655F6A65726B3E0010
:101EA00020540020520020204D3230342050004178
:101EB0006363656C65726174696F6E2028756E6905
:101EC00074732F7332293A20503C7072696E745FBC
:101ED000616363656C3E20523C7265747261637429
:101EE0005F616363656C3E20543C74726176656C1F
:101EF0005F616363656C3E0020204D3230312058B5
:101F0000004D6178696D756D20416363656C657224
:101F10006174696F6E2028756E6974732F7332292E
:101F20003A0020204D3230332058004D6178696DE1
:101F3000756D206665656472617465732028756EC1
:101F40006974732F73293A00537465707320706538
:101F50007220756E69743A0020440020204D3230A2
:101F6000302053002044697361626C65640A004646
:101F7000696C616D656E742073657474696E6773E6
:101F80003A0020286D6D2900202047323120202082
:101F9000203B20556E69747320696E206D6D003D85
:101FA0003D6F6E4C6F616453657474696E67733D09
:101FB0003D0000803B4400803B4400002041000085
:101FC00096420000A0420000A042000048440000E9
:101FD000BE42D0070000D0070000640000004B00A4
:101FE000000024F4D43050C38E20C2A24017828B4C
:101FF0007011127A910D816CD90AA861E108C75855
:102000006607615143061E4B5D05C145A7041A4191
:102010001104093D9803713931034036DB02653301
:102020009102D4305402802E1D02632CEE01752AD9
:10203000C501B028A001102781018F2564012B2440
:102040004B01E0223401AC211F018D200D01801FC6
:10205000FC00841EED00971DDF00B81CD200E61BBB
:10206000C600201BBC00641AB200B219A8000A19ED
:10207000A0006A189900D117910040178B00B5167F
:10208000840031167E00B31579003A157300C71429
:102090006F0058146A00EE1366008813630025135E
:1020A0005E00C7125B006C12570015125400C1117C
:1020B000510070114F0021114B00D61049008D10B6
:1020C00047004610440002104200C00F4000800F3D
:1020D0003E00420F3C00060F3B00CB0E3800930E33
:1020E00037005C0E3500270E3400F30D3200C10DB1
:1020F0003100900D3000600D2E00320D2D00050DC9
:102100002C00D90C2B00AE0C2900850C29005C0C8E
:102110002700350C27000E0C2600E80B2400C40B0A
:102120002400A00B23007D0B23005A0B2100390B48
:102130002100180B2000F80A1F00D90A1E00BB0A54
:102140001E009D0A1D00800A1D00630A1C00470A2C
:102150001B002C0A1B00110A1A00F7091A00DD09DE
:102160001900C4091900AB091900920917007B096D
:102170001800630917004C091600360916002009DB
:1021800016000A091500F5081500E0081400CC082F
:102190001400B8081400A4081400900813007D0867
:1021A00012006B0813005808120046081200340889
:1021B0001100230811001208110001081100F00796
:1021C0001000E0071000D0071000C0071000B00793
:1021D0000F00A107100091070E0083070F0074077E
:1021E0000F0065070E0057070E0049070E003B075A
:1021F0000D002E070E0020070D0013070D00060727
:102200000D00F9060C00ED060D00E0060C00D406EA
:102210000C00C8060C00BC060C00B0060C00A4069E
:102220000B0099060C008D060B0082060B0077064A
:102230000B006C060B0061060A0057060B004C06EB
:102240000A0042060A0038060A002E060A00240682
:102250000A001A060A001006090007060A00FD0512
:102260000900F4050900EB050900E2050900D9059C
:102270000900D0050900C7050900BE050900B5051C
:102280000800AD050800A50509009C050800940597
:1022900008008C050800840508007C05080074050A
:1022A00008006C050700650508005D050700560578
:1022B00008004E05070047050700400508003805DF
:1022C0000700310507002A050700230507001C0544
:1022D0000600160507000F050700080506000205A1
:1022E0000700FB040600F5040700EE040600E804FE
:1022F0000600E2040700DB040600D5040600CF0454
:102300000600C9040600C3040600BD040600B704A5
:102310000600B1040500AC040600A6040600A004F3
:1023200005009B04060095040500900406008A043D
:10233000050085040500800406007A040500750484
:102340000500700405006B040500660405006104C7
:1023500005005C04050057040500520405004D0407
:10236000050048040500430405003E0404003A0447
:10237000050035040500300404002C040500270482
:102380000400230405001E0404001A0404001604BB
:102390000500110404000D040400090405000404F0
:1023A000040000040400FC030400F8030400F40328
:1023B0000400F0030400EC030400E8030400E40359
:1023C0000400E0030400DC030400D8030400D40389
:1023D0000400D0030400CC030400C8030300C503B9
:1023E000030024F404D9201BC40C5C0E9804C40917
:1023F0005F0265077101F405F900FB04B3004804AE
:102400008700C10369005803550003034500BE025D
:102410003A008402310053022A00290225000402F6
:102420002000E4011C00C8011900AF011700980149
:1024300014008401130071011000610110005101AA
:102440000E0043010D0036010B002B010B00200193
:102450000B00150109000C01090003010800FB0035
:102460000800F3000800EB000700E4000600DE00AF
:102470000600D8000600D2000600CC000500C70008
:102480000500C2000500BD000400B9000400B5004D
:102490000400B1000400AD000400A9000400A50080
:1024A0000300A20003009F0004009B0003009800AB
:1024B00003009500020093000300900003008D00CC
:1024C00002008B00030088000200860002008400E6
:1024D0000300810002007F0002007D0002007B00FB
:1024E000020079000200770001007600020074000B
:1024F000020072000100710002006F0002006D0016
:1025000001006C0002006A0001006900020067001F
:102510000100660001006500010064000200620025
:10252000010061000100600001005F0002005D0029
:1025300001005C0001005B0001005A00010059002D
:10254000010058000100570001005600010055002D
:10255000010054000100530000005300010052002C
:10256000010051000100500001004F0001004E0029
:1025700000004E0001004D0001004C0001004B0026
:1025800000004B0001004A00010049000100480022
:10259000000048000100470001004600000046001E
:1025A0000100450000004500010044000100430017
:1025B0000000430001004200000042000100410011
:1025C000000041000100400001003F0000003F000A
:1025D00001003E0000003E0001003D0000003D0003
:1025E00001003C0000003C0000003C0001003B00FA
:1025F00000003B0001003A0000003A0001003900F1
:1026000000003900010038000000380000003800E8
:1026100001003700000037000100360000003600DE
:1026200000003600010035000000350000003500D4
:1026300001003400000034000000340001003300C9
:1026400000003300000033000100320000003200BF
:1026500000003200010031000000310000003100B4
:1026600001003000000030000000300001002F00A9
:1026700000002F0000002F0000002F0001002E009E
:1026800000002E0000002E0001002D0000002D0093
:1026900000002D0000002D0001002C0000002C0087
:1026A00000002C0000002C0001002B0000002B007B
:1026B00000002B0000002B0001002A0000002A006F
:1026C00000002A0000002A00010029000000290063
:1026D0000000290000002900000029000100280056
:1026E000000028000000280000002800000028004A
:1026F000010027000000270000002700000027003D
:10270000000027000100260000002600000026002F
:102710000000260000002600010025000000250022
:102720000000250000002500000025000000250015
:102730000100240000002400000024000000240008
:1027400000002400010023000000230000002300FB
:1027500000002300000023000000230000002300ED
:1027600001002200000022000000220000002200E0
:1027700000002200000022000100210000002100D2
:1027800000002100000021000000210000002100C5
:1027900000002100010020000000200000002000B7
:1027A00000002000000020000000200000002000A9
:1027B0000000200001001F0000001F0000001F009B
:1027C00000001F0000001F0000001F0000001F008D
:1027D00001001E0000001E0000001E0000001E0080
:1027E0000000393000003325000087190000B00FC9
:1027F0000000DB080000BD040000740200003F017F
:10280000000020436F756E7420583A00236465669B
:10281000696E652044454641554C545F0000626531
:1028200064004B6420004B6920004B70200050492D
:1028300044204175746F74756E652066696E6973A6
:10284000686564212050757420746865206C61731C
:1028500074204B702C204B6920616E64204B6420E7
:10286000636F6E7374616E74732066726F6D206235
:10287000656C6F7720696E746F20436F6E66696751
:1028800075726174696F6E2E680A00504944204168
:1028900075746F74756E65206661696C656421205E
:1028A00074696D656F75740A0050494420417574F0
:1028B0006F74756E65206661696C6564212054656E
:1028C0006D706572617475726520746F6F206869D0
:1028D00067680A00204B643A2000204B693A2000C8
:1028E000204B703A200020436C6173736963205061
:1028F0004944200A00204E6F206F76657273686F1E
:102900006F740A002054753A2000204B753A20005D
:10291000206D61783A2000206D696E3A20002064B5
:102920003A200020626961733A20005049442041F6
:1029300075746F74756E652073746172740A0050DB
:102940004944204175746F74756E65206661696CC9
:102950006564212054656D706572617475726520BF
:10296000746F6F20686967680A00426564004531CA
:1029700000626564002C2073797374656D20737434
:102980006F7070656421204865617465725F4944A9
:102990003A200048656174696E67204661696C651C
:1029A000640048656174696E67206661696C65647E
:1029B000004D3131322053687574646F776E0010AA
:1029C00000C90210012C014001220170011801B060
:1029D000010E01F00104015002FA00B002F00030D3
:1029E00003E600D003DC009004D2007005C800A00C
:1029F00006BE000008B400B009AA00D00BA0006019
:102A00000E960060118C000015820020197800C01D
:102A10001D6E00A0226400B0275A00902C500000C8
:102A2000314600E0343C0010383200903A28006013
:102A30003C1E00A03D1400803E0A00203F000054D0
:102A40004845524D414C2052554E41574159005432
:102A50006865726D616C2052756E617761790045B1
:102A600072723A204D415854454D50004D415854D2
:102A7000454D5020747269676765726564004572E0
:102A8000723A204D494E54454D50004D494E5445E3
:102A90004D502074726967676572656400202F006D
:102AA0002042403A0020403A0020573A0020573A4E
:102AB00000496E76616C696420657874727564652E
:102AC000720A007C3C3E5E2B3D3F2F5B5D3B2C2A17
:102AD000225C0043616E6E6F74206F70656E2073B0
:102AE00075626469722000534420496E69742046FF
:102AF00061696C0053442063617264206F6B0A004B
:102B00006F70656E526F6F74206661696C65640AE0
:102B100000766F6C756D652E696E697420666169EB
:102B20006C65640A004E6F20534420636172640A2E
:102B3000000A4D3234004D3233202573002E0A0036
:102B40006F70656E206661696C65642C2046696CE7
:102B5000653A200046696C652073656C6563746531
:102B6000640A002053697A653A200046696C652042
:102B70006F70656E65643A2000454E44205355429F
:102B8000524F5554494E450A002220706F7300225F
:102B900020706172656E743A2200535542524F554F
:102BA00054494E452043414C4C2074617267657412
:102BB0003A220053756263616C6C204F76657266D1
:102BC0006C6F77004578636565646564206D617836
:102BD00020535542524F5554494E452064657074F8
:102BE000683A002E0A0044656C6574696F6E206651
:102BF00061696C65642C2046696C653A2000466901
:102C00006C652064656C657465643A00534420709B
:102C100072696E74696E67206279746520004E6F08
:102C200074205344207072696E74696E670A00578D
:102C3000726974696E6720746F2066696C653A20EA
:102C400000667265736800646F696E67002066696C
:102C50006C653A20004E6F7720002F6175746F25E8
:102C6000632E67002020506C616E6E65724275663F
:102C700066657242797465733A2000204672656514
:102C8000204D656D6F72793A2000436F6D70696CED
:102C900065643A2041707220323420323032310A79
:102CA00000204C61737420557064617465643A202F
:102CB000323032312D30342D3138207C2041757442
:102CC000686F723A2054696E794D616368696E6508
:102CD0007333440A00322E302E375F4457372E3379
:102CE0000A004D61726C696E0020536F66747761E3
:102CF00072652052657365740A00205761746368B9
:102D0000646F672052657365740A002042726F77A2
:102D10006E206F75742052657365740A00204578C3
:102D20007465726E616C2052657365740A00506F31
:102D300077657255700A0073746172740A004732C5
:102D4000385859004D31303031006572726F722041
:102D500077726974696E6720746F2066696C650AA2
:102D600000446F6E6520736176696E672066696CDA
:102D7000652E0A004D323900456E6473746F7073AE
:102D8000002553202563202563202563202563002B
:102D9000205A3A0020593A0020583A00656E647370
:102DA000746F7073206869743A20006001F40170D8
:102DB00001EA019001E001B001D601D001CC01008F
:102DC00002C2013002B8016002AE019002A401D03B
:102DD000029A012003900170038601C0037C013038
:102DE000047201A004680120055E01B00554016071
:102DF000064A0120074001F0073601F0082C0110B7
:102E00000A2201500B1801C00C0E01500E040130B3
:102E100010FA002012F0005014E600C016DC00701A
:102E200019D200501CC800501FBE007022B400B060
:102E300025AA00F028A000202C9600302F8C00102E
:102E4000328200A0347800F0366E00E038640080F2
:102E50003A5A00403B5500E03B5000F03C4600C071
:102E60003D3C00603E3200E03E2800303F1E0050F6
:102E70003F1900703F1400A03F0A00C03F0000D07F
:102E80003FF6FFE03FECFF00000A0B02090C0D0EBD
:102E9000080703040100000000000000000000001B
:102EA0000000000000000000000000000000000022
:102EB00000000012111000000000000000000000DF
:102EC0000000000000000000000000000050726FD1
:102ED00062696E67204661696C656400205A3A2019
:102EE0000020593A200042656420583A20003D3DB8
:102EF0006F6E55736572436F6E6669726D52657160
:102F000075697265643D3D00220A00556E6B6E6FF7
:102F1000776E20636F6D6D616E643A2022002042EF
:102F2000002050006F6B00204500205A00205900FF
:102F3000204D393220580020453A00205A3A0020CE
:102F4000593A00583A0020746F6F206C6F6E6720FA
:102F5000657874727573696F6E2070726576656ED0
:102F60007465640A0020636F6C6420657874727500
:102F700073696F6E2070726576656E7465640A00A1
:102F800043616E6E6F7420656E7465722073756236
:102F90006469723A20004D323520500A4D323400B7
:102FA000526573756D6500554920506175736500F4
:102FB0004E6F204D61746368203A00506755700071
:102FC0005067446F776E0049732046696C65200036
:102FD0004973204469722000476F5570446972003C
:102FE000486173204D656469610046696C656E6176
:102FF0006D652053656C6563746564004D313030D8
:103000003043004D313030300046696C616D656E83
:103010007420537461742030202D20330046696C75
:10302000616D656E7420537461742030202D2032E0
:103030000046696C616D656E742053746174203054
:10304000202D2031002046696C616D656E74205220
:103050006573706F6E7365204E6F00526573756D8A
:10306000652059657320647572696E672070726996
:103070006E74000A204E6F2046696C616D656E7437
:1030800000496E76616C6964204F7074696F6E00E0
:103090004D3530300053746F726520536574746918
:1030A0006E67730042656420504944205374617216
:1030B000746564004D3939390A4D32383050305317
:1030C00031363000424C546F756368205265736529
:1030D00074004D3530320A4D35303000496E697418
:1030E00020454550524F4D00486F74656E64205026
:1030F0004944205374617274656400456E676C695D
:10310000736820416C726561647920536574004373
:1031100068696E657365204E6F7420537570706FAB
:103120007274656400496E4C616E6743686F6963D1
:1031300065000A202A2A2A7265636461742E64611C
:1031400074615B305D203D004732380A47312046CC
:1031500031303030205A313000556E737570706FD9
:1031600072746564204F7074696F6E2053656C656E
:10317000637465640047323652323535004D31395B
:10318000305335350A4732380A4732390A4D343020
:10319000300A4D313034533231350A4732380A4D16
:1031A000313039533231350A4D34323053310A47D8
:1031B00031583130305931303046353030300A47AF
:1031C000315A300A4D3530300A4D31313720536590
:1031D00074205A204F66667365740047312046316B
:1031E000303030205A302E30004732380A473120F4
:1031F0004631303030205A302E30004D35303000DE
:103200005A204F6666736574203A202573004D3549
:103210003030005A204F6666736574203A2025735B
:10322000004732380A473146313530305A302E3077
:10323000004732385A0A473146313530305A302E3D
:1032400030004D383400473146313030305A302E5E
:1032500030004732380A473146313030305A302E4C
:1032600030004D616E75616C53657454656D70000E
:103270005A204F6666736574203A20257300537494
:103280006F70205472696767657265640053746F6C
:1032900070204E6F0053746F705072696E740048E6
:1032A000616E646C6520446174612041646A757369
:1032B0007420322053657474696E6720536372659D
:1032C000656E200048616E646C6520446174612005
:1032D0005072696E7446696C65203320536574744E
:1032E000696E672053637265656E200048616E6485
:1032F0006C652044617461205072696E7446696C1B
:103300006520322053657474696E6720536372655B
:10331000656E20004D38340048616E646C65204451
:10332000617461205072696E7446696C6520506FDB
:1033300073740048616E646C652044617461205050
:1033400072696E7446696C652050726500426567EB
:10335000696E537769746368003D3D204368656317
:103360006B6B65793D3D007265636461742E6164C9
:103370006472203D3D007265636461742E64617403
:10338000615B305D203D3D00776169747761792034
:103390003D3D0020202A2A2A2A2A2A2A5254535FF5
:1033A00048616E646C65446174612A2A2A2A2A2A5B
:1033B0002A2A2000526573656E643A2000000022BC
:1033C00000250028002B002E0031003400020100EF
:1033D00000050108010B0100002100240027002A3C
:1033E000002D003000330001010000040107010A34
:1033F0000105050505070508080808020202020A7A
:103400000A08080404040401010101010101010387
:1034100003030303030303040707070C0C0C0C0C42
:103420000C0C0C0202020206060606060606060B35
:103430000B0B0B0B0B0B0B010210202008081020AC
:103440004010204080020102010804020101020430
:1034500008102040808040201008040201800402EF
:103460000180402010080402010804020101020446
:1034700008102040800102040810204080544D3381
:103480004420453520506C75732052656164792E57
:10349000005072696E74696E672E2E2E005072692C
:1034A0006E7420506175736564006E6F746966692F
:1034B000636174696F6E20005049442054756E65D5
:1034C0002046696E697368656400CA00FA001124B9
:1034D0001FBECFEFD1E2DEBFCDBF00E00CBF14E0D6
:1034E000A0E0B2E0E4E9FFE502E00BBF02C0079014
:1034F0000D92A831B107D9F726E1A8E1B4E001C0E7
:103500001D92A733B207E1F71AE1C6E6DAE100E05F
:1035100006C021970109802FFE010F94F72BC536B5
:10352000D10780E00807A9F70F946F190D94B82F01
:103530000C9400009F92AF92BF92CF92DF92EF92D5
:10354000FF920F931F93CF93DF9300D01F921F9290
:10355000CDB7DEB7EDE5FBE10027BB27462F572FA0
:10356000A82FAA2341F4A52F542FB85FAA2319F43A
:10357000A52F5527B85FA03138F45295A295452F55
:103580004F70507FA42BBC5FA03428F4550FAA1FA6
:10359000550FAA1FBE5FA03818F4550FAA1FB39588
:1035A000550FAA1FEA0FF01F449151E0AA27B85007
:1035B00081F1C8F0B0FF02C0440F551FB1FF04C035
:1035C000440F551F440F551FB2FF06C05295429538
:1035D000142F1F70407F512BB3FF1BC0A52F542FFA
:1035E00044270C94091BB195B0FF02C0559547952F
:1035F000B1FF04C05595479555954795B2FF05C055
:103600005295407F4295452B5F70B3FF02C0452F16
:103610005527DD24CC24BB24B2E0649FD018C10818
:10362000B00AB00B749FC018B108B00B849FB018DB
:10363000B109659FC018B108B00B759FB018B109EA
:10364000859FB0196A9FB018B1097A9FB0194D9D36
:10365000A12C99243327992722275D9DA00C911C2A
:10366000301F901F201FAD9D900C311D901F201FFB
:103670004C9DA00C911C301F901F201F5C9D900C36
:10368000311D901F201FAC9D300D911D201F4B9DA3
:10369000900C311D901F201F5B9D300D911D201F30
:1036A000AB9D900D211D4B9F300D911D201F5B9FE9
:1036B000900D211DAB9F200DB1E0BB24CC24DD2457
:1036C000639FD018C108B00AB00B739FC018B1082F
:1036D000B00B839FB018B109699FC018B108B00B37
:1036E000799FB018B109899FB019629FB018B109CC
:1036F000729FB019D61AC70AB80A20F0B1E03B0F82
:10370000901F201F1124792F632F90E0822F0F909C
:103710000F900F900F900F90DF91CF911F910F910D
:10372000FF90EF90DF90CF90BF90AF909F90089563
:10373000AF92BF92CF92DF92EF92FF920F931F93BF
:10374000CF93DF93C5E4DCE004E019E085E5A82E23
:103750008CE0B82EC12CD12C7601C394699179915B
:10376000899199910F943525288939894A895B89EE
:103770000F9496250F94732DF801619371938193A3
:1037800091938F01C616D706E806F90610F46B016F
:103790007C01AC16BD0611F76FEF7FEFCB01A701DF
:1037A00096010F94742B20931409309315094093BC
:1037B000160950931709DF91CF911F910F91FF9038
:1037C000EF90DF90CF90BF90AF900895CF92DF92AF
:1037D000EF92FF9280911008882309F457C0C0909F
:1037E0000C08D0900D08E0900E08F0900F0820E033
:1037F00030E0A901C701B6010F943025882309F4F0
:1038000045C020E030E040E05FE3C701B6010F941F
:1038100096259B01AC010F9496252BED3FE049E4E2
:1038200050E40F9496259B01AC0160E070E080E8C5
:103830009FE30F94FA2C6B017C01C092410CD09253
:10384000420CE092430CF092440C6091750270912E
:103850007602072E000C880B990B0F9437252AE06F
:1038600037ED43E25CE30F949625A70196010F9490
:103870009625609371027093720280937302909305
:103880007402FF90EF90DF90CF900895C12CD12C5F
:1038900080E8E82E8FE3F82ED0CF0F931F93CF93BD
:1038A000DF9350E0FC01E40FF51F8081440F551FAA
:1038B000440F551F4A545A4FEA01882329F1888141
:1038C0009981AA81BB81EB01088119812A813B8101
:1038D0000097A105B10569F40C591F4F2F4F3F4FB9
:1038E000DA010D931D932D933C9313978FEF8083F3
:1038F00006C0081B190B2A0B3B0B37FDF7CFDF91D6
:10390000CF911F910F910895188219821A821B82FC
:10391000F6CFCF93DF9324E0829FC0011124EC0106
:10392000C951D74FFC01E35EF74F8F5E974FDC0123
:103930002D913D914D915C91608171818281938146
:103940000F94002C688379838A839B83DF91CF91C6
:1039500008958091B1059091B205A091B305B09101
:10396000B4058093410290934202A0934302B09326
:1039700044028091AF059091B005909378028093B6
:10398000770208958091410290914202A0914302F2
:10399000B09144028093B1059093B205A093B30512
:1039A000B093B40580917702909178029093B0051E
:1039B0008093AF0584E690E090937802809377023D
:1039C00008958091901290919112891B877089F4CB
:1039D0008091980D81110DC080918D0C90918E0C6D
:1039E000892B39F481E09091BF06911103C080E0EA
:1039F000089581E00895CF93DF93DB01F9019C9155
:103A00009130C1F0943080F094509C938830D1F480
:103A100080819181009771F0019791838083480F95
:103A2000591FEA01188206C08C3539F49C5F9C93BB
:103A3000943041F4DF91CF9108958B3339F781E0D1
:103A40008C93F8CF20813181B9016F5F7F4F7183F3
:103A50006083420F531FEA018883808191818F35F3
:103A600091056CF7E7CF0F931F9381E00091341419
:103A70001091351420913614309137144091301440
:103A8000509131146091321470913314041715075A
:103A90002607370708F480E01F910F91089590E002
:103AA00080E00895282F90910B08833021F495FD34
:103AB0000FC094FD0FC0892F90E0B0E0A0E004C0DB
:103AC000B695A795979587952A95D2F78170089511
:103AD00081E0089580E00895FC01659175918591DC
:103AE000949108958F929F92AF92BF92CF92DF925E
:103AF000EF92FF92CF93DF93EC018090E3089090D8
:103B0000E408A090E508B090E60820E030E0A901C4
:103B1000C501B4010F943025882309F454C0C8802E
:103B2000D980EA80FB80A7019601C501B4010F94FA
:103B3000302518160CF04CC02091DB083091DC08C1
:103B40004091DD085091DE08C701B6010F94302581
:103B5000882331F1C092DB08D092DC08E092DD08C6
:103B6000F092DE082091DF083091E0084091E108F2
:103B70005091E208688179818A819B810F94962512
:103B80009B01AC0160E070E080E89FE30F94FF2BA5
:103B900060930F02709310028093110290931202AF
:103BA00060910F02709110028091110290911202A7
:103BB000DF91CF91FF90EF90DF90CF90BF90AF90CB
:103BC0009F908F90089560E070E080E89FE3F0CFD1
:103BD00060E070E0CB01ECCFCF92DF92EF92FF92EA
:103BE000CF93DF93EC01CC80DD80EE80FF8027E176
:103BF00037EB41ED58EBC701B6010F94602E87FDFE
:103C000023C023E030E044EB53E4C701B6010F9436
:103C100030251816CCF0C880D980EA80FB8027E1D7
:103C200037EB41ED58EBC701B6010F94602E87FDCD
:103C30000BC0C1E023E030E044EB53E4C701B60120
:103C40000F94302518160CF4C0E08C2FDF91CF9123
:103C5000FF90EF90DF90CF9008952FEB280F2A313F
:103C600008F047C0E22FF0E080914B0590914C05A1
:103C7000A0914D05B0914E0504C0B695A7959795B6
:103C800087952A95D2F780FD02C081700895E35D83
:103C9000FA4FE081EE2341F180919D0790919E07BC
:103CA000E80FF92FF11D808190ED980F9A3030F0D8
:103CB0008E3251F4818180538A3098F4F0931C0540
:103CC000E0931B0581E008958D3211F08B3249F4A9
:103CD000818190ED980F9A3088F38E3211F48281B1
:103CE000EACFF0E0E0E0EACF10921C0510921B054D
:103CF000E9CF80E008950E942D1E882341F081E0E5
:103D000020911B0530911C05232B09F480E00895B8
:103D10008F929F92AF92BF92CF92DF92EF92FF92DB
:103D2000C090ED05D090EE05E090EF05F090F00525
:103D300020E030E0A901C701B6010F9430258823A7
:103D4000E1F1A701960160E070E080E89FE30F9445
:103D5000FA2C6B017C018090F1059090F205A09007
:103D6000F305B090F40520E030E0A901C501B401ED
:103D70000F943025882329F1A501940160E070E0BB
:103D800080E89FE30F94FA2CC092F404D092F504DB
:103D9000E092F604F092F7046093F8047093F9044B
:103DA0008093FA049093FB04FF90EF90DF90CF9004
:103DB000BF90AF909F908F900895C12CD12C760129
:103DC000CACF60E070E0CB01DFCF129A08955F9A0E
:103DD00080913F0C8E7F80933F0C8A9A80913F0C9C
:103DE0008D7F80933F0C8091080180958170809336
:103DF000060180913F0C8B7F80933F0C0C94E51E55
:103E0000269A2E9A0895833B21E0920714F083EBC3
:103E100091E09093F5118093F4110C9417FDE9E271
:103E2000F6E0108211821282138214820C9417FD24
:103E30004F925F926F927F928F929F92AF92BF92BA
:103E4000CF92DF92EF92FF920F931F93CF93DF9366
:103E5000EC012091E5053091E6054091E705509190
:103E6000E805688179818A819B810F94FF2B6B0122
:103E70007C012091E9053091EA054091EB055091D4
:103E8000EC056C817D818E819F810F94FF2B4B010E
:103E90005C01A70196016091030270910402809178
:103EA0000502909106020F943025882309F450C032
:103EB000C0920302D0920402E0920502F092060240
:103EC0002091F4043091F5044091F6045091F704E8
:103ED000C701B6010F9496252B013C010F94A22D2A
:103EE0006B017C0120E030E0A9010F94302587FDB3
:103EF00070C020E030E040E450E4C701B6010F9408
:103F0000602E18162CF4C12CD12CC0E4EC2EFE2C03
:103F1000A7019601C301B2010F94FF2B6093EC043B
:103F20007093ED048093EE049093EF04C701B60103
:103F30000F946C2D6093EA04062E000C770B6F5FD4
:103F40007F4F6430710514F064E070E06093E80422
:103F5000D09101021091EA04A50194016091070239
:103F6000709108028091090290910A020F94302505
:103F7000811133C0D11381C02091D0043091D1047C
:103F80004091D2045091D3046091EC047091ED04FF
:103F90008091EE049091EF040F9496252091D40423
:103FA0003091D5044091D6045091D7040F94002C41
:103FB000DF91CF911F910F91FF90EF90DF90CF9005
:103FC000BF90AF909F908F907F906F905F904F9039
:103FD0000895C12CD12C76019BCF8092070290923C
:103FE0000802A0920902B0920A022091F8043091CE
:103FF000F9044091FA045091FB04C501B4010F94F7
:1040000096254B015C010F94A22D6B017C0120E0F1
:1040100030E0A9010F94302587FDF3C020E030E0A7
:1040200040E450E4C701B6010F94602E18162CF43A
:10403000C12CD12CB0E4EB2EFE2CA7019601C501BA
:10404000B4010F94FF2B6093F0047093F1048093FC
:10405000F2049093F304C701B6010F946C2D6093A2
:10406000EB04062E000C770B6F5F7F4F64307105F9
:1040700014F064E070E06093E904C091EB04D113A4
:1040800005C0809102028C1709F470C08091EA0487
:104090009091EB0490930202809301020C2E000C8D
:1040A000DD0B25E01203C0011124FC01EC0FFD1F04
:1040B000EE0FFF1FEE0FFF1FE955F84F20813181F2
:1040C000428153812093E4043093E5044093E60455
:1040D0005093E7040091E904002E000C110BFC0141
:1040E000E00FF11FEE0FFF1FEE0FFF1FE955F84F16
:1040F00060817181828193810F94FF2B6093E00432
:104100007093E1048093E2049093E3042091E80427
:1041100035E02303F0011124CE0FDF1FCC0FDD1F8C
:10412000CC0FDD1FC955D84F288139814A815B8169
:104130002093DC043093DD044093DE045093DF04CD
:10414000E00FF11FEE0FFF1FEE0FFF1FE955F84FB5
:1041500060817181828193810F94FF2B6093D804D9
:104160007093D9048093DA049093DB048090F00478
:104170009090F104A090F204B090F3042091E00438
:104180003091E1044091E2045091E304C501B4018F
:104190000F9496252091E4043091E5044091E604C3
:1041A0005091E7040F94002C6B017C01C092D40461
:1041B000D092D504E092D604F092D7042091D8048E
:1041C0003091D9044091DA045091DB04C501B40167
:1041D0000F9496252091DC043091DD044091DE049B
:1041E0005091DF040F94002CA70196010F94FF2B30
:1041F0006093D0047093D1048093D2049093D3043D
:10420000BBCEC12CD12C760118CFCF92DF92EF928A
:10421000FF92CF93DF93EC0108960E94721D6B0111
:104220007C0120E030E0A9010F94302520E030E04F
:10423000A901882359F0CE010E94181F9B01AC01EF
:10424000C701B6010F9496259B01AC01688579855D
:104250008A859B850F94FF2B688779878A879B8740
:10426000DF91CF91FF90EF90DF90CF9008952F9244
:104270003F924F925F926F927F928F929F92AF92F6
:10428000BF92CF92DF92EF92FF920F931F93CF9343
:10429000DF93D62FC72FFC0180809180A280B3804E
:1042A000C501B40120E831E541E050E00F94742BE2
:1042B000C9016DE671E00F94E32B6B017C01C50130
:1042C000B40120E13EE040E050E00F94742BCA01BD
:1042D000B90128E130E040E050E00F94742B362E15
:1042E000272E062F172F8CE3482E512C612C712C72
:1042F000C501B401A30192010F94742BB62EA72E11
:10430000CA01B901A30192010F94742BCB01C1140E
:10431000D10479F1AF92BF927F936F932F923F9226
:10432000FF92EF92DF92CF9284E697E19F938F9373
:10433000CF93DF930F94C7248DB79EB70E960FB619
:10434000F8949EBF0FBE8DBF8D2F9C2FDF91CF9114
:104350001F910F91FF90EF90DF90CF90BF90AF90A3
:104360009F908F907F906F905F904F903F902F9095
:104370000895E114F104C9F0AF92BF927F936F9357
:104380002F923F92FF92EF9284E597E19F938F9354
:10439000CF93DF930F94C724EDB7FEB73C960FB6CB
:1043A000F894FEBF0FBEEDBFCFCF012BB9F0AF9297
:1043B000BF927F936F932F923F9288E497E19F93F0
:1043C0008F93CF93DF930F94C7248DB79EB70A9630
:1043D0000FB6F8949EBF0FBE8DBFB6CF892BA9F044
:1043E000AF92BF927F936F9380E497E19F938F93F7
:1043F000CF93DF930F94C724EDB7FEB738960FB66F
:10440000F894FEBF0FBEEDBF9FCFAF92BF928CE37B
:1044100097E19F938F93CF93DF930F94C7240F90CF
:104420000F900F900F900F900F908ECFEF92FF9202
:104430000F931F93CF93DF93CDB7DEB78C01EDB60B
:10444000FEB60F947D2401962DB73EB7281B390B7D
:104450000FB6F8943EBF0FBE2DBF8DB79EB7019625
:10446000B8010F9476240E943AF90FB6F894FEBE74
:104470000FBEEDBEDF91CF911F910F91FF90EF9096
:1044800008958C38910514F08CE890E090938A118F
:10449000809389110C9491BEAB01BC0140933414FC
:1044A0005093351460933614709337148CE995E16A
:1044B0000C9449AF2F923F924F925F926F927F92EE
:1044C0008F929F92AF92BF92CF92DF92EF92FF9224
:1044D0000F931F93CF93DF93CDB7DEB760970FB6DF
:1044E000F894DEBF0FBECDBF8B876C87042F122FD1
:1044F000282F30E03E872D87462F50E05A87498786
:1045000085E0982E929EC001939E900D1124988B69
:104510008F87FA01E80FF91FEE0FFF1FEE0FFF1F45
:10452000E955F84F60817181828193819B01AC01D3
:104530000F94F22E882309F445C14B85400F6C85FA
:10454000610F949EC0011124E985FA85E80FF91FD7
:10455000EE0FFF1FEE0FFF1FE955F84FC080D1800F
:10456000E280F380040F909EA0011124E985FA8572
:10457000E40FF51FEE0FFF1FEE0FFF1FE955F84F79
:104580000081918082807380262F30E0EF85F8894A
:10459000E20FF31FEE0FFF1FEE0FFF1FE955F84F5D
:1045A00020807181798372817A8373817B83610F2B
:1045B00070E0EF85F889E60FF71FEE0FFF1FEE0F93
:1045C000FF1FE955F84FF88BEF87F081FC83EF85EB
:1045D000F889F181FD83EF85F889F281FE83EF850B
:1045E000F889F381FF83FC01E20FF31FEE0FFF1F39
:1045F000EE0FFF1FE955F84F20812887A180B28078
:104600006380FA01E60FF71FEE0FFF1FEE0FFF1F8B
:10461000E955F84F4080518032801381202F392D89
:10462000482D572D602F792D882D972D0F94F22E20
:10463000882321F000E0912C812C712C9601A70198
:10464000B601C7010F94F22E882321F0C02ED92C79
:10465000E82CF72C2C813D814E815F816C817D811E
:104660008E819F810F94F22E882321F01C821D825F
:104670001E821F82222D39814A815B81622D7981C0
:104680008A819B810F94F22E882339F02C803D8102
:1046900039834E814A835F815B839201432D512F81
:1046A000B201832D912F0F94F22E882321F0412CFB
:1046B000512C312C10E028853A2D4B2D562D688534
:1046C0007A2D8B2D962D0F94F22E882321F048867B
:1046D000A52CB32C612E85E02D853E85829FF001AF
:1046E000839FF00D112449855A85E40FF51FEE0FC5
:1046F000FF1FEE0FFF1FE955F84FFA87E987960174
:10470000A701B601C7010F94002C202F392D482D89
:10471000572D0F94FF2B6B017C01222D39814A818B
:104720005B81622D79818A819B810F94002C2C8181
:104730003D814E815F810F94FF2B9B01AC01C7012E
:10474000B6010F94002C6B017C0128853A2D4B2D6E
:10475000562D68857A2D8B2D962D0F94002C920165
:10476000432D512F0F94FF2B9B01AC01C701B601C4
:104770000F94002C20E030E040E450E40F94FA2C39
:10478000E985FA8560837183828393836C858B8549
:1047900060960FB6F894DEBF0FBECDBFDF91CF910C
:1047A0001F910F91FF90EF90DF90CF90BF90AF904F
:1047B0009F908F907F906F905F904F903F902F9041
:1047C0000C94CDF760960FB6F894DEBF0FBECDBF48
:1047D000DF91CF911F910F91FF90EF90DF90CF90DD
:1047E000BF90AF909F908F907F906F905F904F9011
:1047F0003F902F90089580911B0590911C05009784
:1048000031F04AE050E070E060E00D944B2360E04E
:1048100070E0CB01089580911B0590911C050097D5
:1048200031F04AE050E070E060E00D941D2260E05D
:1048300070E0CB010895CF93DF93EB010E947B1EC4
:10484000882319F00E940B24EB01CE01DF91CF9158
:1048500008950E940B2497FD0CC00E940B246F3F0B
:1048600071058105910509F034F40E940B24862F0F
:10487000089580E008958FEF0895CF93C62F0E948A
:104880007B1E882319F0CF910C9429248C2FCF9173
:10489000089580911B0590911C05892B41F00E9481
:1048A000292491E0811101C090E0892F089591E0C1
:1048B000FCCFCF93DF93C82FD62F0E947B1E882377
:1048C00021F0DF91CF910C9449248C2F0E942D1E52
:1048D000811101C08D2FDF91CF9108950E940B248B
:1048E000CB010895CF93DF93EB010E947B1E8823B9
:1048F00021F0DF91CF910C946E24CE01DF91CF9106
:1049000008950F931F93CF9380911B0590911C05E1
:104910000097E9F0FC018F01C1912C2F2F7D81F0D0
:10492000C53411F0C536B9F7F801108270E060E0C7
:104930000F94BF20F801C083CF911F910F9108956C
:1049400070E060E0CF911F910F910D94BF2060E067
:1049500070E0CB01F1CFCF92DF92EF92FF926A012C
:104960007B010E947B1E882331F0FF90EF90DF9047
:10497000CF900C948124C701B601FF90EF90DF9097
:10498000CF9008954F925F926F927F928F929F92F5
:10499000AF92BF92CF92DF92EF92FF921F93CF938D
:1049A000DF9300D01F92CDB7DEB719821A821B8227
:1049B0001C82CE0101964C018BE8C82E87E0D82ED0
:1049C00091E6E92E92E0F92E27EEA22E28E0B22EF3
:1049D00010E088E5810F0E947B1EF40181934F0156
:1049E000882309F4E0C00E9481242B013C01812F1F
:1049F0000E94521D882309F4CCC0F7012081318127
:104A000042815381C301B2010F94002CF6016083EF
:104A10007183828393831F5FF4E0CF0ED11C84E007
:104A2000E80EF11C94E0A90EB11C133091F685E458
:104A30000E947B1E8C83882309F4C0C00E948124BD
:104A40006B017C0183E00E94521D882371F020914C
:104A50006D0230916E0240916F0250917002C70159
:104A6000B6010F94002C6B017C01C0929707D09285
:104A70009807E0929907F0929A078091E4058823BD
:104A800059F18091381482FF27C08C81882321F14D
:104A90008981811103C08A818823F1F02DEC3CECDF
:104AA0004CE45DE3609132087091330880913408E2
:104AB000909135080F94002C9B01AC016091690224
:104AC00070916A0280916B0290916C020F94602E3B
:104AD000181614F40E9413F740E050E0BA0186E47F
:104AE0000E94AB2420E030E0A9010F94602E18163C
:104AF00084F40E94812420E030E040E752E40F94E7
:104B0000FA2C609341027093420280934302909387
:104B100044028091FD0B83FD28C08091AA06882362
:104B200021F120916D0230916E0240916F025091FF
:104B30007002609197077091980780919907909102
:104B40009A070F94FF2B2091B7063091B806409139
:104B5000B9065091BA060F94002C6093B706709373
:104B6000B8068093B9069093BA060F900F900F90F5
:104B70000F90DF91CF911F91FF90EF90DF90CF903A
:104B8000BF90AF909F908F907F906F905F904F906D
:104B90000895F5012081318142815381C301B20121
:104BA0000F94FF2B33CFF70180819181A281B381D4
:104BB000F60180839183A283B3832DCF80916D0210
:104BC00090916E02A0916F02B0917002809397074E
:104BD00090939807A0939907B0939A074ECFCF92DE
:104BE000DF92EF92FF926B017C0183E3C816D10440
:104BF000E104F10470F082E3C81AD108E108F10879
:104C000062E370E080E090E00E94D8FC0E940BC25A
:104C1000ECCFC701B6010E94D8FCFF90EF90DF9067
:104C2000CF900C940BC2CF92DF92EF92FF920F9332
:104C30001F93CF93DF936B017A01EC01C055DB4FDB
:104C400028813CE0389F8001399F100D112427FFF7
:104C500024C0FB011182108288818F5F8883888144
:104C60009801280F311D87FD3A95C90120917B12CB
:104C7000F6012817190629F024F088818C300CF4ED
:104C80003CC080819181049680349C4908F475C0B1
:104C9000F60180819181049672C088819801280F65
:104CA000311D87FD3A95C90120917B1228171906FD
:104CB00099F294F28881A801480F511D87FD5A95F9
:104CC000FA01EE0FFF1FE40FF51FED5CFD4E808132
:104CD00087FFC2CF8881F801E80FF11D87FDFA95A3
:104CE000CF01EE0FFF1FE80FF91FED5CFD4E808135
:104CF00060E08F770E9476FBAFCF80819181288121
:104D0000A801420F511D27FD5A959A01FA01EE0F95
:104D1000FF1FE20FF31FED5CFD4E21813281820FF8
:104D2000931FF7019183808388819801280F311D9B
:104D300087FD3A95F901EE0FFF1FE20FF31FED5CBF
:104D4000FD4E808187FF20C08881080F111D87FDDF
:104D50001A95F801EE0FFF1FE00FF11FED5CFD4EFD
:104D6000808161E08F77DF91CF911F910F91FF904C
:104D7000EF90DF90CF900C9476FB80E49CE9F701F4
:104D8000918380838FEF8883DF91CF911F910F9163
:104D9000FF90EF90DF90CF9008950F931F93CF93E4
:104DA000DF9309E51CE0CDE6D1E1F80121913191D5
:104DB000419151918F0160E070E080E89FE30F9492
:104DC000FA2C6993799389939993F1E1CD37DF07B1
:104DD00061F70E9452F5DF91CF911F910F910C94D2
:104DE000981BCF92DF92EF92FF92CF93DF932091A7
:104DF000400C222329F1EC0108960E94721D6B01E0
:104E00007C0120E030E0A9010F94302520E030E063
:104E1000A901882359F0CE010E94181F9B01AC0103
:104E2000C701B6010F9496259B01AC016885798571
:104E30008A859B850F94002C688779878A879B8752
:104E4000DF91CF91FF90EF90DF90CF9008952F9258
:104E50003F924F925F926F927F928F929F92AF920A
:104E6000BF92CF92DF92EF92FF920F931F93CF9357
:104E7000DF93CDB7DEB76C970FB6F894DEBF0FBEE9
:104E8000CDBF8C015B015A834983FC01EA5BFF4F74
:104E9000208131814281538129873A874B875C8702
:104EA000CA01B9010F9435256B017C01D5012D9103
:104EB0003D914D915C910F9496250F94DE2C2B0122
:104EC0003C01E981FA812081318142815381C7010E
:104ED000B6010F9496250F94DE2C4B015C01C301A3
:104EE000B2010F94732D698B7A8B8B8B9C8B6837F7
:104EF00071058105910540F428E730E040E050E07D
:104F0000298B3A8B4B8B5C8BC501B4010F94732DAD
:104F10006D877E878F87988B68377105810591052E
:104F200040F448E750E060E070E04D875E876F87AF
:104F3000788BF801EE5AFF4F408051806280738079
:104F4000C301B2010F94372569837A838B839C83D5
:104F500069897A898B899C890F9435256D8B7E8B25
:104F60008F8B988F20E030E0A90169817A818B8155
:104F70009C810F943025882309F4E1C1A701960193
:104F8000C701B6010F9496254B015C012D893E891E
:104F90004F89588DCA01B9010F9496259B01AC0128
:104FA000C501B4010F94FF2B4B015C0129813A81AB
:104FB0004B815C81CA01B9010F94002C9B01AC01AB
:104FC000C501B4010F94FA2C0F94DE2C0F94732DAD
:104FD0006D837E838F83988766277727CB0164193B
:104FE0007509860997090F9437254B015C016D857A
:104FF0007E858F8598890F9435252B013C0120E013
:1050000030E0A901C501B4010F943025882309F4CB
:105010009AC1A3019201C301B2010F949625698F31
:105020007A8F8B8F9C8FA7019601C701B6010F94D1
:1050300096259B01AC01698D7A8D8B8D9C8D0F948B
:10504000FF2B6B017C01A5019401C501B4010F94F4
:10505000002C9B01AC01C701B6010F94FA2C0F94F0
:10506000A22DD80195968D909D90AD90BC9098976B
:10507000750164012D813E814F815885C21AD30A82
:10508000E40AF50A0F94732DC61AD70AE80AF90A3A
:10509000F7FE8EC02D893E894F89588DCA01B9010E
:1050A0000F9496256B017C0129813A814B815C81AB
:1050B000CA01B9010F94002C69877A878B879C8776
:1050C00020E030E0A90169817A818B819C810F9475
:1050D0003025882309F43BC1C501B4010F9435255F
:1050E00029853A854B855C850F949625A701960105
:1050F0000F94FF2B6D837E838F839887A30192018A
:10510000C301B2010F9496259B01AC016D817E8194
:105110008F8198850F94002C2B013C0120E030E01A
:1051200040E850E469817A818B819C810F949625B7
:105130009B01AC01C301B2010F94FA2C0F94DE2C39
:105140002B013C0120E030E0A9010F94602E1816DD
:105150001CF0412C512C3201C301B2010F94732D6C
:105160006D837E838F83988786169706A806B90677
:1051700020F48D829E82AF82B8866D817E818F8180
:1051800098850F94352529853A854B855C850F9444
:105190009625A70196010F94002C0F94AE2E0F9424
:1051A000732D69877A878B879C87C12CD12C7601D8
:1051B00069857A858B859C8529893A894B895C89A3
:1051C000621B730B840B950B0F94352529813A8153
:1051D0004B815C810F94FA2C20E034E244EF59E4D7
:1051E0000F9496250F94732D4B015C0169857A8588
:1051F0008B859C852D853E854F855889621B730B59
:10520000840B950B0F94352529813A814B815C8164
:105210000F94FA2C20E034E244EF59E40F949625E1
:105220000F94732D2B013C013FE683169104A104DA
:10523000B10408F090C0F401EE0FFF1FEE0FFF1F46
:10524000EF55F64E85919591A591B4918983292EBC
:105250003A2EBD8B4FE6441651046104710408F0E8
:1052600083C0F201EE0FFF1FEE0FFF1FEF55F64E4A
:1052700045915591659174919A01CB014D815E8163
:105280006F817885D80199964D935D936D937C934A
:105290009C974C0D5D1D6E1D7F1DF80145A756A7FF
:1052A00067A770ABE65BFF4F49895A896B897C8998
:1052B0004083518362837383D5968D929D92AD9284
:1052C000BC92D897F80141AE52AE63AE74AEFD9673
:1052D00049814083218232825D89538334962083C1
:1052E00031838283938369857A858B859C85D1966A
:1052F0006D937D938D939C93D4973D962D853E859C
:105300004F85588920833183428353836C960FB62F
:10531000F894DEBF0FBECDBFDF91CF911F910F91EB
:10532000FF90EF90DF90CF90BF90AF909F908F90C5
:105330007F906F905F904F903F902F90089560E026
:1053400070E0CB0141CE60E070E0CB0188CE60E040
:1053500070E0CB01F3CEC501B4010E949A1A6983B3
:10536000272E382E9D8B76CFC301B2010E949A1A48
:105370009B0184CF8091901290919112891B87702C
:1053800019F490E080E0089590918D12992351F0E6
:10539000833030F48FEF890F19F080938D12F1CFA5
:1053A00010928D12809191122CE5829FC0011124E0
:1053B000835E964FFC01208120FDE3CF2091911266
:1053C0002F5F277020938E123091911220918F12AF
:1053D000321304C020918E1220938F120895909161
:1053E0006F0081E091FD02C080E0089590916F0010
:1053F0009D7F90936F00089580FF04C090913F0CB3
:1054000090FD8E7F81FF05C090913F0C969590FD99
:105410008D7F82FF06C090913F0C9695969590FDEA
:105420008B7F08958F929F92AF92BF92CF92DF921F
:10543000EF92FF92CF93DF9320914502222309F44C
:105440009EC0EC018091B505C82ED12CF12CE12C29
:1054500080FF2CC08090470290904802A0904902A3
:10546000B0904A02288139814A815B81C501B4012B
:105470000F94602E181624F488829982AA82BB8227
:105480008090530290905402A0905502B090560222
:10549000288139814A815B81C501B4010F9430258F
:1054A00087FF04C088829982AA82BB82D701C60185
:1054B000B695A7959795879580FF2CC080904B0255
:1054C00090904C02A0904D02B0904E022C813D81F4
:1054D0004E815F81C501B4010F94602E181624F42B
:1054E0008C829D82AE82BF8280905702909058023B
:1054F000A0905902B0905A022C813D814E815F816B
:10550000C501B4010F94302587FF04C08C829D82B1
:10551000AE82BF8282E0F694E794D794C7948A95CE
:10552000D1F7C0FE2CC0C0904F02D0905002E09046
:105530005102F0905202288539854A855B85C70162
:10554000B6010F94602E181624F4C886D986EA8610
:10555000FB86C0905B02D0905C02E0905D02F09010
:105560005E02288539854A855B85C701B6010F949F
:10557000302587FF04C0C886D986EA86FB86DF917E
:10558000CF91FF90EF90DF90CF90BF90AF909F9022
:105590008F900895CF92DF92EF92FF920F931F9317
:1055A000C12CD12C76018C012DE632E049E652E087
:1055B00065E672E081E692E00E944EF41F910F9141
:1055C000FF90EF90DF90CF9008950C9452F580916A
:1055D000A205659B6EC080618093A2059091030136
:1055E0008091A20591FF67C080628093A20580919F
:1055F000A2054B9B62C084608093A2058091A205A6
:105600009091A105981709F45AC092E09093A005D3
:105610008093A1058091BC06811105C080919B07F4
:10562000882309F459C08091090680FF10C0809139
:10563000BD0680FD0CC080919F0584FF08C080914D
:10564000FF0680618093FF0680E00E946BC6809118
:105650000906869580FF11C08091BD06869580FD64
:105660000CC080919F0585FF08C08091FF06806275
:105670008093FF0681E00E946BC6809109068695A3
:10568000869580FF29C08091BD068695869580FF0E
:1056900023C080919B078823F9F080919F0582FFAA
:1056A0001BC08091FF0684608093FF0682E00C940B
:1056B0006BC68F7E91CF8F7D98CF8B7F9DCF809152
:1056C000A005882309F4A6CF81508093A0058111FD
:1056D000A1CF90939F059ECF08958091BC06811124
:1056E00004C080919B07882331F062E070E080E085
:1056F00090E00C94EF2508950F931F9380912B1148
:10570000813019F50E940BFD0091BE051091BF0577
:105710002091C0053091C105601B710B820B930B6A
:1057200028EE33E040E050E00F94742B6091C20506
:105730007091C3058091C4059091C505620F731FD8
:10574000841F951F1F910F9108956091C605709158
:10575000C7058091C8059091C905D6CF10922B112D
:105760001092BE051092BF051092C0051092C1059F
:105770001092C6051092C7051092C8051092C9056F
:105780001092C2051092C3051092C4051092C5056F
:105790000895CF92DF92EF92FF92CF93DF93C62FBF
:1057A000FC01C080D180E280F38020E030E0A901DC
:1057B000C701B6010F94302520E030E0A90187FD34
:1057C00014C020E030E048EC52E4C701B6010F9469
:1057D000602E24E630E040E050E0181634F0C701B7
:1057E000B6010F946C2D9B01AC01C230A0F4D0E047
:1057F000C85ED64FAFEFB0E00F94B52B24E630E093
:1058000040E050E00F94962B2F3F310519F010F037
:105810002FEF30E02883DF91CF91FF90EF90DF9062
:10582000CF9008958091090180FD06C080913814C1
:1058300083FB882780F9089580E00895CF92DF9256
:10584000EF92FF92FC01C080D180E280F38066304D
:1058500019F510922E0610922F0610923006109213
:105860003106109232060E9491BE20E030E0A9017C
:10587000C701B6010F94302587FF1DC0C12CD12C64
:105880007601C701B6010F946D2ECB01FF90EF900A
:10589000DF90CF900C9441220E940F1F20E030E057
:1058A000A901C701B6010F94302587FF15C0C12C8F
:1058B000D12C760122C020E030E04CE053E4C70157
:1058C000B6010F94602E1816E4F6C12CD12C9CE082
:1058D000E92E93E4F92ED5CF20E030E849ED53E4EA
:1058E000C701B6010F94602E18163CF4C12C80E855
:1058F000D82E89EDE82E83E4F82EC701B6010F9467
:105900006D2ECB01FF90EF90DF90CF900C94031F92
:1059100090913F0C977081E0973009F080E00895F6
:1059200020919D0520FF14C020E83EE3629FA00166
:10593000639F500D729F500D1124CA019695879553
:1059400096958795009731F08A950000E9F70895BC
:105950000C94EF250895CF93DF931092FE0B1092D5
:10596000910C1092930C1092920C10929C05109234
:105970009B05CFEFDFEF8091381485FD07C00E94B3
:10598000AAAAD093B712C093B612F5CF8FEF9FEFAC
:105990009093B7128093B612DF91CF9108958F92B2
:1059A0009F92AF92BF92CF92DF92EF92FF920F93AE
:1059B0001F93CF93DF931092500510924F052FE362
:1059C00020934A0510924905109248051092470508
:1059D00010924B0510924C0510924D0510924E05F9
:1059E0009C01F90190812F5F3F4F9032D1F39E349B
:1059F000C9F4818190ED980F9A3020F08D3211F02A
:105A00008B3281F432969F012F5F3F4F808180530C
:105A10008A3008F47BC09F012F5F3F4F8081803226
:105A200009F476C0F0939E07E0939D078F010F5F06
:105A30001F4FC0816AE270E0C8010F944E2F00979B
:105A400031F0FC01319780818032E1F31182CD3455
:105A500029F0C43519F0C73409F04BC0F801808132
:105A60000F5F1F4F8032D1F380538A3008F041C05E
:105A7000C0934A0530E020E04AE0DF011196429FE2
:105A8000C001439F900D11249C0120533109808156
:105A9000280F311D87FD3A95818190ED980F9A303E
:105AA000C8F130934905209348058E3261F432964F
:105AB00090E04AE0DF0131968C9150ED580F5A305A
:105AC00058F190934705CD01DC0101964C9140328D
:105AD000D9F3CD3489F52E31310539F018F5273158
:105AE000310519F02C31310539F5B0935005A093EB
:105AF0004F05DF91CF911F910F91FF90EF90DF90B5
:105B0000CF90BF90AF909F908F900895F9017BCF79
:105B1000F90181CFFD01B1CF949F800D112490ED4B
:105B2000980FC8CF2537310538F027373105E8F20F
:105B3000203A83E03807C9F2D0919D0740E050E059
:105B4000BA0110E000E0C12CD12C7601C394FD0114
:105B500031968C91882309F47FC08132E1F4CD34F1
:105B6000D1F420323105B9F440934B0550934C05E4
:105B700060934D0570934E05F0935005E0934F05EB
:105B800063E270E0CF010F944E2F009709F4B1CF7C
:105B9000FC011082AECF81548A3108F058C0DF0179
:105BA0009D91903291F0A0EDA90FAA30E8F09E32BD
:105BB00071F4918190539A30B8F00115110519F4E0
:105BC0008F010150110990E013C0FD01E8CF9D3213
:105BD00011F09B3291F79181A0EDA90FAA3020F02E
:105BE0009E3259F79281E6CF9E2F9D1B309759F335
:105BF000A82FB0E04601570104C0880C991CAA1CCC
:105C0000BB1C8A95D2F7482959296A297B29A35DAB
:105C1000BA4F9C9380818154DF018A3108F497CF79
:105C2000DF018191882309F492CF90ED980F9A308B
:105C3000B8F393ED980F923098F38B3289F3CD013E
:105C40000196EC91E03209F082CFDC01F8CF01152A
:105C5000110501F78D01DECF1093500500934F051C
:105C600040934B0550934C0560934D0570934E0542
:105C700040CF4F925F926F927F928F929F92AF929E
:105C8000BF92CF92DF92EF92FF92CF93DF9300D03B
:105C900000D01F921F92CDB7DEB75C01DB01CD9023
:105CA000DD90ED90FC90E0918B12F0918C12FE83D0
:105CB000ED8384819581A681B78189839A83AB83A3
:105CC000BC839C01AD01C701B6010F94FF2B2B01D2
:105CD0003C01F50180809180A280B380AD81BE81BE
:105CE0008D919D910D90BC91A02D8D839E83AF834E
:105CF000B88727E137EB41ED58EBC301B2010F94B0
:105D0000602E87FDD1C023E030E044EB53E4C301B3
:105D1000B2010F94302518160CF4C6C02D813E81B7
:105D20004F815885C501B4010F94FF2B2B013C0115
:105D300027E137EB41ED58EB0F94602E87FDB4C09F
:105D400023E030E044EB53E4C301B2010F9430256B
:105D500018160CF4A9C020E030E0A9016D817E8105
:105D60008F8198850F94002C2B013C0120E030E0BE
:105D700040E450E40F94302587FF05C0412C512C9E
:105D800030E4632E762C27E137EB41ED58E3C30175
:105D9000B2010F94FF2B9B01AC01C501B4010F941C
:105DA000602E87FD81C020E030E044EB53E46D813C
:105DB0007E818F8198850F94002C2B013C0120E07F
:105DC00030E842EB53E40F94602E18163CF4412C5B
:105DD00020E8522E22EB622E23E4722E27E137EBCD
:105DE00041ED58E3C301B2010F94002C9B01AC01BB
:105DF000C501B4010F94302518160CF455C020E0ED
:105E000030E0A90169817A818B819C810F94002CFB
:105E10004B015C0120E030E040EE51E40F9430256E
:105E200087FF06C0812C912C90EEA92E91E4B92E0B
:105E300027E137EB41ED58E3C501B4010F94FF2B87
:105E40009B01AC01C701B6010F94602E87FD2CC0E9
:105E500020E030E044EB53E469817A818B819C81BE
:105E60000F94002C4B015C0120E030E046EA53E443
:105E70000F94602E181634F4812C912C86EAA82EEB
:105E800083E4B82E27E137EB41ED58E3C501B401B7
:105E90000F94002C9B01AC01B1E0B983C701B6019E
:105EA0000F94302518160CF41982898128960FB6A4
:105EB000F894DEBF0FBECDBFDF91CF91FF90EF9082
:105EC000DF90CF90BF90AF909F908F907F906F901A
:105ED0005F904F900895E9E2F8E082EBDF011D92B8
:105EE0008A95E9F708958091E405811104C00E9424
:105EF0006B2F0C940BB88091381482FD0C9413F71F
:105F0000089580912908882361F09091DA08891317
:105F100008C08091381483FF04C087E698E00C9491
:105F2000D5B680E00895FC01238121110C940AB3B9
:105F30000895EFE6F0E08081826080830895CF923B
:105F4000DF92EF92FF92CF93DF93C82F0E94EF2949
:105F500094E0C99FE0011124FE01E95EF94FC08081
:105F6000D180E280F38081110E94992FC359DE4EC7
:105F7000C701B6010F943725288139814A815B8199
:105F80000F949625DF91CF91FF90EF90DF90CF9007
:105F900008958F929F92AF92BF92CF92DF92EF922D
:105FA000FF921F93CF93DF93CDB7DEB760970FB605
:105FB000F894DEBF0FBECDBF182F80E00E949F2F48
:105FC0004B015C018092A3059092A405A092A505C7
:105FD000B092A60581E00E949F2F6B017C01C092C8
:105FE000A705D092A805E092A905F092AA0582E043
:105FF0000E949F2F6093AB057093AC058093AD0515
:106000009093AE051D861E861F86188A89829A8205
:10601000AB82BC82CD82DE82EF82F88669877A8786
:106020008B879C8783E00E949F2F6D877E878F8759
:10603000988B8091400C882321F0CE0101960E941C
:1060400005211E3FD9F480E1FE013196A1E6B2E0C0
:1060500001900D928A95E1F760960FB6F894DEBF35
:106060000FBECDBFDF91CF911F91FF90EF90DF90DA
:10607000CF90BF90AF909F908F90089584E0189F2D
:10608000F0011124DF01AF59BD4F81E090E08C0F8A
:106090009D1FE80FF91F40815181628173814D93EB
:1060A0005D936D937C931397D7CFCF92DF92EF924E
:1060B000FF92CF93DF93C82F0E94EF2994E0C99FEE
:1060C000E0011124FE01E55FF94FC080D180E2803C
:1060D000F38081110E94992FC359DE4EC701B6018A
:1060E0000F943725288139814A815B810F94962549
:1060F000DF91CF91FF90EF90DF90CF9008950E94B5
:10610000EF29909191129093901290938F12909307
:106110008E1294E690938D1220ED33E030931C099B
:1061200020931B0981110E94992F81E080930A0618
:106130000895CF93DF93CDB7DEB72C970FB6F894C1
:10614000DEBF0FBECDBF0E9430F60E94EF299CE05B
:10615000E7E1F6E0DE01119601900D929A95E1F7E4
:1061600081110E94992FCE0101960E944BC62C9658
:106170000FB6F894DEBF0FBECDBFDF91CF9108956B
:106180002F923F924F925F926F927F928F929F9247
:10619000AF92BF92CF92DF92EF92FF920F931F9335
:1061A000CF93DF9300D0CDB7DEB78090610290909F
:1061B0006202A0906302B090640240906502509029
:1061C00066026090670270906802C0906902D09089
:1061D0006A02E0906B02F0906C020E94981B0E9491
:1061E000E61B01E81CE187E492E09B838A8385E754
:1061F000282E8CE1382E198289810E94891CC801C1
:106200000E946C1DEA81FB8161937193819391934C
:10621000FB83EA83C1010E946C1DEA81FB816087D8
:10622000718782879387F981FF5FF9830C5F1F4F26
:1062300084E0280E311CF330F9F685EF95E00E94DA
:1062400095F60E94881E0E94CD26A50194016091BA
:1062500061027091620280916302909164020F94D6
:10626000302581111CC0A3019201609165027091DB
:10627000660280916702909168020F943025811127
:106280000EC02091690230916A0240916B025091D8
:106290006C02C701B6010F9430258823B9F00F9026
:1062A0000F900F90DF91CF911F910F91FF90EF9082
:1062B000DF90CF90BF90AF909F908F907F906F9026
:1062C0005F904F903F902F900C9499300F900F90CB
:1062D0000F90DF91CF911F910F91FF90EF90DF9082
:1062E000CF90BF90AF909F908F907F906F905F9076
:1062F0004F903F902F90089580918111909182113D
:10630000892B79F48091811190918211892B49F424
:10631000209181113091821181E0232B19F480E0CA
:10632000089581E0089510920105809122029091D4
:106330002302A0912402B09125028093010690933C
:106340000206A0930306B093040608959091981155
:1063500010929811923071F0943079F0913099F454
:10636000813089F480910105882369F0109226021A
:106370000C94933110923E0C089588E898E1909324
:106380008E0C80938D0C08959091381493FB882780
:1063900080F993FF06C081E090919F15911101C093
:1063A00080E00895CF93C0919E05CF7739F50E9484
:1063B000C431882319F18091301490913114A09147
:1063C0003214B09133140097A105B105B9F0BC01A6
:1063D000CD016D597F4F8F4F9F4F24E630E040E055
:1063E00050E00F94742B60913414709135148091A7
:1063F0003614909137140F94742BC22F8C2FCF9199
:106400000895E8E1F9E010821182089581E008958D
:10641000DC01EC918E2F90E0FC01EE0FFF1FE80FE6
:10642000F91FED5CFD4E80818F77808308958F92F8
:106430009F92AF92BF92CF92DF92EF92FF920F9313
:10644000CF93DF931F92CDB7DEB75C017B0149018B
:106450006B01C40ED51EF501808191810F944E2BE6
:106460008983002311F0F7018083BE016F5F7F4FA6
:10647000C4010E94B3E0F50180819181019691836E
:106480008083FFEFEF1AFF0AEC14FD0421F780E090
:106490000F90DF91CF910F91FF90EF90DF90CF9011
:1064A000BF90AF909F908F9008950F93AB01009194
:1064B000F90521E002272AEF35E0BC018AED95E0DD
:1064C0000E9417320F910895009781F41092900066
:1064D00082E0809391001092950010929400C19AEE
:1064E000809171008260809371000895019761F43A
:1064F0001092A00082E08093A1001092A50010925B
:10650000A40089BB8093720008957F928F929F921E
:10651000AF92BF92CF92DF92EF92FF920F931F93B1
:10652000CF93DF93EC017B018881883108F0C3C0F1
:1065300090E0FC01EE0FFF1FE80FF91FED5CFD4E30
:1065400080818F770E94FBE619821A8288812CE075
:10655000622F0F94D72B829FB001112430E020E0EE
:10656000AB01420F531FFA01EE0FFF1FE40FF51F9F
:10657000ED5CFD4E908197FD08C02F5F3F4F2C30A2
:10658000310571F790E00E9464327880072D10E0A9
:106590006801CC0CDD1CF601E00FF11FED5CFD4E37
:1065A00080818068808377FC86C080E2E81682E084
:1065B000F8060CF03FC08A8128E532E0281B31093B
:1065C00087FD3395220F331F220F331F032E000C3C
:1065D000440B550B898178E8872E912C881A9108F5
:1065E00087FD9394880C991C880C991C092C000C2D
:1065F000AA08BB0860E070E0CB01F7FC0AC0B70155
:10660000653B710514F064EB70E0072E000C880BFD
:10661000990B281939094A095B090F94642B24EB5B
:1066200030E040E050E00F94962B820E931EA41EA3
:10663000B51E740187E18715D8F0298188E890E0BC
:10664000821B910927FD9395880F991F880F991F29
:10665000E816F90604F502972FB7F894E601C00F83
:10666000D11FCD5CDD4E880F991F9A8389832FBF80
:1066700062E370E080E090E0DF91CF911F910F9195
:10668000FF90EF90DF90CF90BF90AF909F908F9052
:106690007F900C94EF252A8188E592E0821B910976
:1066A00027FD9395880F991F880F991FE816F90603
:1066B00094F6C701D0CFDF91CF911F910F91FF903A
:1066C000EF90DF90CF90BF90AF909F908F907F9092
:1066D0000895CF93DF93EB01682F70E08CE792E190
:1066E0000E948532688179818A819B81643F21E0A3
:1066F00072078105910520F464EF71E080E090E07D
:106700000E94EF2589B183FB882780F9DF91CF9123
:106710000895CF93DF9300D01F92CDB7DEB78EEEF2
:1067200092E0A0E0B0E089839A83AB83BC83BE0192
:106730006F5F7F4F8AE50E9469330F900F900F9033
:106740000F90DF91CF910895CF93DF9300D01F92E8
:10675000CDB7DEB78EEE92E0A0E0B0E089839A83F9
:10676000AB83BC83BE016F5F7F4F8AE00E946933B9
:106770000F900F900F900F90DF91CF910895CF93CE
:10678000DF9300D01F92CDB7DEB784EF91E0A0E099
:10679000B0E089839A83AB83BC83BE016F5F7F4F78
:1067A00080EA0E9469330F900F900F900F90DF9155
:1067B000CF9108951F920F920FB60F9211240BB62E
:1067C0000F922F933F934F935F936F937F938F938A
:1067D0009F93AF93BF93EF93FF9348EA50E064EA2F
:1067E00070E081E090E00E941326FF91EF91BF914D
:1067F000AF919F918F917F916F915F914F913F9159
:106800002F910F900BBE0F900FBE0F901F901895F9
:106810001F920F920FB60F9211240BB60F922F9367
:106820003F934F935F936F937F938F939F93AF9318
:10683000BF93EF93FF9348E950E064E970E090E084
:1068400080E00E941326FF91EF91BF91AF919F913D
:106850008F917F916F915F914F913F912F910F9009
:106860000BBE0F900FBE0F901F9018959091D10006
:1068700095FD0CC09091D00095FF08C08093D60084
:106880008091D00080648093D000089520912E04E0
:106890002F5F2F770FB607FC27C090912F0492131C
:1068A00028C09091D00095FF1EC090912F04409178
:1068B0002E04941306C09091D1009F7D9093D10037
:1068C00012C0E92FF0E0E25DFB4F32819F5F9F77BE
:1068D0003093D60090932F043091D00030643093E1
:1068E000D000491741F3D9CF90912F04921301C0E2
:1068F000FBCFE0912E04F0E0E25DFB4F828320931A
:106900002E048091D10080628093D10008958F92EF
:106910009F92AF92BF92CF92DF92EF92FF920F932E
:106920001F93CF93DF937C0121E5E20EF11CD70189
:106930004C914A3509F0A4C06C01B2E5CB0ED11CD4
:10694000F6013081353A09F09BC0EC01C05BDF4FA6
:106950002881233008F494C08C0100561F4FD801C1
:106960004C93E15BFF4F308331962083EF54F10964
:106970003081E05BFF4F30833038B1F43196AC5456
:10698000B1093C913083E854F109AF5ABF4F50E050
:1069900040E02250330B42175307CCF480813296EB
:1069A0008D934F5F5F4FF7CF233031F5313809F0CA
:1069B00074C0FC01EC55FF4FDC01AC5ABF4F2C9169
:1069C00020833196885A9F4FDC018C918083480147
:1069D000B12CA12C888190E002968A159B050CF4BD
:1069E0003FC0F40181914F010E9436340E94C9E0FA
:1069F000FFEFAF1ABF0AEECF323821F5FC01EC5A97
:106A0000FF4F30814181E05BFF4F408331963083FF
:106A1000DC01AA55BF4F50E040E02350330B421732
:106A20005307ACF6FA01EE7FE45AFF4FE80FF91F67
:106A3000608171817C9311966C9311974E5F5F4FCB
:106A40001296EDCF243019F6333809F6FC01EC5AD2
:106A5000FF4F20813181E05BFF4F30833196B0CF13
:106A600080E5DE011D928A95E9F78AE1F80111922D
:106A70008A95E9F78AE5D7018C9385EAF601808348
:106A8000DF91CF911F910F91FF90EF90DF90CF900A
:106A9000BF90AF909F908F900895323809F097CFB4
:106AA000ADCFAF92BF92CF92DF92EF92FF920F9352
:106AB0001F93CF93DF93EC0184E6C82E80E2D82E9B
:106AC000E12CF12C02E8A12C90E2B92E15E0009304
:106AD000C513C092C613D092C713E092C813F092A8
:106AE000C913B092CF13A092CE131093C21382E7B2
:106AF00093E10E9487348FEFC81AD80AE80AF80A8F
:106B000088E7C81680E2D806E104F10401F724E61C
:106B100030E240E050E0BE0182E793E1DF91CF91A7
:106B20001F910F91FF90EF90DF90CF90BF90AF90AB
:106B30000C94CEE0CF92DF92EF92FF920F931F93CF
:106B4000CF93DF93CDB7DEB77C01CDB6DEB60F9421
:106B50007D2401962DB73EB7281B390B0FB6F8944C
:106B60003EBF0FBE2DBF0DB71EB70F5F1F4FB70142
:106B7000C8010F947624F80101900020E9F73197BD
:106B8000E01BF10B759720F08BE892E0F801848B05
:106B9000C8010E9451350FB6F894DEBE0FBECDBEBF
:106BA000DF91CF911F910F91FF90EF90DF90CF90E9
:106BB00008958F929F92AF92BF92CF92DF92EF9201
:106BC000FF920F931F93CF93DF930E94AB2C3AE079
:106BD000C32E30E2D32EE12CF12C15E002E8460161
:106BE0005701CAE0D0E01092CF131092CE13109349
:106BF000C2130093C5138092C6139092C713A0923C
:106C0000C813B092C91382E793E10E948734219799
:106C10008FEF881A980AA80AB80A209721F78AE005
:106C2000C80ED11CE11CF11C82EDC81680E2D8060A
:106C3000E104F104A1F6C12C20E2D22EE12CF12CCA
:106C4000D5E0C2E81092CF131092CE13D093C213A6
:106C5000C093C513C092C613D092C713E092C81355
:106C6000F092C91382E793E10E9487341092CF1308
:106C70001092CE13D093C213C093C513D701C6018F
:106C80008C529F4FAF4FBF4F8093C6139093C71343
:106C9000A093C813B093C91382E793E10E9487348D
:106CA0008FEFC81AD80AE80AF80A8AE0C81680E204
:106CB000D806E104F10431F69EEDC92E90E2D92EFA
:106CC000E12CF12CD5E0C2E81092CF131092CE1334
:106CD000D093C213C093C513C092C613D092C713EA
:106CE000E092C813F092C91382E793E10E948734BF
:106CF0008FEFC81AD80AE80AF80A86EEC81680E2AA
:106D0000D806E104F10401F7CC24C39482E1D82E23
:106D1000E12CF12C0AE010E0D5E0C2E81093CF138B
:106D20000093CE13D093C213C093C513C092C61361
:106D3000D092C713E092C813F092C91382E793E18F
:106D40000E9487341093CF130093CE13D093C213B5
:106D5000C093C513D701C6018096A11DB11D8093B4
:106D6000C6139093C713A093C813B093C91382E7B7
:106D700093E10E9487348FEFC81AD80AE80AF80A0C
:106D800085E1C81682E1D806E104F10439F682E112
:106D900090E09093CF138093CE13D093C213C093FF
:106DA000C51384E190E1A0E0B0E08093C613909316
:106DB000C713A093C813B093C91382E793E1DF917F
:106DC000CF911F910F91FF90EF90DF90CF90BF90E8
:106DD000AF909F908F900C9487341F920F920FB6B4
:106DE0000F9211240BB60F922F938F939F93EF93D3
:106DF000FF9380912F0420912E04821306C080916E
:106E0000D1008F7D8093D10012C0E82FF0E0E25DC9
:106E1000FB4F92818F5F8F779093D60080932F04E2
:106E20009091D00090649093D000281741F3FF9187
:106E3000EF919F918F912F910F900BBE0F900FBEEE
:106E40000F901F9018951F920F920FB60F9211245A
:106E50000BB60F920F931F932F933F934F935F9314
:106E60006F937F938F939F93AF93BF93CF93DF9352
:106E7000EF93FF93C091D60000915205D091510538
:106E800011E01D0F1F7390912D04913108F09FC0E8
:106E9000E92FF0E08827E05BF84C8F4F0D94F72B3B
:106EA000613790379F37AE37B537E737B937E737B0
:106EB000BD37C137E737C537C937CD37D437E7379F
:106EC000DF37C03229F028F5CA3011F0CD3031F566
:106ED000011731F0ED2FF0E0EF5AFA4FC283D12FB6
:106EE000D0935105FF91EF91DF91CF91BF91AF9179
:106EF0009F918F917F916F915F914F913F912F91D2
:106F00001F910F910F900BBE0F900FBE0F901F900F
:106F10001895CD3481F081E0CE3471F080E10CC061
:106F2000CA3338F4C033A0F6C03291F2CD32B1F793
:106F3000CFCFCD3499F782E080932D04C9CFC133F0
:106F400059F018F4C03221F2E9CF88E0C433A1F33C
:106F50008BE0C83389F3E2CF83E0EECF84E0C03327
:106F600059F386E0C13341F3D9CF85E0C833B1F698
:106F7000E3CF87E0C23391F6DFCF89E0C13371F60A
:106F8000DBCF8AE0C03351F6D7CF8CE0C73331F680
:106F9000D3CF8DE0C63311F6CFCFC03209F498CFEE
:106FA0008EE0C33549F2BACF80ED8C0F8A3008F0FD
:106FB0008FCF9FE090932D0480932C0489CFCA300B
:106FC00019F0CD3009F084CF10922D0481CFCA3052
:106FD00019F0CD3009F07CCF80912C148823A1F3D7
:106FE000973089F038F4953079F710923C0210927E
:106FF0003E0CEACF9A3059F09F3031F780912C0443
:107000000E94A631E1CF81E080932806DDCF81E0A8
:1070100080932706D9CF9091C00095FFFCCF809335
:10702000C6000895CF93DF93EC018991882319F06E
:107030000E940B38FACF8DE00E940B388AE0DF9176
:10704000CF910C940B38CF92DF92EF92FF92CF93B7
:107050006B017C01C42F4A3069F4F7FE0BC0F09439
:10706000E094D094C094C11CD11CE11CF11C8DE2B1
:107070000E940B384C2FC701B601CF91FF90EF90C3
:10708000DF90CF900C9443AACF93DF93EC01FE01E5
:1070900084912196882319F00E940B38F8CFDF9154
:1070A000CF910895CF93DF93D0912B118DE59CE183
:1070B0000E9444388AE00E940B388091AA0C8730E5
:1070C00009F449C083E08093A80C81E080937E029C
:1070D00080E190E09093CF138093CE1385E080936E
:1070E000C213C2E8C093C51384E190E1A0E0B0E010
:1070F0008093C6139093C713A093C813B093C9137A
:1071000082E793E10E94873461E070E080E090E0E4
:107110000E94902C81E09AE59093CF138093CE1338
:1071200085E390E09093D1138093D01387E0809310
:10713000C213C093C51384E890E0A0E0B0E0809350
:10714000C6139093C713A093C813B093C91382E7D3
:1071500093E10E94873480912B11813089F1823034
:1071600061F50E947C2B6093C2057093C3058093E8
:10717000C4059093C50581E080932B110E940BFDFF
:107180006093BE057093BF058093C0059093C105C1
:10719000D23089F08091AB069091AC060196909325
:1071A000AC068093AB061092CA051092CB051092E4
:1071B000CC051092CD0581E004C00E94AE2BDBCF40
:1071C00080E0DF91CF910895CF93C82FCB010E942B
:1071D000443881ED98E10E94443882EC98E1CC2358
:1071E00011F087EC98E10E9444388AE0CF910C942A
:1071F0000B38CF93DF9300D01F92CDB7DEB784EF6B
:1072000091E0A0E0B0E089839A83AB83BC83BE01A8
:107210006F5F7F4F8CE30E9469338FEE98E10E948D
:1072200044388CB169EE78E185FB882780F90E94AB
:10723000E4388091030163EE78E1869581700E94C5
:10724000E43889B16DED78E183FB882780F90E94ED
:10725000E4388CB164ED78E1829581700E94E43865
:107260004B9909C00E94A4330F900F900F900F907C
:10727000DF91CF9108950E9489330F900F900F9066
:107280000F90DF91CF91089580912B118130C1F53E
:107290008DE998E10E9444388AE00E940B3881E031
:1072A0009AE59093CF138093CE1387E590E0909367
:1072B000D1138093D01387E08093C21382E8809328
:1072C000C51384E890E0A0E0B0E08093C6139093EB
:1072D000C713A093C813B093C91382E793E10E9428
:1072E000873482E080932B110E940BFD6093C605CA
:1072F0007093C7058093C8059093C90581E00895F0
:1073000080E008950F931F930E940BFD0091A60645
:107310001091A7062091A8063091A9060115110524
:107320002105310509F067C02091A412222309F438
:107330005FC0E091A21221502093A41221E02E0FF1
:107340002093A2123091A512231302C01092A21210
:1073500024E0E29FF0011124EA55FD4E00811181E5
:10736000228133810093A2061093A3062093A406E2
:107370003093A506600F711F811D911D6093A606B5
:107380007093A7068093A8069093A9068091A406FF
:107390009091A506892B61F11FB7F8948CE898E1CC
:1073A0000E9444388AE00E940B3884E096E0909373
:1073B000CF138093CE1380EA90E89093D1138093FB
:1073C000D01387E08093C21382E88093C51380EACC
:1073D00090E0A0E0B0E08093C6139093C713A09311
:1073E000C813B093C91382E793E10E9487341FBF8B
:1073F0001F910F910895601B710B820B930B97FDEA
:10740000F7CF40981092A6061092A7061092A806F1
:107410001092A906EDCF0F931F93CF93DF938C01AA
:10742000EB019091A4122091A512921305C00E9425
:1074300082390E940BC2F5CF8091A31234E0839F62
:10744000F0011124EA55FD4E11830083D383C283DA
:107450009F5F9093A4128F5F281739F08093A31237
:10746000DF91CF911F910F9108951092A312F8CF41
:10747000CF92DF92EF92FF921F93CF93DF93182F5B
:10748000662351F0109200051092FC041092FD0446
:107490001092FE041092FF040E940BFD6B017C0110
:1074A0008091FC049091FD04A091FE04B091FF0432
:1074B000A7019601281B390B4A0B5B0BDA01C901A6
:1074C000B7FD3DC02091000517FD13C0412F012ECF
:1074D000000C550B4C5F5F4F822F022E000C990B56
:1074E0004817590764F184EF91E0A0E0B0E021175C
:1074F00024F488EE93E0A0E0B0E08C0D9D1DAE1D5D
:10750000BF1D8093FC049093FD04A093FE04B093F0
:10751000FF042170C22F30E0D32F84E28C9FB00192
:107520008D9F700D7C1B112460597C4F82E390E08D
:107530000E940B3A809100058F5F80930005DF91D8
:10754000CF911F91FF90EF90DF90CF900895CF9350
:10755000DF9300D01F92CDB7DEB782E198E10E94A1
:1075600044388AE00E940B388091AA0C8330D9F10C
:1075700019821A821B821C8260E0CE0101960E9451
:10758000C92B19821A821B821C8261E0CE010196EE
:107590000E94C92B81E080937D021092A70C8093FA
:1075A0007E0281E09AE59093CF138093CE1383E31C
:1075B00090E09093D1138093D01387E08093C2130F
:1075C00082E88093C51384E890E0A0E0B0E0809367
:1075D000C6139093C713A093C813B093C91382E73F
:1075E00093E10E9487340F900F900F900F90DF91DE
:1075F000CF9108956F927F928F929F92AF92BF9298
:10760000CF92DF92EF92FF920F931F93CF93DF936E
:10761000CDB7DEB764970FB6F894DEBF0FBECDBF0F
:107620001092D0008091D00082608093D0001092A0
:10763000D50080E18093D4008091D1008061809357
:10764000D1008091D10088608093D1008091D100D9
:1076500080688093D1008091D1008F7D8093D1008C
:107660008AE58093C3138093731385EA8093C413D0
:1076700080937413E2E1F4E18AE1DF011D928A95BF
:10768000E9F78091A60C882309F473C283E090E0A7
:107690009093CF138093CE1385E08093C21382E83A
:1076A0008093C5138FE190E1A0E0B0E08093C61312
:1076B0009093C713A093C813B093C91382E793E1C3
:1076C0000E94873484E690E09093CF138093CE138A
:1076D00005E00093C21312E81093C51386E090E111
:1076E000A0E0B0E08093C6139093C713A093C81393
:1076F000B093C91382E793E10E9487348BE090E056
:107700009093CF138093CE130093C2131093C5139D
:1077100080E092E1A0E0B0E08093C6139093C7139D
:10772000A093C813B093C91382E793E10E948734F2
:107730001092CF131092CE130093C2131093C5135F
:1077400084E390E1A0E0B0E08093C6139093C71368
:10775000A093C813B093C91382E793E10E948734C2
:107760001092CF131092CE130093C2131093C5132F
:107770008AE390E1A0E0B0E08093C6139093C71332
:10778000A093C813B093C91382E793E10E94873492
:107790008091F2119091F3119093CF138093CE13B7
:1077A0000093C2131093C51386E390E1A0E0B0E00C
:1077B0008093C6139093C713A093C813B093C913B3
:1077C00082E793E10E94873480918711909188111C
:1077D0009093CF138093CE130093C2131093C513CD
:1077E0008CE390E1A0E0B0E08093C6139093C713C0
:1077F000A093C813B093C91382E793E10E94873422
:1078000082E090E09093CF138093CE130093C21345
:107810001093C5138EE190E1A0E0B0E08093C61311
:107820009093C713A093C813B093C91382E793E151
:107830000E94873481E080937D0270E6C72E70E15C
:10784000D72EE12CF12C1092CF131092CE1300936F
:10785000C2131093C513C092C613D092C713E092FF
:10786000C813F092C91382E793E10E948734BFEFF7
:10787000CB1ADB0AEB0AFB0AE4E7CE16E0E1DE06F0
:10788000E104F10401F7CE0101967C0184E1D70106
:107890001D928A95E9F781E08F9390E99F938F93EA
:1078A00098E69F938F939F9389EA93E09F938F939A
:1078B000FF92EF920F94882F20E630E140E050E0F5
:1078C00066EB73E082E793E10E94CEE02AE630E1C6
:1078D00040E050E063EC73E082E793E10E94CEE089
:1078E00024E730E140E050E0B70182E793E10E94F5
:1078F000CEE02EE730E140E050E06FEC73E082E74D
:1079000093E10E94CEE01092CF131092CE13009319
:10791000C2131093C5138EE090E1A0E0B0E0809315
:10792000C6139093C713A093C813B093C91382E7EB
:1079300093E10E9487341092CF131092CE130093DC
:10794000C2131093C5138FE090E1A0E0B0E08093E4
:10795000C6139093C713A093C813B093C91382E7BB
:1079600093E10E9487340FB6F894DEBF0FBECDBFFF
:107970004AE0C42E40E2D42EE12CF12C55E0752EC5
:1079800062E8662E460157010AE010E01092CF131C
:107990001092CE137092C2136092C5138092C613D8
:1079A0009092C713A092C813B092C91382E793E1D3
:1079B0000E94873401501109FFEF8F1A9F0AAF0A06
:1079C000BF0A0115110511F78AE0C80ED11CE11C90
:1079D000F11C92EDC91690E2D906E104F10491F68A
:1079E000C12C30E2D32EE12CF12C05E012E81092EC
:1079F000CF131092CE130093C2131093C513C092ED
:107A0000C613D092C713E092C813F092C91382E74D
:107A100093E10E9487341092CF131092CE130093FB
:107A2000C2131093C513D701C6018C529F4FAF4F9D
:107A3000BF4F8093C6139093C713A093C813B093FE
:107A4000C91382E793E10E948734AFEFCA1ADA0ABA
:107A5000EA0AFA0ABAE0CB16B0E2DB06E104F10466
:107A600031F62EEDC22E20E2D22EE12CF12C05E0D3
:107A700012E81092CF131092CE130093C2131093FA
:107A8000C513C092C613D092C713E092C813F092E8
:107A9000C91382E793E10E948734EFEFCE1ADE0A22
:107AA000EE0AFE0AF6EECF16F0E2DF06E104F1047C
:107AB00001F7CC24C39482E1D82EE12CF12C9AE07A
:107AC000A92EB12C05E012E8B092CF13A092CE13EC
:107AD0000093C2131093C513C092C613D092C7135C
:107AE000E092C813F092C91382E793E10E948734B1
:107AF000B092CF13A092CE130093C2131093C5136C
:107B0000D701C6018096A11DB11D8093C613909325
:107B1000C713A093C813B093C91382E793E10E94DF
:107B200087348FEFC81AD80AE80AF80A95E1C9160F
:107B300092E1D906E104F10439F688E797E10E9461
:107B400044388AE00E940B3864960FB6F894DEBF82
:107B50000FBECDBFDF91CF911F910F91FF90EF909E
:107B6000DF90CF90BF90AF909F908F907F906F905D
:107B7000089582E090E08CCD0E94FA3A10929A0526
:107B800081E080937E028AE298E10E9444388AE094
:107B90000C940B380F931F93CF938C01C62F84E264
:107BA00094E10E944438C8010E9444388AE30E944C
:107BB0000B3880E38C0F0E940B388AE0CF911F9125
:107BC0000F910C940B3887EA95E10E94443860E0ED
:107BD00087E995E10E94CA3D60E082E895E10E9454
:107BE000CA3D61E08BE795E10E94CA3D61E080E714
:107BF00095E10E94CA3D61E080E695E10E94CA3DA0
:107C000060E087E595E10E94CA3D61E08DE495E181
:107C10000E94CA3D61E083E495E10E94CA3D61E0B3
:107C20008CE395E10E94CA3D61E084E395E10E9406
:107C3000CA3D61E086E295E10E94CA3D61E088E1CB
:107C400095E10E94CA3D60E089E095E10E94CA3D4D
:107C500060E08BEF94E10E94CA3D60E085EE94E124
:107C60000E94CA3D61E084ED94E10E94CA3D61E05A
:107C700085EC94E10E94CA3D61E08EEB94E10E94A4
:107C8000CA3D60E087EB94E10E94CA3D61E08EEA64
:107C900094E10E94CA3D61E089E994E10E94CA3DF5
:107CA00061E08BE894E10E94CA3D61E088E794E1DD
:107CB0000E94CA3D60E08BE694E10E94CA3D61E00B
:107CC00086E694E10E94CA3D61E089E594E10E9464
:107CD000CA3D60E085E494E10E94CA3D60E082E331
:107CE00094E10E94CA3D60E08BE394E10E944F1D45
:107CF000682F617089E294E10C94CA3D80914B0534
:107D0000827149F480914D058C7829F480914E055B
:107D1000837009F475C082E40E942D1E882351F0FF
:107D20000E94FB236093550C7093560C8093570C64
:107D30009093580C83E50E942D1E882351F00E94D9
:107D400081246093850C7093860C8093870C9093AC
:107D5000880C84E50E942D1E882351F00E94812406
:107D60006093890C70938A0C80938B0C90938C0C8D
:107D700088E50E942D1E882351F00E948124609383
:107D8000F4087093F5088093F6089093F70889E556
:107D90000E942D1E882351F00E9481246093F808D0
:107DA0007093F9088093FA089093FB088AE50E9483
:107DB0002D1E8823B1F00E9481246093FC087093EB
:107DC000FD088093FE089093FF082DEC3CEC4CECF2
:107DD0005DE30F943025181624F088E99EE00E9498
:107DE000443885E40E942D1E882351F00E9481248E
:107DF000609300097093010980930209909303092D
:107E00000895AF92BF92CF92DF92EF920F931F939C
:107E1000CF93DF935B01EA016901882309F463C012
:107E200081E99EE00E944438F50160817181828180
:107E3000938146E00E944BBAE1100BC088E89EE0B7
:107E40000E944438688179818A819B8146E00E9442
:107E50004BBA81E89EE00E944438F601608171814E
:107E60008281938143E00E944BBA8AE79EE00E94A0
:107E70004438F801608171818281938143E00E94DE
:107E80004BBA81E79EE00E944438F601208131819F
:107E900042815381F80160817181828193810F94C5
:107EA000FF2B43E00E944BBAEE20F9F08AE00E94DB
:107EB0000B388CE59EE00E944438688179818A8184
:107EC0009B8146E00E944BBA8AE00E940B388AE010
:107ED000DF91CF911F910F91EF90DF90CF90BF90E6
:107EE000AF900C940B38E110E4CFDF91CF911F914C
:107EF0000F91EF90DF90CF90BF90AF9008950F93C8
:107F00001F93CF938C01C62F89E798E00E944438D5
:107F1000C8010E944438CC2331F08AE0CF911F91F0
:107F20000F910C940B38CF911F910F9108950E94DF
:107F300063E410923E0C10923C020E94C4318823EC
:107F400051F08091381482FD06C088E898E1909342
:107F50008E0C80938D0C61E081E898E10E947F3F58
:107F60000C9452380F931F93CF93DF938C016F3F84
:107F700019F410926C1160E020916C11862F062E7E
:107F8000000C990B2817190609F08CF560936C11F9
:107F900060E08BE498E10E947F3FC8010E94443872
:107FA0008AE00E940B38C8010F947D24800F911F36
:107FB000EC01C01BD10BC034D1053CF00197FC0192
:107FC0002491207C2038D1F3F3CFDD27AE01B80116
:107FD0008CE291E10F949E24C45DDE4E18828CE207
:107FE00091E1DF91CF911F910F910C945135DF9169
:107FF000CF911F910F91089510923E0C10923C0268
:108000008091381480648093381461E089E598E1A8
:108010000E947F3F4EE658E166E778E185E00E94E6
:10802000E8E260E080E698E10C94B23F0F931F9382
:10803000CF938C01C62F60E083E898E00E947F3FD9
:10804000C8010E944438CC2331F08AE0CF911F91BF
:108050000F910C940B38CF911F910F91089561E00F
:108060008BE898E00C941640EF92FF920F931F93C9
:10807000CF937C018B01C42F60E083E898E00E94DD
:108080007F3FC7010E94443880E20E940B38C8013C
:108090000E944438CC2319F08C2F0E940B388AE0C0
:1080A000CF911F910F91FF90EF900C940B38DF92BE
:1080B000EF92FF920F931F93CF93DF93D82E7B0104
:1080C0008A01E9010E942F40D092981140E0B70147
:1080D00084E799E00E9434400115110531F040E039
:1080E000B8018DE699E00E943440209731F040E0DD
:1080F000BE018DE699E00E94344061E088E699E097
:10810000DF91CF911F910F91FF90EF90DF900C9432
:108110001640AF92BF92CF92DF92EF92FF920F93F1
:108120001F93CF93DF9386EE97E00E944438C0E020
:10813000D7E0D15021F080E20E940B38FACF8C2F8B
:108140000E9421E1CF5FC53099F78AE00E940B3889
:1081500007EA17E0C0E080E20E940B388C2F0E94F3
:1081600021E15801D5E080E20E940B38F501C08082
:10817000D180E280F380A7019601C701B6010F9478
:10818000F22E882369F180E20E940B388DE30E9471
:108190000B388DE30E940B388DE30E940B388DE382
:1081A0000E940B388DE30E940B38D150F4E1AF0EE2
:1081B000B11CD111D8CF8AE00E940B38CF5F0C5F81
:1081C0001F4FC53041F68AE0DF91CF911F910F918B
:1081D000FF90EF90DF90CF90BF90AF900C940B3852
:1081E00020E030E0A901C701B6010F94602E87FDA1
:1081F00003C08BE20E940B3843E0C701B6010E9426
:108200004BBAD3CF811107C08AEC9EE00E9444385C
:108210008AE00C940B388EEC9EE0F8CFCF93DF937E
:10822000EB010E944438CE01DF91CF910C94DFE145
:10823000CF93C62F0E9444388C2FCF910C9421E10C
:10824000CF92DF92EF92FF926A017B010E94443845
:1082500042E0C701B601FF90EF90DF90CF900C9401
:108260004BBACF92DF92EF92FF926A017B010E949C
:1082700044384AE0C701B601FF90EF90DF90CF90FD
:108280000C942338CF93DF93EB010E944438CE0146
:10829000DF91CF910C9428E14F925F926F927F9281
:1082A0008F929F92AF92BF92CF92DF92EF92FF9206
:1082B0000F931F93CF93DF9300D000D01F921F9294
:1082C000CDB7DEB78091990581110AC480919705D9
:1082D000909198059C012F5F3F4F30939805209314
:1082E00097058E3E924008F4FBC38091F211909165
:1082F000F3119093CF138093CE1305E00093C21334
:1083000012E81093C51386E390E1A0E0B0E08093FB
:10831000C6139093C713A093C813B093C91382E7F1
:1083200093E10E94873480918711909188119093F6
:10833000CF138093CE130093C2131093C5138CE315
:1083400090E1A0E0B0E08093C6139093C713A09390
:10835000C813B093C91382E793E10E9487348091D8
:10836000F4119091F5119093CF138093CE13009355
:10837000C2131093C51384E390E1A0E0B0E08093B2
:10838000C6139093C713A093C813B093C91382E781
:1083900093E10E9487348091891190918A11909382
:1083A000CF138093CE130093C2131093C5138AE3A7
:1083B00090E1A0E0B0E08093C6139093C713A09320
:1083C000C813B093C91382E793E10E94873481E018
:1083D0008093990510929805109297058091AA0CA8
:1083E000882339F10E94E11C811123C080919605F8
:1083F0008F5F8093960580919605853620F01092C8
:1084000096051092AA0CE091AA0CE150E73008F012
:108410006AC00E2E000CFF0B8827EE5EFD4B8F4FBF
:108420000D94F72B1C426B4237446344A444DC4454
:108430006F4210929605DFCF0E94882C882309F4A2
:1084400052C081E080937E0284E098E10E9444382B
:108450008AE00E940B3880E190E09093CF138093E4
:10846000CE1385E08093C21312E81093C51384E104
:1084700090E1A0E0B0E08093C6139093C713A0935F
:10848000C813B093C91382E793E10E94873481E057
:108490009AE59093CF138093CE1386E390E0909368
:1084A000D1138093D01387E08093C2131093C51328
:1084B00084E890E0A0E0B0E08093C6139093C713E7
:1084C000A093C813B093C91382E793E10E94873445
:1084D0001092AA0C08C00E94882C882321F00E94C8
:1084E000E11C8823A9F380917E02882309F433C715
:1084F00080919A058111C0C284E096E09093CF13D9
:108500008093CE1380EA90E89093D1138093D01398
:1085100017E01093C21302E80093C51380EA90E0BD
:10852000A0E0B0E08093C6139093C713A093C81344
:10853000B093C91382E793E10E9487348091790256
:1085400090917A02A0917B02B0917C020097A105E4
:10855000B10509F03FC21092CF131092CE1315E06F
:108560001093C2130093C5138AE890E1A0E0B0E035
:108570008093C6139093C713A093C813B093C913E5
:1085800082E793E10E94873489E090E09093CF13D3
:108590008093CE131093C2130093C5138CE890E11F
:1085A000A0E0B0E08093C6139093C713A093C813C4
:1085B000B093C91382E793E10E94873480917902D6
:1085C00090917A02A0917B02B0917C020097F1E039
:1085D000AF07B10508F441C2B093CF13A093CE13F7
:1085E0009093D1138093D01387E08093C21382E8D5
:1085F0008093C51388E890E1A0E0B0E08093C613B3
:108600009093C713A093C813B093C91382E793E163
:108610000E9487348091790290917A02A0917B0226
:10862000B0917C02BA2FA92F982F8827009721E0BC
:10863000A207B10508F417C2B093CF13A093CE13CD
:108640009093D1138093D01387E08093C21312E8E4
:108650001093C51381EA90E0A0E0B0E08093C613C8
:108660009093C713A093C813B093C91382E793E103
:108670000E9487348091400C882309F4FAC183E07A
:1086800090E09093CF138093CE1385E08093C21334
:108690001093C51385E490E1A0E0B0E08093C61389
:1086A0009093C713A093C813B093C91382E793E1C3
:1086B0000E94873480919A05875E80939A05209165
:1086C0009A05822F90E0253608F021C29093CF13AF
:1086D0008093CE1385E08093C21382E88093C51304
:1086E00080E090E1A0E0B0E08093C6139093C713C0
:1086F000A093C813B093C91382E793E10E94873413
:108700000E94E11C811114C20E94C431811105C074
:1087100090919D0591FD0E94E11C90919D0580FB2B
:1087200091F990939D0591FD03C28091381482FDCB
:10873000FFC180912B118150823008F4F9C1609102
:10874000891170918A11072E000C880B990B0F94D8
:1087500037256B017C0120E030E0A9010F94302522
:10876000882309F4BBC66091871170918811072E88
:10877000000C880B990B0F9437252B013C0120E04E
:1087800030E040E050E4C701B6010F94FF2BA30195
:1087900092010F94602E18160CF4C2C66091F2116B
:1087A0007091F311072E000C880B990B0F9437254D
:1087B0006D837E838F8398876091F4117091F5119A
:1087C000072E000C880B990B0F9437254B015C0189
:1087D00020E030E040E251E40F94FF2B2D813E81F8
:1087E0004F8158850F94602E18160CF499C620E01E
:1087F00030E040E050E4C701B6010F94002CA30123
:1088000092010F94302587FD10C020E030E040E257
:1088100051E4C501B4010F94002C2D813E814F819C
:1088200058850F94302587FF6AC684E190E09093C5
:10883000CF138093CE1385E08093C21382E8809398
:10884000C51384E190E1A0E0B0E08093C61390935B
:10885000C713A093C813B093C91382E793E10E9492
:1088600087348091A80C81117CC682E07AC686EF9D
:1088700097E10E9444388AE00E940B3881E09AE533
:108880009093CF138093CE1380E490E09093D11314
:108890008093D01317E01093C21382E88093C5131E
:1088A00084E890E0A0E0B0E08093C6139093C713F3
:1088B000A093C813B093C91382E793E10E94873451
:1088C0001093AA0C10CE8091970C882309F40BCE3C
:1088D0000E94882C882309F406CE0E94E11C811195
:1088E00002CE88EE97E10E9444388AE00E940B385D
:1088F0008091980C90E0B0E0A0E0895B9F4FAE4F74
:10890000B54A21E03AE53093CF132093CE139093EC
:10891000D1138093D01387E08093C21382E88093B1
:10892000C51384E890E0A0E0B0E08093C613909374
:10893000C713A093C813B093C91382E793E10E94B1
:1089400087341092970CC4CD0E94882C882309F498
:10895000CACD0E94E11C8111C6CD81E080937E02C8
:108960001092AA0C8AED97E10E9444388AE00E9496
:108970000B3881E09AE59093CF138093CE138EE469
:1089800090E09093D1138093D01387E08093C2132B
:1089900082E88093C51384E890E0A0E0B0E0809383
:1089A000C6139093C713A093C813B093C91382E75B
:1089B00093E10E94873497CD0E94E11C811193CDF1
:1089C00019821A821B821C8262E0CE0101960E94EB
:1089D000B0F47ECD0196A11DB11D35E0B695A795E9
:1089E000979587953A95D1F70197A109B109009715
:1089F000E1E0AE07B10548F1B093CF13A093CE13D9
:108A00009093D1138093D0131093C21312E8109354
:108A1000C5138AE890E1A0E0B0E08093C61390937C
:108A2000C713A093C813B093C91382E793E10E94C0
:108A3000873488E090E09093CF138093CE1385E045
:108A40008093C2131093C513A9CD9093CF13809335
:108A5000CE1385E08093C213D9CF9093CF13809328
:108A6000CE1385E0C2CD9093CF138093CE1385E0D3
:108A7000ECCD82E090E005CE8A3F08F020CE8EEF6C
:108A800080939A0589EC97E10E9444388AE00E941D
:108A90000B3881E080937E0281E09AE59093CF13BA
:108AA0008093CE138DE290E09093D1138093D013F6
:108AB00087E08093C21382E88093C51384E890E036
:108AC000A0E0B0E08093C6139093C713A093C8139F
:108AD000B093C91382E793E10E94873410929905FD
:108AE00028960FB6F894DEBF0FBECDBFDF91CF91B1
:108AF0001F910F91FF90EF90DF90CF90BF90AF90BC
:108B00009F908F907F906F905F904F9008958456C4
:108B100091099093CF138093CE1385E08093C21375
:108B200082E88093C51381E090E1A0E0B0E0DCCD65
:108B30008CE090E09093CF138093CE1315E01093C8
:108B4000C21382E88093C51384E190E1A0E0B0E015
:108B50008093C6139093C713A093C813B093C913FF
:108B600082E793E10E9487340E947C2B20E13EE063
:108B700040E050E00F94742B2115310581E0480747
:108B8000510508F470C05093CF134093CE13309327
:108B9000D1132093D01387E08093C21312E810936F
:108BA000C51380E190E1A0E0B0E08093C6139093FC
:108BB000C713A093C813B093C91382E793E10E942F
:108BC00087340E947C2B20E13EE040E050E00F948F
:108BD000742B2CE330E040E050E00F94742B309382
:108BE000CF132093CE1305E00093C2131093C51347
:108BF00082E190E1A0E0B0E08093C6139093C713A8
:108C0000A093C813B093C91382E793E10E948734FD
:108C10000E94D231882309F45CC48F5F809395054C
:108C2000E82EF12C833330F5EE0CFF1CF092CF13BD
:108C3000E092CE130093C2131093C5138EE090E11F
:108C4000A0E0B0E08093C6139093C713A093C8131D
:108C5000B093C91382E793E10E9487341092CF1337
:108C60001092CE132BC03093CF132093CE131093BA
:108C7000C21394CF84E690E09093CF138093CE13E9
:108C80000093C2131093C5138EE090E1A0E0B0E012
:108C90008093C6139093C713A093C813B093C913BE
:108CA00082E793E10E948734A2E3EA1AA0E8FA0A75
:108CB000EE0CFF1CF092CF13E092CE130093C21380
:108CC0001093C5138FE090E1A0E0B0E08093C6134D
:108CD0009093C713A093C813B093C91382E793E18D
:108CE0000E9487340E94D23190E09093CF138093FA
:108CF000CE1385E08093C21382E88093C51386E18A
:108D000090E1A0E0B0E08093C6139093C713A093C6
:108D1000C813B093C91382E793E10E94873420E01F
:108D200030E0A901609187127091881280918912B8
:108D300090918A120F94002C20E030E048EC52E42D
:108D40000F9496250F946C2D7093CF136093CE13D0
:108D500005E00093C21312E81093C51386E290E178
:108D6000A0E0B0E08093C6139093C713A093C813FC
:108D7000B093C91382E793E10E9487348091750212
:108D8000909176029093CF138093CE130093C213E9
:108D90001093C51380E093E1A0E0B0E08093C61388
:108DA0009093C713A093C813B093C91382E793E1BC
:108DB0000E94873420E030E040E251E46091590C99
:108DC00070915A0C80915B0C90915C0C0F949625DD
:108DD0000F94732D7093CF136093CE130093C2132F
:108DE0001093C51382E492E1A0E0B0E08093C61333
:108DF0009093C713A093C813B093C91382E793E16C
:108E00000E94873420E030E040E251E460915D0C44
:108E100070915E0C80915F0C9091600C0F94962580
:108E20000F94732D7093CF136093CE130093C213DE
:108E30001093C51386E492E1A0E0B0E08093C613DE
:108E40009093C713A093C813B093C91382E793E11B
:108E50000E94873420E030E040E251E46091610CF0
:108E60007091620C8091630C9091640C0F94962524
:108E70000F94732D7093CF136093CE130093C2138E
:108E80001093C5138AE492E1A0E0B0E08093C6138A
:108E90009093C713A093C813B093C91382E793E1CB
:108EA0000E94873420E030E040E251E46091650C9C
:108EB0007091660C8091670C9091680C0F949625C8
:108EC0000F94732D7093CF136093CE130093C2133E
:108ED0001093C5138EE492E1A0E0B0E08093C61336
:108EE0009093C713A093C813B093C91382E793E17B
:108EF0000E94873420E030E048EC52E460917F1219
:108F00007091801280918112909182120F94962517
:108F10000F946C2D7093CF136093CE130093C213F4
:108F20001093C51386E392E1A0E0B0E08093C613EE
:108F30009093C713A093C813B093C91382E793E12A
:108F40000E94873420E030E048EC52E460918312C4
:108F50007091841280918512909186120F949625BB
:108F60000F946C2D7093CF136093CE130093C213A4
:108F70001093C5138AE392E1A0E0B0E08093C6139A
:108F80009093C713A093C813B093C91382E793E1DA
:108F90000E94873480918502909186029093CF132E
:108FA0008093CE130093C2131093C51382E592E110
:108FB000A0E0B0E08093C6139093C713A093C813AA
:108FC000B093C91382E793E10E94873480918302B2
:108FD000909184029093CF138093CE130093C21389
:108FE0001093C51384E592E1A0E0B0E08093C6132E
:108FF0009093C713A093C813B093C91382E793E16A
:109000000E94873420E030E040E251E46091F711A3
:109010007091F8118091F9119091FA110F949625A1
:109020000F94732D7093CF136093CE130093C213DC
:109030001093C51386E592E1A0E0B0E08093C613DB
:109040009093C713A093C813B093C91382E793E119
:109050000E9487342CEA35EC47E25EE36091FB1115
:109060007091FC118091FD119091FE110F94FA2CDA
:1090700020E030E040E251E40F9496250F94732DE8
:109080007093CF136093CE130093C2131093C51344
:109090008AE592E1A0E0B0E08093C6139093C713F5
:1090A000A093C813B093C91382E793E10E94873459
:1090B0002CEA35EC47E25EE36091FF1170910012FB
:1090C00080910112909102120F94962520E030E0D9
:1090D00040E251E40F9496250F94732D7093CF13B3
:1090E0006093CE130093C2131093C5138EE592E1E3
:1090F000A0E0B0E08093C6139093C713A093C81369
:10910000B093C91382E793E10E94873420E030E0F6
:1091100040E251E460918C1170918D1180918E111B
:1091200090918F110F9496250F94732D7093CF13F8
:109130006093CE130093C2131093C51382E692E19D
:10914000A0E0B0E08093C6139093C713A093C81318
:10915000B093C91382E793E10E9487342CEA35EC7F
:1091600047E25EE3609190117091911180919211AC
:10917000909193110F94FA2C20E030E040E251E4FA
:109180000F9496250F94732D7093CF136093CE1385
:109190000093C2131093C51386E692E1A0E0B0E0FD
:1091A0008093C6139093C713A093C813B093C913A9
:1091B00082E793E10E9487342CEA35EC47E25EE3D4
:1091C00060919411709195118091961190919711E1
:1091D0000F94962520E030E040E251E40F9496256C
:1091E0000F94732D7093CF136093CE130093C2131B
:1091F0001093C5138AE692E1A0E0B0E08093C61315
:109200009093C713A093C813B093C91382E793E157
:109210000E9487348091A10C811105C08091A30C1C
:10922000882309F46DC06091F2117091F311072E3B
:10923000000C880B990B0F94372520E030E048ECA8
:1092400052E40F9496256B017C016091F4117091AA
:10925000F511072E000C880B990B0F9437259B01F5
:10926000AC01C701B6010F94FA2C0F94732D65362B
:10927000710510F064E670E07093CF136093CE1325
:1092800005E00093C21312E81093C51384E290E145
:10929000A0E0B0E08093C6139093C713A093C813C7
:1092A000B093C91382E793E10E9487346091F21171
:1092B0007091F311072E000C880B990B0F94372532
:1092C0006B017C0120E030E04AE253E40F94602E11
:1092D000181624F48091A10C811146C16091F411FB
:1092E0007091F511072E000C880B990B0F94372500
:1092F0009B01AC01C701B6010F94602E87FFAFC17F
:109300008091970C882339F18091960C91E0980F09
:109310009093960C90E09093CF138093CE1385E0BA
:109320008093C21382E88093C51382E490E1A0E0A9
:10933000B0E08093C6139093C713A093C813B09363
:10934000C91382E793E10E9487348091960C8A309A
:1093500010F01092960C0E94122C882309F4B5C1CB
:1093600060918F0C7091900CEE24E394F12C6115B8
:109370007105A9F090E080E00F94352520E030E001
:1093800040E85EE30F9496250F94DE2C20E030E059
:1093900040E85FE30F94002C0F94732D7B0101E0F4
:1093A00010E08091910C811102C010E000E08091EA
:1093B000B6129091B7128F3F980711F40E94A0B394
:1093C0009093B7128093B612080F191FB80190E05E
:1093D00080E00F94352520E030E040E85EE30F9414
:1093E00096250F94DE2C4B015C01F092CF13E09296
:1093F000CE1305E00093C21312E81093C51380E169
:1094000093E1A0E0B0E08093C6139093C713A093BC
:10941000C813B093C91382E793E10E948734C50152
:10942000B4010F94732D7093CF136093CE130093F8
:10943000C2131093C51382E193E1A0E0B0E08093E2
:10944000C6139093C713A093C813B093C91382E7B0
:1094500093E10E94873402E114E1AAE1FA2E80919F
:109460005105909152052091930530919405891BE7
:109470008F7309F449C12A3131050CF0DBC1909199
:109480005105809152054FEF5FEF981749F0E82F93
:10949000F0E0EF5AFA4F42818F5F8F73809352054D
:1094A000F901EE5EFB4E4083809112148A3509F07B
:1094B000B3C162E070E080E090E00E94902C809167
:1094C000930590919405019690939405809393054C
:1094D000C6CF1092CF131092CE13ACCB6091F41183
:1094E0007091F511072E000C880B990B0F943725FE
:1094F00020E030E0A9010F943025811134C98CE0BF
:1095000090E09093CF138093CE1385E08093C213A5
:1095100082E88093C51384E190E1A0E0B0E0F3CB52
:109520008DE090E09093CF138093CE1385E08093ED
:10953000C21382E88093C51384E190E1A0E0B0E01B
:109540008093C6139093C713A093C813B093C91305
:1095500082E793E10E9487348091A80C811101C0B9
:1095600081E08093A80CDBCB1092A10C20E030E0CE
:1095700040E251E46091990C70919A0C80919B0C9F
:1095800090919C0C0F9496250F946C2D7093CF1393
:109590006093CE130093C2131093C51384E590E13A
:1095A000A0E0B0E08093C6139093C713A093C813B4
:1095B000B093C91382E793E10E94873420E030E042
:1095C00040E251E460919D0C70919E0C80919F0C43
:1095D0009091A00C0F9496250F946C2D7093CF133F
:1095E0006093CE130093C2131093C51388E590E1E6
:1095F000A0E0B0E08093C6139093C713A093C81364
:10960000B093C91382E793E10E94873488EA97E117
:109610000E9444388AE00E940B3881E09AE59093DA
:10962000CF138093CE1381E490E09093D113809375
:10963000D01387E08093C2131093C51384E890E0A1
:10964000A0E0B0E08093C6139093C713A093C81313
:10965000B093C91382E793E10E94873451CE6091A1
:10966000A30C662309F44CCE062E000C770B8FE872
:1096700097E10E9442418AE00E940B381092A30CAD
:1096800084E090E09093CF138093CE1385E0809395
:10969000C21312E81093C5138EE890E1A0E0B0E089
:1096A0008093C6139093C713A093C813B093C913A4
:1096B00082E793E10E94873481E09AE59093CF138B
:1096C0008093CE1383E590E0B0CF1092CF13109229
:1096D000CE1305E00093C21312E81093C51380E186
:1096E00093E1A0E0B0E08093C6139093C713A093DA
:1096F000C813B093C91382E793E10E948734109294
:10970000CF131092CE1393CE121613060CF492C000
:109710008091761390917713A0917813B09179137B
:109720008C34E0E19E07A105B10509F4D7C98A345C
:109730009041A105B10509F4D1C920E030E040E233
:1097400051E4609161027091620280916302909194
:1097500064020F9496250F946C2D7093CF13609331
:10976000CE1305E00093C21312E81093C51388E4EA
:1097700090E1A0E0B0E08093C6139093C713A0934C
:10978000C813B093C91382E793E10E94873420E0A5
:1097900030E040E251E46091650270916602809190
:1097A0006702909168020F9496250F946C2D709328
:1097B000CF136093CE130093C2131093C5138AE4A2
:1097C00090E1A0E0B0E08093C6139093C713A093FC
:1097D000C813B093C91382E793E10E94873420E055
:1097E00030E040E251E46091690270916A02809138
:1097F0006B0290916C020F9496250F946C2D7093D0
:10980000CF136093CE130093C2131093C5138CE44F
:1098100090E1A0E0B0E056C9121613060CF01FCE7E
:10982000F8012F2D11922A95E9F7109294051092C4
:10983000930515CE9091731380911214981321C043
:10984000909174138091131498131BC02330310529
:10985000C4F0909114149093721380911514809316
:1098600075139330D1F4982F9D7F9038B1F4909177
:1098700016149F3409F059C0909117149B3409F0C5
:1098800054C0E2E1F4E18AE1DF011D928A95E9F733
:1098900010929405109293053BCF833809F045C090
:1098A0008091161490911714982789279827B0E073
:1098B000A0E08093761390937713A0937813B093DE
:1098C0007913C0901814D12CF12CE12CC0927A138A
:1098D000D0927B13E0927C13F0927D1329E134E166
:1098E00040E050E0BA014C155D056E057F0508F0BB
:1098F0004AC0DB01CA01B695A7959795879506964C
:10990000880F991FFC01EE58FC4ED9018C911196DD
:109910009C91892798278927918380834E5F5F4F89
:109920006F4F7F4F2E5F3F4FDECF813861F58091C3
:10993000161490E0B0E0A0E0809376139093771334
:10994000A0937813B093791380911714482F50E0A7
:1099500070E060E040937A1350937B1360937C1324
:1099600070937D13A8E1B4E1EEE7F3E190E030E01D
:1099700020E08217930739F04D9150E041935193C5
:109980002F5F3F4FF6CFE2E1F4E18AE1DF011D9264
:109990008A95E9F710929405109293050E94BBFDF9
:1099A000B7CE3F924F925F926F927F928F929F922B
:1099B000AF92BF92CF92DF92EF92FF920F931F93DD
:1099C000CF93DF9380914D0587FD38C080914E0580
:1099D0008370A1F5C0918B12D0918C12488159816E
:1099E0006A817B8189E197E10E9420414C815D8100
:1099F0006E817F818DE29FE20E942041409187121B
:109A0000509188126091891270918A128AE29FE2C5
:109A10000E9420418AE0DF91CF911F910F91FF902A
:109A2000EF90DF90CF90BF90AF909F908F907F90FE
:109A30006F905F904F903F900C940B3860907F1226
:109A4000709080128090811290908212A090831268
:109A5000B09084120091851210918612C0908712E6
:109A6000D0908812E0908912F0908A1288E50E94C6
:109A70007B1EC82F882309F49AC00E948124362EA9
:109A8000472E582ED92F20E030E044EB53EC0F94B2
:109A9000602E87FD0DC020E030E044EB53E4632DE1
:109AA000742D852D9D2F0F94302518160CF081C034
:109AB00068E671E086E097E10E94424168E671E065
:109AC00081E097E10E9442418EEF96E10E94443886
:109AD000C0E089E50E947B1E882361F10E948124F9
:109AE000362E472E582ED92F20E030E044EB53EC91
:109AF0000F94602E87FD0DC020E030E044EB53E46E
:109B0000632D742D852D9D2F0F94302518160CF084
:109B100055C068E671E08BEE96E10E94424168E62E
:109B200071E086EE96E10E94424183EE96E10E944A
:109B30004438C0E08AE50E947B1E882309F443C0B4
:109B40000E9481246B017C0120E030E040E151EC77
:109B50000F94602E87FD0AC020E030E040E151E420
:109B6000C701B6010F94302518166CF567EF7FEF2B
:109B700081ED96E10E94424169E070E08CEC96E153
:109B80000E94424189EC96E1DF91CF911F910F91A4
:109B9000FF90EF90DF90CF90BF90AF909F908F900D
:109BA0007F906F905F904F903F900C944438C1E04D
:109BB00090CF632C742C852C9D2E8BCFA32CB42C92
:109BC000052D1D2FB7CFCC23E1F0C301D401809325
:109BD0007F1290938012A0938112B0938212C501DC
:109BE000D8018093831290938412A0938512B0932E
:109BF0008612C0928712D0928812E0928912F09257
:109C00008A12DF91CF911F910F91FF90EF90DF901B
:109C1000CF90BF90AF909F908F907F906F905F900C
:109C20004F903F9008958FED97E00C94443889ED64
:109C300097E00C94443884E690E09093DB058093A1
:109C4000DA051092FB051092FA050C9492DBEF9264
:109C5000FF920F931F93CF93DF93CDB7DEB7629739
:109C60000FB6F894DEBF0FBECDBF0E94FC2988233B
:109C700009F43FC04EEF53E082FF02C042EE53E0D2
:109C80002EEF33E081FF02C024EE33E080FD2EC0D2
:109C90008EEF93E05F934F933F932F939F938F9318
:109CA00083E499E19F938F938E010F5F1F4F1F9362
:109CB0000F930F94C7240E94174EC8010E941238B8
:109CC000C8010E942BE40FB6F894DEBF0FBECDBFD3
:109CD00081E062960FB6F894DEBF0FBECDBFDF9174
:109CE000CF911F910F91FF90EF90089586EE93E032
:109CF000D1CF80E0EECFCF92DF92EF92FF928AE554
:109D00000E947B1E882309F45AC00E94812420E00F
:109D100030E040E050EC0F943025C12CD12CE12CE8
:109D200090ECF92E87FD0FC00E94812420E030E0E6
:109D300040E050E40F94602E18160CF462C00E94AC
:109D400081246B017C012091610C3091620C409167
:109D5000630C5091640CC701B6010F9496250F94C3
:109D60006C2DCB010E9444FD80E50E942D1E8111C7
:109D70004EC0A70196016091871270918812809160
:109D8000891290918A120F94002C6093871270931D
:109D900088128093891290938A120E94174E4091E4
:109DA0008712509188126091891270918A128AEB01
:109DB00096E10E9420418AE00E940B3805C083E5AD
:109DC0000E947B1E8111A1CF80914D0587FD24C08B
:109DD00080914E05837001F50E94174E40918712C5
:109DE000509188126091891270918A128BEA96E1E3
:109DF0000E9420418AE0FF90EF90DF90CF900C947A
:109E00000B38C12CD12CE12C80E4F82E9CCF0E9481
:109E100049248111AECFD8CF82E50E942D1E811139
:109E2000DBCFFF90EF90DF90CF900895CF9384E544
:109E30000E947B1EC0E08823D9F00E942924C82FED
:109E40001816B4F40E94174E8DE40E940B388091CE
:109E50004805909149050E94DFE16C2FCC0F770BEC
:109E600088EA9FE00E9442418AE00E940B38CFEFCF
:109E70008C2FCF9108954F925F926F927F928F9225
:109E80009F92AF92BF92CF92DF92EF92FF92CF93C9
:109E9000DF93CDB7DEB72C970FB6F894DEBF0FBEB9
:109EA000CDBF4090E7085090E8086090E9087090B6
:109EB000EA082091470230914802409149025091AE
:109EC0004A02C301B2010F94002C69837A838B8309
:109ED0009C838090EB089090EC08A090ED08B090E7
:109EE000EE0820914B0230914C0240914D0250916E
:109EF0004E02C501B4010F94002C6D837E838F83C5
:109F00009887C090EF08D090F008E090F108F090AA
:109F1000F20820914F02309150024091510250912D
:109F20005202C701B6010F94002C69877A878B878C
:109F30009C872091530230915402409155025091D8
:109F40005602C301B2010F94002C2B013C01209159
:109F50005702309158024091590250915A02C5015E
:109F6000B4010F94002C4B015C0120915B023091F5
:109F70005C0240915D0250915E02C701B6010F94F0
:109F8000002C6B017C010E94174E83EE9EE00E9424
:109F9000443883E50E942D1E882321F00E94492425
:109FA0008093450280914502811151C08AEC9EE068
:109FB0000E9444388BED9EE00E94443849815A81CA
:109FC0006B817C8181E19EE10E9420414D815E8117
:109FD0006F8178858DE29FE20E94204149855A85F4
:109FE0006B857C858AE29FE20E94204189ED9EE09C
:109FF0000E94443881ED9EE00E944438B301A201E2
:10A0000081E19EE10E942041B501A4018DE29FE221
:10A010000E942041B701A6018AE29FE20E942041EE
:10A020008AE02C960FB6F894DEBF0FBECDBFDF914D
:10A03000CF91FF90EF90DF90CF90BF90AF909F9027
:10A040008F907F906F905F904F900C940B388EECB8
:10A050009EE0AECF5F926F927F928F929F92AF926F
:10A06000BF92CF92DF92EF92FF920F931F93CF9305
:10A07000DF931F92CDB7DEB77C0139018B015B0105
:10A08000A40EB51ED12CC12CA016B10609F450C0E7
:10A09000F70180809180F80151908F015982C401AD
:10A0A0000F944E2B5816B9F1652DC4010F94562B01
:10A0B000FFEFCF1ADF0AC6018F779927892B21F18D
:10A0C00062E070E080E090E00E94D8FCC4010F9450
:10A0D0004E2B99818917F9F00E94174E8FE694E074
:10A0E0000E94443881E00F90DF91CF911F910F9132
:10A0F000FF90EF90DF90CF90BF90AF909F908F90A8
:10A100007F906F905F90089562E070E080E090E053
:10A110000E94EF25DBCFBE016F5F7F4FC3010E941E
:10A12000B3E0F70180819181019691838083ACCF68
:10A1300080E0D9CFDF92EF92FF920F931F93CF93DE
:10A14000DF93CDB7DEB7CA5AD1090FB6F894DEBF98
:10A150000FBECDBFCF55DF4F188219821A821B82E6
:10A16000C15AD0408091E8039091E903A091EA039D
:10A17000B091EB03CB55DF4F88839983AA83BB83D0
:10A18000C55AD04084E690E09093DB058093DA05D1
:10A190001092FB051092FA051092FC052AEF35E0AB
:10A1A00044E050E0BE016B557F4F8AED95E00E9480
:10A1B0002A508091DA059091DB0502969093DB0599
:10A1C0008093DA051092FB051092FA0581E0C655DE
:10A1D000DF4F8883CA5AD040CE0186559F4F0E94D8
:10A1E000B7D12AEF35E048E450E065E47CE08AED41
:10A1F00095E00E942A502AEF35E040E150E064EFFC
:10A2000078E08AED95E00E942A508AE097EDA3EA73
:10A21000BCE3CF55DF4F88839983AA83BB83C15AA0
:10A22000D040CE018F559F4F0E94AED18DE198E076
:10A230000E94C9D186E292E00E94C0D182E292E0FF
:10A240000E94AED18091E3089091E408A091E508C6
:10A25000B091E60889839A83AB83BC838E010F5F3C
:10A260001F4FC8010E94AED1CF55DF4F188219820F
:10A270001A821B82C15AD0407E018DE6E80EF11C85
:10A2800083E0D7018C938983CE018F559F4F0E9425
:10A29000AED1C7010E94B7D1C8010E94B7D14AE030
:10A2A000D42EDA94DD2031F0CE018F559F4F0E94DD
:10A2B000AED1F7CF8FE792E10E94C9D1CF55DF4FE2
:10A2C000188219821A821B82C15AD0403AE0D32EDA
:10A2D000DA94DD2031F0CE018F559F4F0E94AED130
:10A2E000F7CF85E0D82ED982F701D082C8010E942D
:10A2F000B7D1C7010E94B7D12AEF35E048E050E05E
:10A300006DEE75E08AED95E00E942A502AEF35E067
:10A3100048E050E065EE75E08AED95E00E942A5035
:10A320002AEF35E044E650E067EA77E08AED95E011
:10A330000E942A5019828FEFD7018C93C8010E9486
:10A34000C0D1C7010E94B7D12AEF35E044E050E008
:10A3500066EF72E08AED95E00E942A508091BE0679
:10A360008983C8010E94C0D1198A1A8A1B8A1C8A53
:10A3700080E090E0A0E8BFE38D879E87AF87B88B31
:10A380008091F7119091F811A091F911B091FA1103
:10A3900089839A83AB83BC832CEA35EC47E25EE386
:10A3A0006091FB117091FC118091FD119091FE1153
:10A3B0000F94FA2C6D837E838F8398872CEA35EC7B
:10A3C00047E25EE36091FF117091001280910112EB
:10A3D000909102120F94962569877A878B879C87C4
:10A3E0002AEF35E044E150E0B8018AED95E00E94A3
:10A3F0002A5084E190E09A838983C8010E949CD10D
:10A4000080918C1190918D11A0918E11B0918F112E
:10A4100089839A83AB83BC832CEA35EC47E25EE305
:10A42000609190117091911180919211909193117E
:10A430000F94FA2C6D837E838F8398872CEA35ECFA
:10A4400047E25EE3609194117091951180919611AD
:10A45000909197110F94962569877A878B879C87AF
:10A46000C8010E94A5D18CE0EDE8F2E0D80101908E
:10A470000D928A95E1F7C8010E94A5D11982C80101
:10A480000E94B7D18FE790E09A838983C8010E9428
:10A490009CD1E9E9F2E0D80101900D92DA94E1F75C
:10A4A0002AEF35E045E050E0B8018AED95E00E94E2
:10A4B0002A508091E4058983C8010E94C0D180E2BE
:10A4C000EEE9F2E0D80101900D928A95E1F72AEFCA
:10A4D00035E040E250E0B8018AED95E00E942A5054
:10A4E000F7011082C7010E94C0D180E198E00E946C
:10A4F000C0D18CE098E00E94AED1CF55DF4F1882DA
:10A5000019821A821B82C15AD040CE018F559F4FAB
:10A510000E94AED180E2D8011D928A95E9F72AEF18
:10A5200035E040E250E0B8018AED95E00E942A5003
:10A53000FE01F99688E0DF011D928A95E9F744E66D
:10A5400050E060E070E049835A836B837C834D83E5
:10A550005E836F83788783E090E0A0E0B0E0898736
:10A560009A87AB87BC874D875E876F87788B498BCF
:10A570005A8B6B8B7C8B8D8B9E8BAF8BB88F898F1F
:10A580009A8FAB8FBC8F8D8F9E8FAF8FB8A38EE1CC
:10A5900090E0A0E0B0E089A39AA3ABA3BCA38DA3F5
:10A5A0009EA3AFA3B8A789A79AA7ABA7BCA78DA75F
:10A5B0009EA7AFA7B8AB89AB9AABABABBCAB8DAB2F
:10A5C0009EABAFABB8AF2AEF35E040E450E0B80146
:10A5D0008AED95E00E942A5090E1D92EF8018D2D48
:10A5E00011928A95E9F72AEF35E040E150E0B80191
:10A5F0008AED95E00E942A50D8011D92DA94E9F77D
:10A600002AEF35E040E150E0B8018AED95E00E9484
:10A610002A50CF55DF4F188219821A821B82C15AE5
:10A62000D040CE018F559F4F0E94AED12CE0D22E4C
:10A63000F8018D2D11928A95E9F72AEF35E04CE06B
:10A6400050E0B8018AED95E00E942A508CE6D801CE
:10A650001D928A95E9F72AEF35E04CE650E0B80103
:10A660008AED95E00E942A508EEC95E00E94A5D1DB
:10A670002AEF35E048E050E06CED75E08AED95E0BA
:10A680000E942A50F7011192DA94E9F7C755DF4F7B
:10A690001882C95AD04080E090E0A0E4B0E4C356EC
:10A6A000DF4F88839983AA83BB83CD59D040C701EC
:10A6B0000E94C9D1CE0187559F4F0E94B7D1CE01CC
:10A6C00083569F4F0E94AED180E3D7011D928A9599
:10A6D000E9F78DE89CE10E9444388AE00E940B383B
:10A6E0002AEF35E040E350E0B7018AED95E00E94A3
:10A6F0002A508091FC05811128C00091DA05109143
:10A70000DB058091FA059091FB05F7019183808329
:10A7100084E690E09093DB058093DA052AEF35E03C
:10A7200044E050E066E073E08AED95E00E942A5034
:10A73000C7010E949CD191E00536134009F490E0D6
:10A740008091FC05892B8093FC058091FC0581118B
:10A7500005C060E081EC9CE10E94B23F81EA9CE18F
:10A760000E9444388AE00E940B389091FC0581E0F9
:10A770008927C655DF4F0FB6F894DEBF0FBECDBF99
:10A78000DF91CF911F910F91FF90EF90DF9008958F
:10A79000CF93DF9300D01F92CDB7DEB78091AA068A
:10A7A0008823C1F083E390E09C838B831A82198213
:10A7B0009E012F5F3F4F40E150E06BEA76E0CE0113
:10A7C00003960E942A5081EA9CE10E9444388AE064
:10A7D0000E940B380F900F900F900F90DF91CF9148
:10A7E0000895CF92DF92EF92FF92CF93C82F80917E
:10A7F0002B118150823008F069C00E94A73A109254
:10A800002B110E940BFD6093C6057093C7058093C2
:10A81000C8059093C905C090CA05D090CB05E090BB
:10A82000CC05F090CD050E947C2BAB01BC01409380
:10A83000CA055093CB056093CC057093CD058091EC
:10A84000AF069091B006A091B106B091B2068C19F6
:10A850009D09AE09BF09840F951FA61FB71F8093DE
:10A86000AF069093B006A093B106B093B206C111A3
:10A870000AC0C1E00E94C8538C2FCF91FF90EF9087
:10A88000DF90CF9008958091AD069091AE0601962D
:10A890009093AE068093AD060E947C2BC090B306C9
:10A8A000D090B406E090B506F090B606C616D7066E
:10A8B000E806F906F0F60E947C2B6093B3067093CD
:10A8C000B4068093B5069093B606D3CFC0E0D2CF3E
:10A8D00081E00C94F1530E94BEBE0E94685480E057
:10A8E0000E94DAF8809100078130A1F40E94134E93
:10A8F00082E697E00E94443860E088E597E00E9495
:10A90000B23F6EE571E080E090E00E94EF2588E0C4
:10A91000809300070895CF92DF92EF92FF921F93EA
:10A92000CF93DF9300D01F92CDB7DEB78EEEC82E47
:10A9300082E0D82EE12CF12CC982DA82EB82FC82F3
:10A94000BE016F5F7F4F8AE50E94693381110EC09F
:10A9500010E0812F0F900F900F900F90DF91CF910B
:10A960001F91FF90EF90DF90CF9008950E94BF332A
:10A97000C982DA82EB82FC82BE016F5F7F4F8AE57B
:10A980000E946933182F882319F30E94134E8CE319
:10A9900098E00E9444380E946B54DBCFCF92DF9244
:10A9A000EF92FF921F93CF93DF9300D01F92CDB70A
:10A9B000DEB78EEEC82E82E0D82EE12CF12CC982B3
:10A9C000DA82EB82FC82BE016F5F7F4F8AE00E94D9
:10A9D000693381110EC010E0812F0F900F900F90FE
:10A9E0000F90DF91CF911F91FF90EF90DF90CF906C
:10A9F00008950E94BF330E9489330E94A4330E94AD
:10AA00008933C982DA82EB82FC82BE016F5F7F4F9D
:10AA10008AE00E946933182F8823E9F20E94134EBE
:10AA20008FEF97E00E9444380E946B54D5CFCF93AC
:10AA3000DF9300D01F921F92CDB7DEB781E08093E5
:10AA4000AA0680E1EBEAF6E0DF011D928A95E9F7BC
:10AA50000E94C85386E18D8382E390E09C838B83C0
:10AA60001A8219829E012F5F3F4F41E050E0BE01E4
:10AA70006B5F7F4FCE0103960E942A500F900F907C
:10AA80000F900F900F90DF91CF910895CF93DF93A8
:10AA9000CDB7DEB7A8970FB6F894DEBF0FBECDBF17
:10AAA0008C01F42E0E94BEBE0E94134E88E397E0F4
:10AAB0000E9444380115110511F40FE217E080914E
:10AAC0009D0580FD79C0816080939D058BE197E0B5
:10AAD0000E9444388AE00E940B38CC24C3948AE553
:10AAE000D82ED092CF13C092CE138FE090E09093E7
:10AAF000D1138093D01397E0792E7092C21322E87D
:10AB0000E22EE092C51334E8832E912CA12CB12CB7
:10AB10008092C6139092C713A092C813B092C91323
:10AB200082E793E10E948734D092CF13C092CE1374
:10AB300088E590E09093D1138093D0137092C21364
:10AB4000E092C5138092C6139092C713A092C813C7
:10AB5000B092C91382E793E10E9487348AE2898325
:10AB60008A838B838C83F801DE011596BE016F5FAB
:10AB70007F4FCD01861B970B2491319621110CC07C
:10AB8000FB01E80FF91F8AE29F01261B370B2832D1
:10AB9000310524F48193F8CF2D93EBCF20E630E1FB
:10ABA00040E050E082E793E10E94CEE06AE070E08E
:10ABB00080E090E00E94902C61E086E297E00E94A5
:10ABC0007F3F89EE93E030E6019729F0232F2A9505
:10ABD0000000E9F7F9CFF89489EE93E038EE019799
:10ABE00029F0232F2A950000E9F7F9CF0E94BEBE75
:10ABF000FF2031F00E94E71E0E94001FA895FECFA3
:10AC00000E94E51EF9CF8091FF06882319F010926B
:10AC1000FF06089540E070E060E084EB98E10E9458
:10AC200046558091AB0C9091AC0C2FEF3FEF9817ED
:10AC300051F0E92FF0E0E555F34F228130E09F5FBE
:10AC40009F779093AC0CC90108951F920F920FB695
:10AC50000F9211240F900FBE0F901F9018951F9206
:10AC60000F920FB60F9211240BB60F920F931F93F2
:10AC70002F933F934F935F936F937F938F939F9304
:10AC8000AF93BF93CF93DF93EF93FF93C091C60031
:10AC90000091AC0CD091AB0C11E01D0F1F7790917F
:10ACA0002B04913108F09FC0E92FF0E08827E45A87
:10ACB000F94A8F4F0D94F72B6D569C56AB56BA56EA
:10ACC000C156F356C556F356C956CD56F356D1560E
:10ACD000D556D956E056F356EB56C03229F028F532
:10ACE000CA3011F0CD3031F5011731F0ED2FF0E021
:10ACF000E555F34FC283D12FD093AB0CFF91EF9169
:10AD0000DF91CF91BF91AF919F918F917F916F9183
:10AD10005F914F913F912F911F910F910F900BBE1B
:10AD20000F900FBE0F901F901895CD3481F081E0E9
:10AD3000CE3471F080E10CC0CA3338F4C033A0F6D1
:10AD4000C03291F2CD32B1F7CFCFCD3499F782E056
:10AD500080932B04C9CFC13359F018F4C03221F2CB
:10AD6000E9CF88E0C433A1F38BE0C83389F3E2CFA5
:10AD700083E0EECF84E0C03359F386E0C13341F382
:10AD8000D9CF85E0C833B1F6E3CF87E0C23391F67F
:10AD9000DFCF89E0C13371F6DBCF8AE0C03351F6F3
:10ADA000D7CF8CE0C73331F6D3CF8DE0C63311F661
:10ADB000CFCFC03209F498CF8EE0C33549F2BACF75
:10ADC00080ED8C0F8A3008F08FCF9FE090932B049A
:10ADD00080932C0489CFCA3019F0CD3009F084CF8C
:10ADE00010922B0481CFCA3019F0CD3009F07CCFFE
:10ADF00080912C148823A1F3973089F038F4953092
:10AE000079F710923C0210923E0CEACF9A3059F03A
:10AE10009F3031F780912C040E94A631E1CF81E070
:10AE200080932806DDCF81E080932706D9CF8EBDA1
:10AE30000DB407FEFDCF08958FEF8EBD0DB407FE54
:10AE4000FDCF8EB50895909164009B7F9093640030
:10AE5000982F906A96959CBD80FD03C091E0863046
:10AE600009F490E09DBD0895CF93DF93EB010E941C
:10AE70004438CE01DF91CF910C9408AF2F923F92CE
:10AE80004F925F926F927F928F929F92AF92BF92FA
:10AE9000CF92DF92EF92FF920F931F93CF93DF93A6
:10AEA000009709F0AAC11092930C1092920C909303
:10AEB0009C0580939B05BAE0CB2EB0E2DB2EE12C03
:10AEC000F12C15E002E846015701C4E1D0E01092F0
:10AED0001513109214131093081300930B13809200
:10AEE0000C1390920D13A0920E13B0920F1388EBD7
:10AEF00092E10E94873421972FEF821A920AA20AC8
:10AF0000B20A209721F744E1C40ED11CE11CF11CC8
:10AF10008AE5C81680E2D806E104F104A1F6C12C46
:10AF2000A0E2DA2EE12CF12CD5E0C2E81092151344
:10AF300010921413D0930813C0930B13C0920C13E8
:10AF4000D0920D13E0920E13F0920F1388EB92E162
:10AF50000E9487341092151310921413D093081383
:10AF6000C0930B13D701C6018C529F4FAF4FBF4FF9
:10AF700080930C1390930D13A0930E13B0930F13A3
:10AF800088EB92E10E948734EFEFCE1ADE0AEE0AD8
:10AF9000FE0AFAE0CF16F0E2DF06E104F10431F632
:10AFA000FEEDCF2EF0E2DF2EE12CF12CD5E0C2E851
:10AFB0001092151310921413D0930813C0930B130F
:10AFC000C0920C13D0920D13E0920E13F0920F1357
:10AFD00088EB92E10E9487342FEFC21AD20AE20A6C
:10AFE000F20A46EEC41640E2D406E104F10401F789
:10AFF000CC24C394E2E1DE2EE12CF12C0AE010E037
:10B00000D5E0C2E81093151300931413D0930813DE
:10B01000C0930B13C0920C13D0920D13E0920E1339
:10B02000F0920F1388EB92E10E948734109315136E
:10B0300000931413D0930813C0930B13D701C601C8
:10B040008096A11DB11D80930C1390930D13A093B6
:10B050000E13B0930F1388EB92E10E9487348FEFA9
:10B06000C81AD80AE80AF80AE5E0CE16E2E1DE06D8
:10B07000E104F10439F60091920C1091930C011542
:10B08000110509F0D6C08091910C882309F4E1C024
:10B090002AE030E240E050E06CEE73E088EB92E1B1
:10B0A0000E94CEE0C1E0D0E003E010E0E090920C1E
:10B0B000F090930C35E0332E42E8242E44244A9439
:10B0C000542C64E0662E712C7FE1C72E74E0D72EDD
:10B0D0008091920C9091930C800F911FE816F906C5
:10B0E00008F0D5C0C7010E94E5E1882309F481C0BA
:10B0F0008091A61169E971E1882311F066EA71E196
:10B10000FB0101900020E9F7CF010197861B970B07
:10B11000F4E1FC9F9001FD9F300D1124265F3F4D0F
:10B1200050E040E0459710F0FB01128A88EB92E175
:10B130000E94CEE0CE018F5F9D4EB0E0A0E0219650
:10B140004E0124E0880C991C2A95E1F7FDEF8F1A37
:10B15000FFE99F0AB12CA12C2091381424FF7EC056
:10B1600070921513609214133092081320920B13EF
:10B1700080930C1390930D13A0930E13B0930F13A1
:10B1800088EB92E10E948734D0921513C092141379
:10B190003092081320920B1380920C1390920D138F
:10B1A000A0920E13B0920F1388EB92E10E948734A5
:10B1B000B70189E498E10E940E418091A61166EAE8
:10B1C00071E1811102C069E971E186E498E10E94B0
:10B1D00034576EEF7BE082E498E10E94345769E9CE
:10B1E00071E181E498E10E9434578DE398E10E9477
:10B1F00044382FEFE21AF20A6BCF2091920C309173
:10B20000930CA9014150510960919B0570919C05D7
:10B210006817790738F42C5F3F4F3093930C2093D5
:10B22000920C45CE4430510508F43DCE24503109EE
:10B23000F4CF0430110569F48091910C882331F02A
:10B2400083E090E09093930C8093920CD0E0C0E068
:10B250002DCFD0E0C0E004E010E028CF109215130D
:10B26000109214133092081320920B1380930C1336
:10B2700090930D13A0930E13B0930F1388EB92E1EC
:10B280000E948734509215134092141381CFDF919E
:10B29000CF911F910F91FF90EF90DF90CF90BF90D3
:10B2A000AF909F908F907F906F905F904F903F9066
:10B2B0002F900895AF92BF92CF92DF92EF92FF92BC
:10B2C0000F931F93CF93DF93CDB7DEB7E6970FB6FB
:10B2D000F894DEBF0FBECDBF00914F051091500511
:10B2E000F80101900020E9F731976F01C01AD10AE7
:10B2F000F801CF01801B910B8C159D053CF48191C9
:10B300008F32B9F7DF0111971C92F3CF8BE1E8E59B
:10B31000F4E1DE015C9601900D928A95E1F7F12C43
:10B32000E12CEC14FD040CF05DC0F801EE0DFF1DE6
:10B330008081811103C08FEFE81AF80A5801AE0C22
:10B34000BF1CF5018081882309F44CC0FFEFEF1A80
:10B35000FF0AF801EE0DFF1D7F01E01AF10A81914D
:10B360008111FACFCE014C960E949BB38BE1FE0176
:10B370007C96DE01119601900D928A95E1F7B50158
:10B38000CE0101960E94A9ABCE0101960E94932F97
:10B390008FE20E940B388091A61181113BC089EF8A
:10B3A00093E00E9408AF8091381484FF1BC019827B
:10B3B0001C8221E0A501BE01645E7F4FCE01019693
:10B3C0000E94DDB5811129C08AE00E940B380E94DD
:10B3D000174EB50188E297E10E943457CE010196DD
:10B3E0000E94932F8AE00E940B38CE014C960E9457
:10B3F000932FE6960FB6F894DEBF0FBECDBFDF9158
:10B40000CF911F910F91FF90EF90DF90CF90BF9061
:10B41000AF90089586EA91E1C4CFCE014C960E9488
:10B420000AB38BE1FE013196DE015C9601900D922C
:10B430008A95E1F7CE0101960E94932F72CF2F9249
:10B440003F924F925F926F927F928F929F92AF92B4
:10B45000BF92CF92DF92EF92FF920F931F93CF9301
:10B46000DF9300D000D000D01F921F92CDB7DEB77F
:10B47000B82E8091980D843008F0D1C10E940BFD48
:10B480006B017C018091980D811108C08091AB0CFB
:10B490009091AC0C891B8F7709F4A4C681E6A82E85
:10B4A00013C08A3019F08D3009F0F6C01092930D58
:10B4B0008091310D9091320DFC01E35DF24F1682C7
:10B4C000892BF1F40E940BC28091980D843008F012
:10B4D000ECC08091AB0C9091AC0C891B8F7709F478
:10B4E000E4C00E94115697FFDCCF0E94134E85EBFB
:10B4F00095E00E9444388091AB0C8093AC0CE4CF73
:10B500001092320D1092310D03E31DE0F80181918C
:10B51000803209F446C08E3409F0A9C060EB75E0B2
:10B52000C8010F94AD244C01892B41F06EE470E00A
:10B53000C80104960F944E2F009709F4C8014AE001
:10B5400050E070E060E001960F941D222B013C0159
:10B5500080912D0D90912E0DA0912F0DB091300D59
:10B560000196A11DB11D481659066A067B0629F0F1
:10B5700060E08DE795E0892851F16AE270E0C8014A
:10B580000F947D2F9C01009729F1982F901B912CEF
:10B59000992349F09150F801E90FF11D8081982617
:10B5A000F7CF8F01B3CF4AE050E070E060E0C9010F
:10B5B00001960F941D22292D30E050E040E06217E3
:10B5C00073078407950751F060E08EE595E00E94CF
:10B5D00060E77ACF60E084E395E0F9CF40922D0DEB
:10B5E00050922E0D60922F0D7092300D80910007B9
:10B5F0008130E1F067E470E0C8010F944E2F0097AE
:10B60000A9F04AE050E070E060E001960F941D223E
:10B61000643071058105910548F483E994E00E9446
:10B62000443860E089E894E00E94B23FC0929F07EE
:10B63000D092A007E092A107F092A2078091330D6B
:10B640008B3309F441CF8091980D843008F03CCFC2
:10B6500080919A0D8A9DC001112463E37DE0855697
:10B66000924F0F94592F80E00E941AE72DCF8091BE
:10B67000381480FFBBCF64E77DE2C8010F94AD248E
:10B68000009731F0FC01838180538A3008F0AECFFF
:10B6900060E08AE095E09BCF21E33DE043E35DE09D
:10B6A00063E97DE00E94FB1C0FCF8091381482FF7C
:10B6B000B6C01A82198271E6F72EE0E1EE2EF9E6A5
:10B6C000DF2E8091980D843008F0A9C00E94331DB0
:10B6D0008111A5C041E050E0BE016B5F7F4F8CE956
:10B6E00095E10E945DB10D8110E0019711F00FEF1F
:10B6F0001FEF8091A4159091A515A091A615B0916A
:10B70000A7158093341490933514A0933614B093F6
:10B7100037140E94331D0F3F100749F4811107C0F1
:10B720000E94134E83ED95E00E944438CACF4091A9
:10B730009A0D242F30E00A3061F00D3051F088234B
:10B7400009F45FC089819A81009719F001969A8364
:10B7500089831092B20489819A81F29EF001F39E4E
:10B76000F00D1124E856F24FE80FF91F1382892BD0
:10B7700069F50E940BC20E94331D882309F4A1CFF2
:10B780000E9483618CE995E10E940AB380912F1495
:10B79000882391F1815080932F148D9DC001112435
:10B7A00062E0885C994F0E945FB8E0912F1424E01A
:10B7B000E29FF0011124EC5CF94F6081718182817C
:10B7C00093810E944C220E9412AB7BCF1A82198275
:10B7D00081E00E941AE78091341490913514A09171
:10B7E0003614B09137148093940D9093950DA093D7
:10B7F000960DB093970DBFCF0E9413B3E092000750
:10B8000060CF4F9DA00111244556524F9E012F5FDE
:10B810003F4F62EB74E0802F0E94FB1C52CF0E94CE
:10B820000BFD6B017C01B11004C080912A118823AB
:10B8300051F0C0927D11D0927E11E0927F11F09272
:10B840008011BB24B3948091270590912805A09185
:10B850002905B0912A050097A105B105B1F04091E5
:10B860007D1150917E1160917F1170918011840F34
:10B87000951FA61FB71FA7019601281B390B4A0B5E
:10B880005B0BDA01C901B7FF92C18091130290915D
:10B890001402A0911502B0911602892B8A2B8B2BD2
:10B8A00009F099C10E940BFD4B015C0180913E0C97
:10B8B000811108C0209190129091911281E029137A
:10B8C00001C080E02091F2113091F31191E08927BD
:10B8D0002A3A31050CF480E091E04091B704509190
:10B8E000B8046091B9047091BA04452B462B472BDC
:10B8F00009F490E0981789F0882309F4BDC1D501B7
:10B90000C40180569444A24FBF4F8093B7049093D4
:10B91000B804A093B904B093BA0440906D0250905B
:10B920006E0260906F02709070022091B3043091AB
:10B93000B4044091B5045091B604C301B2010F9410
:10B940003025882319F18091B7049091B804A09113
:10B95000B904B091BA044092B3045092B404609216
:10B96000B5047092B604892B8A2B8B2B09F449C03D
:10B97000D501C40180569444A24FBF4F8093B704B1
:10B980009093B804A093B904B093BA048091B7041B
:10B990009091B804A091B904B091BA040097A105A0
:10B9A000B10579F1881A990AAA0ABB0AB7FC29C01D
:10B9B0001092B7041092B8041092B9041092BA040D
:10B9C00083E396E00E94443860E08FE196E00E94B5
:10B9D000B23F8091F4119091F5111816190624F4D4
:10B9E00090E080E00E94031F8091891190918A115C
:10B9F0001816190634F410928A11109289110E94B7
:10BA000091BE8091BF049091C004A091C104B091F7
:10BA1000C20446015701881A990AAA0ABB0AD5012D
:10BA2000C401B7FDB9C1209190129091911240913B
:10BA30002D0280912C02291323C190911809899F0E
:10BA4000C0011124880F892F881F990B91958D8330
:10BA500080911909489FC0011124880F892F881FE0
:10BA6000990B91958E830E940BFD69837A838B835A
:10BA70009C8340E0BE016F5F7F4FCE0105960E9420
:10BA80004D1C6D8170E089E00E9402FC41E0BE0126
:10BA90006F5F7F4FCE0105960E944D1C6E8170E056
:10BAA00087E00E9402FC80913306882309F467C175
:10BAB0000091200210912102C80102972091F411F7
:10BAC0003091F511281739070CF459C18090911263
:10BAD0008F82188619861A861B86809190129F8005
:10BAE000891509F4E7C0892D90E03CE5A32EA89EB6
:10BAF000F001A99EF00D1124E35EF64F45895689A9
:10BB00006789708D452B462B472B81F4418D528DD3
:10BB1000638D748D452B462B472B41F4458D568DF7
:10BB2000678D70A1452B462B472BE1F12CE5B22EFA
:10BB3000B89E9001B99E300D1124A901435E564F65
:10BB40001A01FA0161817281838194810F94AE2E72
:10BB50004B015C01F10161A172A183A194A10F9439
:10BB600035252B013C01F10165A176A187A190A5A6
:10BB70000F9435259B01AC01C301B2010F94FA2C3F
:10BB8000A50194010F9496254B015C012885398508
:10BB90004A855B850F94602E181624F48886998652
:10BBA000AA86BB868F818F5F87708F8396CF0E9416
:10BBB000134E60919D0770919E0782EE95E00E9462
:10BBC00034578AE00E940B3840E070E060E090E07B
:10BBD00080E00E94465590919012809191129817A2
:10BBE00049F0C0927D11D0927E11E0927F11F092C7
:10BBF000801158CEBB2019F01092C30453CE0E947E
:10BC00000BFD00917D1110917E1120917F113091DB
:10BC100080118090130290901402A0901502B090B1
:10BC20001602080D191D2A1D3B1D601B710B820B8E
:10BC3000930B97FDE1CF8091C304811133CE81E056
:10BC40008093C3045F9A80913F0C8E7F80933F0C5A
:10BC50008A9A80913F0C8D7F80933F0C80910801E0
:10BC6000809581708093060180913F0C8B7F80933B
:10BC70003F0C0E94E51E16CE80E090E0DC0145CE30
:10BC8000209191125CE5259F90011124235E364F8F
:10BC9000F901EA5AFF4F9081899FC0011124880F52
:10BCA000892F881F990B91958D83295A3F4FF90150
:10BCB0008081D0CE20911A0230911B0240911C024B
:10BCC00050911D02688579858A859B850F949625FC
:10BCD0004B015C01B801012E000C880B990B0F94ED
:10BCE00037259B01AC01C501B4010F94002C698379
:10BCF0007A838B839C8340911E0250911F02B8016E
:10BD0000CE0101960E94C9C189809A80AB80BC8017
:10BD10004090BB045090BC046090BD047090BE0481
:10BD2000A3019201C501B4010F94302587FF16C00D
:10BD300028E431EE4AE75FE3C301B2010F94962590
:10BD400020E037ED43EA5CE30F94002CA501940159
:10BD50000F94962569837A838B839C8369817A818A
:10BD60008B819C816093BB047093BC048093BD0461
:10BD70009093BE040F946C2DCB010E94031FF4E638
:10BD8000CF0ED11CE11CF11CC092BF04D092C004A4
:10BD9000E092C104F092C2040E940BC2809100079D
:10BDA000882309F4E0C180912602882309F4A3C006
:10BDB0008091010581119FC080912A11811108C0D5
:10BDC00080912B11813021F08091381482FF93C033
:10BDD000F894649B10C08091220290912302A0915C
:10BDE0002402B09125028093010690930206A0934D
:10BDF0000306B093040660910106709102068091DB
:10BE0000030690910406789420E030E0A9010F9495
:10BE1000302587FF70C001E00093010580912A1151
:10BE2000811167C088E496E00E9444388AE00E944D
:10BE30000B3884E08093A80C82E08093940C81E01E
:10BE40009AE59093CF138093CE138EE490E0909375
:10BE5000D1138093D01387E08093C21382E880933C
:10BE6000C51384E890E0A0E0B0E08093C6139093FF
:10BE7000C713A093C813B093C91382E793E10E943C
:10BE800087340E942F400093981140E36CE876E0DD
:10BE900084E799E00E94344061E088E699E00E94DE
:10BEA000164010912B0560E010278CE399E069F4AF
:10BEB0008AE796E00E947F3F80E30E940B388AE089
:10BEC0000E940B3860E08DE596E00E947F3F88E697
:10BED00096E00E94443880E30E940B388AE00E947A
:10BEE0000B38112331F083E696E090938E0C80930B
:10BEF0008D0C0E94836190910901892F809581703A
:10BF0000109100021817C9F0209138142062209374
:10BF100038148093000290FD3FC164EF71E080E02F
:10BF200090E00E94EF250E9435B38091381483FD84
:10BF30007CC1111133C10E94D9350E940BFD6B01E8
:10BF40007C01109117021123F1F080912C058823B8
:10BF5000D1F04091C4045091C5046091C604709121
:10BF6000C70446015701841A950AA60AB70AB50103
:10BF7000A40177FD1AC0833009F42FC10CF01EC153
:10BF800081300CF023C1212F30E0A8EEB3E00F94F4
:10BF9000C82BC60ED71EE81EF91EC092C404D0924C
:10BFA000C504E092C604F092C70480912B11813041
:10BFB00009F073C00E940BFD6B017C018091CC04E1
:10BFC0009091CD04A091CE04B091CF04A701960129
:10BFD000281B390B4A0B5B0BDA01C901B7FD3AC0CC
:10BFE000D701C601805F984DAF4FBF4F8093CC04FF
:10BFF0009093CD04A093CE04B093CF048090CA0553
:10C000009090CB05A090CC05B090CD050E947C2BE4
:10C01000AB01BC014093CA055093CB056093CC059E
:10C020007093CD058091AF069091B006A091B106B6
:10C03000B091B20688199909AA09BB09840F951F06
:10C04000A61FB71F8093AF069093B006A093B106CA
:10C05000B093B2068091C8049091C904A091CA041B
:10C06000B091CB0446015701881A990AAA0ABB0A63
:10C07000D501C401B7FD11C020E8C20E2EEED21EBC
:10C0800026E3E21EF11CC092C804D092C904E092DB
:10C09000CA04F092CB040E94C8530E9482390E94C5
:10C0A0004C4180912605882379F10E940BFD6B019C
:10C0B0007C018091220590912305A0912405B091E7
:10C0C000250546015701881A990AAA0ABB0AD50113
:10C0D000C401B7FD19C02091260530E0A8EEB3E0F9
:10C0E0000F94C82BC60ED71EE81EF91EC09222055B
:10C0F000D0922305E0922405F092250580E00E946D
:10C10000EFBA8AE00E940B3880912105882359F10B
:10C110000E940BFD6B017C0180911D0590911E0515
:10C12000A0911F05B0912005A7019601281B390B8E
:10C130004A0B5B0BDA01C901B7FD15C0209121053F
:10C1400030E0A8EEB3E00F94C82BC60ED71EE81E51
:10C15000F91EC0921D05D0921E05E0921F05F092B7
:10C1600020050E94D0AA2B960FB6F894DEBF0FBE12
:10C17000CDBFDF91CF911F910F91FF90EF90DF9096
:10C18000CF90BF90AF909F908F907F906F905F9077
:10C190004F903F902F9008950E9424B3123008F0E2
:10C1A000CCCE0E94D93560E085EC96E050C083ED9E
:10C1B00096E090938E0C80938D0CBFCE843009F066
:10C1C000E2CE0E94174E8AED96E004C00E94174E00
:10C1D00089E097E00E944438D6CE0E94174E82EF45
:10C1E00096E0F8CF80919F079091A007A091A107BA
:10C1F000B091A207A7019601281B390B4A0B5B0BD4
:10C20000DA01C901885E9340A109B109B7FD46C9A9
:10C210008DEC95E00E944438C0929F07D092A00711
:10C22000E092A107F092A20739C9123098F48DE983
:10C2300096E00E9444388AE00E940B380E94AB2CA2
:10C2400090E080E00E943E5760E086EB96E00E941E
:10C25000B23F73CE123009F070CE0E948FB78823A0
:10C2600079F081E00E9465B742EB50E069E278E046
:10C270008DE394E10E945DB18DE394E10E940AB3E5
:10C280000E94812F811193CF0E946B2F0E940BB8C7
:10C290000E9460B752CECF93DF938091901290911D
:10C2A0009112891B8095877019F40E941F5AF5CF4F
:10C2B000809190128F5F8770A09190129CE5A99F4A
:10C2C000D0011124FD01E35EF64FEF0119929A951A
:10C2D000E9F798E09083AE5CB64F90E1E2E9F2E1D5
:10C2E00001900D929A95E1F7209190129091911200
:10C2F000291303C094E690938D1280939012DF91DE
:10C30000CF910C94992F9091901280919112981343
:10C3100006C080911B0990911C09892B21F080E0B7
:10C320000E941F5AF0CF0895FC0120813181428183
:10C3300053816091650C7091660C8091670C9091AF
:10C34000680C0F9496250F946D2E60939E12709337
:10C350009F128093A0129093A112909190128091BD
:10C36000911298130C944B610E9483610E94EF29F3
:10C3700040919E1250919F126091A0127091A11253
:10C380004093230650932406609325067093260657
:10C3900081110C94992F08954F925F926F927F9222
:10C3A0008F929F92AF92BF92CF92DF92EF92FF92C5
:10C3B0000F931F93CF93DF93EC018B015A01F90187
:10C3C0002091650C3091660C4091670C5091680C7F
:10C3D00060817181828193810F9496250F946D2ED7
:10C3E0006B017C012091610C3091620C4091630CD7
:10C3F0005091640CF50160817181828193810F9469
:10C4000096250F946D2E4B015C0120915D0C3091AF
:10C410005E0C40915F0C5091600CF801608171815D
:10C42000828193810F9496250F946D2E2B013C01F0
:10C430002091590C30915A0C40915B0C50915C0C3E
:10C44000688179818A819B810F9496250F946D2E46
:10C45000609392127093931280939412909395121A
:10C46000409296125092971260929812709299127E
:10C4700080929A1290929B12A0929C12B0929D125E
:10C48000C0929E12D0929F12E092A012F092A1123E
:10C490009091901280919112981791F0DF91CF9125
:10C4A0001F910F91FF90EF90DF90CF90BF90AF90D2
:10C4B0009F908F907F906F905F904F900C944B6106
:10C4C0000E9483610E94EF2940919A1250919B1221
:10C4D00060919C1270919D1200919612109197128A
:10C4E0002091981230919912C0909212D09093128C
:10C4F000E0909412F0909512C0921706D092180610
:10C50000E0921906F0921A0600931B0610931C067F
:10C5100020931D0630931E0640931F06509320065D
:10C52000609321067093220640919E1250919F12B3
:10C530006091A0127091A11240932306509324069B
:10C540006093250670932606882391F0DF91CF91A2
:10C550001F910F91FF90EF90DF90CF90BF90AF9021
:10C560009F908F907F906F905F904F900C94992F39
:10C57000DF91CF911F910F91FF90EF90DF90CF90BF
:10C58000BF90AF909F908F907F906F905F904F90F3
:10C5900008953F924F925F926F927F928F929F92F7
:10C5A000AF92BF92CF92DF92EF92FF920F931F93C1
:10C5B000CF93DF93CDB7DEB768970FB6F894DEBFA1
:10C5C0000FBECDBFD82E2A013B01480159013E2C98
:10C5D00020E030E0A901C501B8010F943025811198
:10C5E00010C081E08D1508F0B6C060E070E080E713
:10C5F00093E420E030E040E752E40F94FA2C4B0142
:10C600005C018D8A9E8AAF8AB88E0D2D10E0F801EC
:10C61000E256F64EE491BB24B3941E160CF4B12CF2
:10C62000CC24C39420E030E0A901C301B2010F94EF
:10C63000602E18160CF0C12CBC1471F092E0D912C7
:10C640000BC0332049F081E00E94DAF869E170E024
:10C6500080E090E00E94EF2580E00E949F2F698398
:10C660007A838B839C8381E00E949F2F6D837E83DE
:10C670008F83988782E00E949F2F69877A878B87B4
:10C680009C8783E00E949F2F6D877E878F87988B82
:10C69000000F111F000F111FE1E0F0E0EC0FFD1F74
:10C6A0000E0F1F1FF80110821182128213829E0149
:10C6B000235F3F4FAE01475F5F4FBE016B5F7F4F10
:10C6C000CE0101960E94CC61F801408251826282C3
:10C6D0007382198A1A8A1B8A1C8A80911B0990917D
:10C6E0001C09892B91F4CE0141967C018E010B5ED1
:10C6F0001F4F9E01235F3F4FAE01475F5F4FBE015B
:10C700006B5F7F4F40970E9484E70E948361BC1457
:10C7100051F092E0D91205C0332019F080E00E9458
:10C72000DAF80E94035668960FB6F894DEBF0FBE83
:10C73000CDBFDF91CF911F910F91FF90EF90DF90D0
:10C74000CF90BF90AF909F908F907F906F905F90B1
:10C750004F903F90089560E070E88BE395E449CFF7
:10C760004F925F926F927F928F929F92AF92BF9201
:10C77000CF92DF92EF92FF920F931F93CF93DF93AD
:10C78000CDB7DEB72C970FB6F894DEBF0FBECDBF86
:10C790002B013C0129873A874B875C874701580169
:10C7A000F601E080F1800281138120E030E0A901F0
:10C7B000B701C8010F943025882309F488C05E2D85
:10C7C0004F2D302F212F852F942FA32FB22F898308
:10C7D0009A83AB83BC8320E030E0A901B701C80194
:10C7E0000F943025811108C0E0903D02F0903E0288
:10C7F00000913F0210914002C701D8018D839E83B2
:10C80000AF83B887A50194016091690270916A02B3
:10C8100080916B0290916C020F94302587FF0CC0C1
:10C820008092690290926A02A0926B02B0926C02AE
:10C83000CE0101960E94CA2A409261025092620281
:10C84000609263027092640289859A85AB85BC858B
:10C850008093650290936602A0936702B09368028A
:10C86000CE0105960E94CA2AA50194016091690231
:10C8700070916A0280916B0290916C020F94602E0D
:10C88000181664F48092690290926A02A0926B0278
:10C89000B0926C02CE0101960E94CA2A0E94836166
:10C8A0002C960FB6F894DEBF0FBECDBFDF91CF91AF
:10C8B0001F910F91FF90EF90DF90CF90BF90AF90BE
:10C8C0009F908F907F906F905F904F90089550E071
:10C8D00040E030E820E477CFCF92DF92EF92FF92F2
:10C8E0000F931F936A01E0906902F0906A02009131
:10C8F0006B0210916C02FB012081318142815381D6
:10C90000FC0160817181828193810E94B0631F91DB
:10C910000F91FF90EF90DF90CF900895CF92DF922C
:10C92000EF92FF920F931F936B01FC01E080F18067
:10C9300002811381E1E6F2E024813581468157814D
:10C9400060817181828193810E94B0631F910F91F8
:10C95000FF90EF90DF90CF9008950F931F93CF93A8
:10C96000DF93EC018B0181E00E94DAF869E170E06D
:10C9700080E090E00E94EF25B801CE010E948E6415
:10C98000C091FF0680E00E94DAF81092FF0682E074
:10C990000E94C92F0E94E52AC2FBCC27C0F981E082
:10C9A0008C27DF91CF911F910F910895AF92BF9285
:10C9B000CF92DF92EF92FF920F931F93CF93DF936B
:10C9C00000D01F92CDB7DEB7FC01E080F18002817C
:10C9D0001381611112C0A0906902B0906A02C090E8
:10C9E0006B02D0906C029501A601B701C8010F94AB
:10C9F000302587FF02C07501860120E030E048EC59
:10CA000053E4B701C8010F94302587FD04C0E12C21
:10CA1000F12C08EC13E4C701D80189839A83AB8316
:10CA2000BC8362EF72E0CE0101960E948E640F908B
:10CA30000F900F900F90DF91CF911F910F91FF906A
:10CA4000EF90DF90CF90BF90AF9008953F924F92BC
:10CA50005F926F927F928F929F92AF92BF92CF928E
:10CA6000DF92EF92FF920F931F93CF93DF9300D04B
:10CA70001F92CDB7DEB7382E80E090E0A0E2B1E49F
:10CA800089839A83AB83BC83C0908712D09088122D
:10CA9000E0908912F0908A1220E030E0A901C701ED
:10CAA000B6010F94302587FF0CC0A701960160E006
:10CAB00070E080E291E40F94FF2B69837A838B838B
:10CAC0009C8360E0CE0101960E94D6644090610292
:10CAD00050906202609063027090640280906502E0
:10CAE00090906602A0906702B0906802332089F1AE
:10CAF0000E94CE5419821A821B821C82E090690225
:10CB0000F0906A0200916B0210916C02CE010196C6
:10CB10006C01A5019401C301B2010E94B06330927F
:10CB20009B070E946D2B0F900F900F900F90DF913D
:10CB3000CF911F910F91FF90EF90DF90CF90BF901A
:10CB4000AF909F908F907F906F905F904F903F90AD
:10CB500008950E948B54CECF80919B07882319F0B3
:10CB600080E00E94266580E008952F923F924F92C8
:10CB70005F926F927F928F929F92AF92BF92CF926D
:10CB8000DF92EF92FF920F931F93CF93DF93CDB776
:10CB9000DEB766970FB6F894DEBF0FBECDBFF82E96
:10CBA000282E312CF101E256F64ED49022E0821369
:10CBB00035C080919B07811103C081E00E942665EA
:10CBC0000E94CE54811139C18AE999E10E946C1DFD
:10CBD00020E030E0A9010F9430258823F9F06D2D75
:10CBE000DD0C770B880B990B0F9437252B013C013B
:10CBF0008AE999E10E946C1D4B015C0120E030E064
:10CC000040EA50E40F94302511E087FF1CC0812CCE
:10CC1000912C90EAA92E90E4B92E15C06D2DDD0C53
:10CC2000770B880B990B0F9437252B013C01C10121
:10CC3000880F991F880F991F8E56964E0E946C1D63
:10CC40004B015C0110E0A3019201C501B4010F94F6
:10CC500096254B015C016101CC0CDD1CCC0CDD1C6C
:10CC6000C6018A57964E0E946C1DEE24E394E1267D
:10CC700020E030E040EC5FE30F949625A3019201A1
:10CC80000F949625AB01BC0100E010E098018F2DB8
:10CC90000E94C96220E030E0A901C501B4010F94EF
:10CCA0003025F601E658F64EFA8BE98B882309F415
:10CCB0004DC0F2E000E010E020E431E4FF1619F08E
:10CCC00000E010E09801B501A4017058E12C8F2D0F
:10CCD0000E94C962A5019401C501B4010F94002C02
:10CCE0006B8B7C8B8D8B9E8B22E0F216E9F0F10131
:10CCF000E958F64E6491611107C00E94174E85E510
:10CD000099E10E9444386AE070E090E080E00F947E
:10CD100035259B01AC0160E070E088E492E40F945B
:10CD2000FA2C8B019C0104C000E010E020EC30E400
:10CD3000EE24E3944B895C896D897E898F2D0E9456
:10CD4000C96232E0F312D0C00E948B5481E090E0BF
:10CD5000A0E0B0E00F2C04C0880F991FAA1FBB1FD2
:10CD60000A94D2F720913F0C282B20933F0C20915E
:10CD7000B505822B8093B50589899A890E946C1D1F
:10CD8000F601EF59FD4F608371838283938382E0C4
:10CD9000F8121AC02091871230918812409189129E
:10CDA00050918A126091690270916A0280916B02BF
:10CDB00090916C020F94FF2B6093690270936A024A
:10CDC00080936B0290936C02F601EF5EF74F108236
:10CDD0001182128213828F2D0E94891C0E94E52AE3
:10CDE000F601EF59FD4F80819181A281B381F60157
:10CDF000E557F84F80839183A283B38392E0F916BD
:10CE0000A9F18CE0EEEBF2E0DE01119601900D92BB
:10CE10008A95E1F7E1E0F0E0EC0FFD1FEC0DFD1D60
:10CE200080809180A280B38020E030E0A901C5011C
:10CE3000B4010F94302581111EC066960FB6F89488
:10CE4000DEBF0FBECDBFDF91CF911F910F91FF903D
:10CE5000EF90DF90CF90BF90AF909F908F907F909A
:10CE60006F905F904F903F902F9008950E94AC6517
:10CE70008111E3CFC6CF20E030E0A901C501B401A4
:10CE80000F94602E87FF04C0B7FAB094B7F8B0943F
:10CE9000F601EF59FD4F6F01A3019201C501B401E5
:10CEA0000F9496259B01AC01F6016081718182810E
:10CEB00093810F94FF2BF6016083718382839383A8
:10CEC000F2E080E090E0A0E4B1E4FF1621F080E021
:10CED00090E0A8E4B2E48D879E87AF87B88BCE013F
:10CEE0000D960E94CA2AA9CF81E090E0A0E0B0E0B0
:10CEF0000F2C04C0880F991FAA1FBB1F0A94D2F7DA
:10CF000020913F0C282B20933F0C2091B505822BBC
:10CF10008093B50589899A890E946C1DF601EF59A5
:10CF2000FD4F60837183828393834ECFCF93DF93D2
:10CF300000D01F92CDB7DEB780E090E0A0EAB0E469
:10CF400089839A83AB83BC8361E0CE0101960E9402
:10CF5000D6640F900F900F900F90DF91CF910895AE
:10CF60008F929F92AF92BF92CF92DF92EF92FF92F9
:10CF70000F931F93CF93DF93CDB7DEB72C970FB6E8
:10CF8000F894DEBF0FBECDBF8B0140E050E068E4F7
:10CF900072E44D835E836F83788740E050E060EAFF
:10CFA00070E449875A876B877C878130B9F182307A
:10CFB00009F459C020E030E040E050E4609169029B
:10CFC00070916A0280916B0290916C020F94002C18
:10CFD0004B017C0120E030E048EC53E40F94602EDC
:10CFE000181634F4812C912C88ECE82E93E4F92E59
:10CFF000F801A084B184C284D3849401A701B5014F
:10D00000C6010F94602E181614F054016701C50173
:10D01000D60189839A83AB83BC8348C0BE01675F16
:10D020007F4FC80108960E948E64B8016C5F7F4FE5
:10D03000AE014B5F5F4FC8010E946C640E94993043
:10D040002C960FB6F894DEBF0FBECDBFDF91CF9107
:10D050001F910F91FF90EF90DF90CF90BF90AF9016
:10D060009F908F900895F8012085318542855385E2
:10D070006091690270916A0280916B0290916C02DA
:10D080000F94002C6B017C0120E030E048EC53E46D
:10D090000F94302587FD06C0C12CD12C28ECE22E40
:10D0A00023E4F22EC982DA82EB82FC82BE01675F42
:10D0B0007F4FCE010196B7CFEF92FF920F931F9350
:10D0C000CF93DF937C018B010E949331C1E6D2E0C4
:10D0D000209171023091720240917302509174025A
:10D0E000F70160817181828193810F94FA2C2C85E4
:10D0F0003D854E855F850F94002C6C877D878E87DC
:10D100009F87C8010E94CA2ADF91CF911F910F917A
:10D11000FF90EF900C9483614F925F926F927F9299
:10D12000AF92BF92CF92DF92EF92FF920F931F9335
:10D13000CF93DF9300D000D01F921F92CDB7DEB700
:10D140005C0180E090E0A0E7B2E489839A83AB833E
:10D15000BC8380E090E0A0E8B0EC8D839E83AF8339
:10D16000B887BE016F5F7F4FCE0105960E945C6855
:10D1700068E873E180E090E00E94EF25C12CD12C9B
:10D1800088ECE82E81E4F82EC982DA82EB82FC82F8
:10D1900080E090E0A0E8B0E48D839E83AF83B88701
:10D1A000BE016F5F7F4FCE0105960E945C6805E46B
:10D1B0001CE0F80140AC51AC62AC73ACC0AED1AE77
:10D1C000E2AEF3AE80E090E0A0E2B2E489839A831D
:10D1D000AB83BC83F50180819181A281B3818D8372
:10D1E0009E83AF83B887BE016F5F7F4FCE010596E8
:10D1F0000E945C68F80140AE51AE62AE73AE129A06
:10D2000064E670E080E090E00E94EF2581E02896DF
:10D210000FB6F894DEBF0FBECDBFDF91CF911F9147
:10D220000F91FF90EF90DF90CF90BF90AF907F90E5
:10D230006F905F904F9008951F93CF93DF93CDB77A
:10D24000DEB72C970FB6F894DEBF0FBECDBF182FF8
:10D25000882379F020E030E0A9016091ED0570911C
:10D26000EE058091EF059091F0050F94302588230D
:10D27000F9F08091400C8117D9F00E9483618CE015
:10D28000EAECF2E0DE01119601900D928A95E1F749
:10D29000CE0101960E94181F8091400C882391F0C6
:10D2A00081E692E00E94F1261092400C0E94E52A4D
:10D2B0002C960FB6F894DEBF0FBECDBFDF91CF9195
:10D2C0001F91089581E08093400C81E692E00E94D6
:10D2D0000521ECCF2F923F924F925F926F927F92F7
:10D2E0008F929F92AF92BF92CF92DF92EF92FF9276
:10D2F0000F931F93CF93DF93CDB7DEB7CB54D109F4
:10D300000FB6F894DEBF0FBECDBF2DB73EB739AF15
:10D3100028AF87E00E94274E81110BC061E086E5AF
:10D320000E943D248DA3853060F087E39EE00E943B
:10D330004438A8ADB9AD0FB6F894BEBF0FBEADBFAF
:10D3400040C33DA1332321F087E19EE00E94443891
:10D350006AE080E50E943D24182F8CEF810F8F3208
:10D3600018F083EF9DE0E3CF60E085E40E9459244C
:10D37000882309F448C081E08FABE0908B12F090D5
:10D380008C12D7012D913D914D915C91609161027C
:10D390007091620280916302909164020F94002C5C
:10D3A000AB01BC0188E50E94AB2469877A878B8733
:10D3B0009C87F70124813581468157816091650200
:10D3C0007091660280916702909168020F94002C20
:10D3D000AB01BC0189E50E94AB246D877E878F87F6
:10D3E000988BBE01635F7F4FCE0109960E94392E54
:10D3F000382E81110BC063E68FED9DE00E94B23F95
:10D4000087EC9DE094CF92E09FABB7CF8CE40E9475
:10D410002D1E082F882309F431C10E9429248EA3D0
:10D42000803118F080EA9DE082CFFEA1F13009F44E
:10D4300027C160E083E50E9459248AAF882321F048
:10D44000011102C037E03EA38DA1833020F086E8B1
:10D450009DE00E9444389091400C9DAF80E00E9476
:10D460001C690E94C21C1D8A1E8A1F8A188E198E72
:10D470001A8E1B8E1C8E83EF9FE4A3ECB7E48D8F76
:10D480009E8FAF8FB8A383EF9FE4A3ECB7EC89A383
:10D490009AA3ABA3BCA3A12FB0E0BCA7ABA7EDB7E9
:10D4A000FEB724E0129FE019F10911240FB6F89499
:10D4B000FEBF0FBEEDBF8DB79EB701969CAF8BAF81
:10D4C0002DA14FA9BE01635F7F4FCE0109960E9437
:10D4D00069F99B01AC010F94F22E811162C20E9486
:10D4E0000BFD611571058105910511F00F94B620B2
:10D4F000212C1BAA1CAA1DAA1EAAAEA1A150BB0BBF
:10D500002C96BFAFAEAF2C97E22DF0E0F8A7EFA3BB
:10D510002BA53CA5E217F3070CF074C23196FEA7C9
:10D52000EDA73F932F93FF93EF9382E79DE09F93A7
:10D530008F938CE79DE09F938F931F920E94F8F842
:10D540008DB79EB709960FB6F8949EBF0FBE8DBFDC
:10D550009EA1992309F458C10F9467202AE030E076
:10D5600040E050E00F94962B0F94372520E030E0F8
:10D5700040EA50E40F94602E0FEF1FEF181614F0DE
:10D5800001E010E00F94672028E631E040E050E031
:10D590000F94962B0F9437252B013C010F94672095
:10D5A00028E230E040E050E00F94962B6B5F7F4F15
:10D5B0008F4F9F4F0F9437254B015C01ADA1A430D5
:10D5C000D1F4BC01A40184E69DE00E942041B30196
:10D5D000A2018CE59DE00E94204186E59DE00E942D
:10D5E00044380130110519F483E40E940B3882E5B8
:10D5F0009DE00E944438312CC801110FAA0BBB0BCF
:10D600002A968CAF9DAFAEAFBFAF2A972C96AEAD2A
:10D61000BFAD2C973A161B060CF0F6C02A966CADDF
:10D620007DAD8EAD9FAD2A970F9437256B017C01A0
:10D63000BAADBB2341F1AC019B010F94002C20E05B
:10D6400030E040E952E40F9496259B01AC01C30100
:10D65000B2010F94002C2B013C0120E030E044EBA0
:10D6600053E40F94602E1816FCF420E030E044EBF5
:10D6700053E4C301B2010F94FF2BEDCF1EA2D9CE0C
:10D6800022E02EA3D6CE0F94672024E130E040E0C4
:10D6900050E00F94962B675E7F4F8F4F9F4F0F94F4
:10D6A0003725A7019601CFCF20E030E0A901C301C3
:10D6B000B2010F94302587FF0BC020E030E044EB2F
:10D6C00053E4C301B2010F94002C2B013C01ECCFB9
:10D6D00000918B1210918C12F801248135814681C2
:10D6E00057816D857E858F8598890F94FF2B2296B3
:10D6F0006CAF7DAF8EAF9FAF22972BED3FE049E43B
:10D7000050E4C301B2010F94962520E030E044E3D9
:10D7100053E40F94FA2C6B017C010F94F52C6FA746
:10D7200078AB89AB9AABD8012D913D914D915C912D
:10D7300069857A858B859C850F94FF2B26966CAF27
:10D740007DAF8EAF9FAF2697A50194016FA578A9F5
:10D7500089A99AA90F9496259B01AC0126966CADD8
:10D760007DAD8EAD9FAD26970F94002C69837A8393
:10D770008B839C83C701B6010F94A02EA501940151
:10D780000F94962522962CAD3DAD4EAD5FAD229700
:10D790000F94002C6D837E838F83988748E651E039
:10D7A00070E060E0CE0101960E94C9C148E651E0F8
:10D7B00070E060E0CE0105960E94C9C1BDA1B43001
:10D7C00099F449815A816B817C8186E49DE00E94B5
:10D7D00020414D815E816F8178858DE29FE20E94BC
:10D7E00020418AE00E940B38198A1A8A1B8A1C8AF7
:10D7F000AE014F5E5F4FBE016B5F7F4FCE01019662
:10D800000E946C64339402CF20E04FA9BE01635F95
:10D810007F4FCE0109960E9469F94B015C01312CC2
:10D82000AC019B010F94F22E811102C0332433947A
:10D83000A5019401C501B4010F94F22E8111E2C03B
:10D84000EFA1F8A5EE0FFF1FEE0FFF1F2BAD3CADB4
:10D85000E20FF31F80829182A282B382A50194011C
:10D860006D8D7E8D8F8D98A10F94602E181624F4E7
:10D870008D8E9E8EAF8EB8A2A501940169A17AA16A
:10D880008BA19CA10F94302587FF04C089A29AA286
:10D89000ABA2BCA2A50194016BA97CA98DA99EA9EC
:10D8A0000F94002C6BAB7CAB8DAB9EABADA5BEA536
:10D8B000BD01BB0F880B990B0F9437256FA378A779
:10D8C00089A79AA79B01AC016BA97CA98DA99EA9E8
:10D8D0000F94FA2C2B013C014D8A5E8A6F8A788E58
:10D8E000EBADFCADF8ABEFA710E0C12CD12C76016D
:10D8F000AFA5B8A96D917D918D919D91B8ABAFA762
:10D90000A30192010F94FF2B9B01AC010F9496256C
:10D910009B01AC01C701B6010F94002C6B017C0187
:10D920001F5F211628F72FA138A549A55AA50F94E6
:10D93000FA2C0F94AE2E698F7A8F8B8F9C8FBDA19E
:10D94000B23068F18DA59EA50E9428E16BA57CA54B
:10D9500081E49DE00E9442418BE39DE00E944438B7
:10D9600043E0C501B4010E944BBA80E20E940B382B
:10D9700081E0EDA1E3300CF480E0E12C8E010F5D3D
:10D980001F4F9E01235E3F4FAE01475E5F4FBE01BA
:10D990006B5E7F4F0E94013F8AE00E940B38239408
:10D9A000B3CD0E94AC650E94A91C8DAD0E941C697C
:10D9B0000E94993088AD99AD0FB6F8949EBF0FBE06
:10D9C0008DBFE8ADF9AD0FB6F894FEBF0FBEEDBF49
:10D9D000C55BDF4F0FB6F894DEBF0FBECDBFDF9142
:10D9E000CF911F910F91FF90EF90DF90CF90BF905C
:10D9F000AF909F908F907F906F905F904F903F90EF
:10DA00002F9008950E94AC65332069F280E39DE079
:10DA10000E94443881E0FDA11F160CF080E0EE2446
:10DA2000E3948E010F5D1F4F9E01235E3F4FAE01B9
:10DA3000475E5F4FBE016B5E7F4F0E94013F698D65
:10DA40007A8D8B8D9C8D0052110926E042E00F9457
:10DA5000FD1F9F938F938FE19DE09F938F9389E2AA
:10DA60009DE09F938F931F920E94F8F82DB73EB7C9
:10DA7000295F3F4F0FB6F8943EBF0FBE2DBF93CF27
:10DA80002F923F924F925F926F927F928F929F92CE
:10DA9000AF92BF92CF92DF92EF92FF920F931F93BC
:10DAA000CF93DF93CDB7DEB76A970FB6F894DEBF9A
:10DAB0000FBECDBF83E50E942D1E182F3090400C65
:10DAC000882319F00E944924382E4090610250901A
:10DAD000620260906302709064028091650290918E
:10DAE0006602A0916702B09168028B8B9C8BAD8B14
:10DAF000BE8B8091690290916A02A0916B02B091F5
:10DB00006C028F8B988FA98FBA8F112329F0311057
:10DB100003C080E00E941C6986E50E942D1E8A8B4E
:10DB200020E030E0A9016091ED057091EE05809153
:10DB3000EF059091F0050F943025882309F4C9C0B2
:10DB400083E40E942D1E882309F49DC00E94812435
:10DB50006B017C01A7EAB7E0B987A887BF83AE83D2
:10DB6000F5E0FD831D861E8628EC2F8702EC1A86C1
:10DB7000212C88EC8B8792E49C87AE81BF81B98B86
:10DB8000A88B15E0E889F98981909190A190B190D6
:10DB9000F98BE88B2A85322D4B855C85C501B40154
:10DBA0000F94302587FF04C08A86292CAB86BC865B
:10DBB0002D853E854F85502FC501B4010F94602EF1
:10DBC000181624F48D869E86AF860B2D1150D1F643
:10DBD000FD81F150FD838E819F8144969F838E83CA
:10DBE000F111CBCF2D853E854F85502F6A85722D43
:10DBF0008B859C850F94002C20E030E040E05FE3B3
:10DC00000F949625A70196010F94002C4B015C01FF
:10DC10002DEB37E346E855EB0F94602E87FD0AC0E5
:10DC20002DEB37E346E855E3C501B4010F943025E9
:10DC300018164CF580E00E941C6910E0E884F98415
:10DC400000E0D7016D917D918D919D917D016D01D8
:10DC5000B4E0CB1AD108A50194010F94FF2BF60173
:10DC60006083718382839383602F812F0E94CDF71D
:10DC70000F5F053031F71F5F888599854496998736
:10DC800088871530D9F6AA89AA2381F020E030E0F0
:10DC9000A9016091ED057091EE058091EF059091DD
:10DCA000F0050F94302581110E9489408AE50E9479
:10DCB0002D1E882351F00E94812469837A838B83EF
:10DCC0009C83CE0101960E9495F6832D0E941C69CB
:10DCD0000BC0311003C09A89992341F30E94174E5B
:10DCE00080E69CE00E944438332051F08091400C43
:10DCF000811106C00E94134E81E49CE00E944438CA
:10DD00000E94174E83E39CE00E9444388091400CAF
:10DD10000E9402410E94174E86E29CE00E94443815
:10DD2000C090E308D090E408E090E508F090E608A1
:10DD300020E030E0A901C701B6010F94602E18164B
:10DD40000CF053C042E0C701B6010E944BBA8DE00F
:10DD50000E940B388AE00E940B38A3019201609167
:10DD600061027091620280916302909164020F944B
:10DD7000302581111FC02B893C894D895E896091B6
:10DD800065027091660280916702909168020F941B
:10DD9000302581110FC02F89388D498D5A8D6091A2
:10DDA000690270916A0280916B0290916C020F94EB
:10DDB000302581110E9499306A960FB6F894DEBF23
:10DDC0000FBECDBFDF91CF911F910F91FF90EF90CC
:10DDD000DF90CF90BF90AF909F908F907F906F908B
:10DDE0005F904F903F902F90089581E29CE00E94B9
:10DDF0004438B3CF8F929F92AF92BF92EF92FF922F
:10DE00000F931F93CF93DF9380E00E941C691092C1
:10DE1000E9051092EA051092EB051092EC051092BC
:10DE2000E5051092E6051092E7051092E8051092BC
:10DE3000F1051092F2051092F3051092F40510927C
:10DE4000ED051092EE051092EF051092F00507EA2D
:10DE500017E0C0E0812C912C80ECA82E8FE7B82E23
:10DE60007801D0E0F70181929192A192B1927F0165
:10DE70006D2F8C2F0E94CDF7DF5FD53099F7CF5FE4
:10DE80000C5E1F4FC53061F7DF91CF911F910F914D
:10DE9000FF90EF90BF90AF909F908F9008959091DA
:10DEA000901280919112981308C080911B09909153
:10DEB0001C09892B11F40C94E71E80E00E941F5A64
:10DEC000EECF83E50E947B1E8823E9F00E940BFDC4
:10DED00060937D1170937E1180937F1190938011D8
:10DEE0000E94812420E030E04AE754E40F94962514
:10DEF0000F94732D60931302709314028093150294
:10DF000090931602089580914B0584FD0AC080917C
:10DF10004D0587FD06C080914E05837011F40C9469
:10DF20004F6F0E94836188E50E942D1E882331F087
:10DF30005F9A80913F0C8E7F80933F0C89E50E9411
:10DF40002D1E882331F08A9A80913F0C8D7F80931B
:10DF50003F0C8AE50E942D1E882359F0809108010C
:10DF6000809581708093060180913F0C8B7F809318
:10DF70003F0C85E40E942D1E81110C94E51E08952E
:10DF80002F923F924F925F926F927F928F929F92C9
:10DF9000AF92BF92CF92DF92EF92FF920F931F93B7
:10DFA000CF93DF93CDB7DEB7A6970FB6F894DEBF59
:10DFB0000FBECDBF8BE897E00E94122A8091FD0B27
:10DFC00083FD7EC020916D0230916E0240916F0200
:10DFD000509170026091970770919807809199070E
:10DFE00090919A070F943025882309F469C0109105
:10DFF0001A09111161C080915F029091600201972E
:10E000002091F2113091F311281739073CF40E9446
:10E01000174E88E299E10E94443811E020916D0288
:10E0200030916E0240916F0250917002609197079B
:10E03000709198078091990790919A070F94FF2B00
:10E040006B017C0120E030E0A9010F94602E87FF76
:10E0500004C0F7FAF094F7F8F0942091710230912F
:10E0600072024091730250917402C701B6010F947D
:10E07000962520E030E84BE354E40F94602E181608
:10E08000ECF40E94174E89E099E10E944438809197
:10E09000970790919807A0919907B0919A0780935C
:10E0A0006D0290936E02A0936F02B093700287E9A5
:10E0B00097E00E94946104C010E0B0CF1111E7CF47
:10E0C0002AE037ED43E25CE3609141027091420245
:10E0D00080914302909144020F9496256B017C013C
:10E0E0006091770270917802072E000C880B990BD3
:10E0F0000F9437259B01AC01C701B6010F949625FB
:10E10000698B7A8B8B8B9C8B8091400C882309F1D7
:10E110008090E3089090E408A090E508B090E608AD
:10E12000C0909307D0909407E0909507F0909607E1
:10E1300020E030E0A901C501B4010F943025882307
:10E14000D1F1A7019601C501B4010F94602E1816F4
:10E1500094F1C12CD12C76018E010F5E1F4F27E95F
:10E1600037E043E957E06FE877E08BE897E00E94FB
:10E170004EF480E1EBE8F7E0A1E6B2E001900D9209
:10E180008A95E1F7A6960FB6F894DEBF0FBECDBF15
:10E19000DF91CF911F910F91FF90EF90DF90CF9083
:10E1A000BF90AF909F908F907F906F905F904F90B7
:10E1B0003F902F900895209161023091620240912A
:10E1C00063025091640260918B0770918C0780917B
:10E1D0008D0790918E070F94FF2B6D8B7E8B8F8B0D
:10E1E000988F2091650230916602409167025091AC
:10E1F000680260918F0770919007809191079091CC
:10E2000092070F94FF2B698F7A8F8B8F9C8F2091B1
:10E21000690230916A0240916B0250916C02C70111
:10E22000B6010F94FF2B6D8F7E8F8F8F98A3209157
:10E230006D0230916E0240916F02509170026091B8
:10E240009707709198078091990790919A070F947A
:10E25000FF2B6B017C0120E030E0A9016D897E89F4
:10E260008F89988D0F94302581110CC020E030E00B
:10E27000A901698D7A8D8B8D9C8D0F943025882313
:10E2800009F467CF2D893E894F89588DCA01B9019C
:10E290000F9496254B015C01298D3A8D4B8D5C8D39
:10E2A000CA01B9010F9496259B01AC01C501B401C7
:10E2B0000F94002C4B015C012D8D3E8D4F8D58A18C
:10E2C000CA01B9010F9496259B01AC01C501B401A7
:10E2D0000F94002C4B015C01A7019601C701B60108
:10E2E0000F9496259B01AC01C501B4010F94002C3D
:10E2F0000F94AE2E4B015C012DEB37E346E855E35E
:10E300000F94302587FF0FC020E030E0A901C7013E
:10E31000B6010F94602E4601570187FF04C0B7FA7B
:10E32000B094B7F8B0942DEB37E346E855E3C50158
:10E33000B4010F94302587FD1CCF20E030E040EA87
:10E3400051E4C501B4010F94FA2C0F94732D1B01F5
:10E35000672B19F422242394312CB10190E080E042
:10E360000F9435259B01AC0160E070E080E89FE3ED
:10E370000F94FA2C2B013C01AC019B01C501B401A7
:10E380000F9496254B015C01A30192016D897E8952
:10E390008F89988D0F9496256D8B7E8B8F8B988FA0
:10E3A000A3019201698D7A8D8B8D9C8D0F9496259A
:10E3B000698F7A8F8B8F9C8FA30192016D8D7E8DDB
:10E3C0008F8D98A10F9496256D8F7E8F8F8F98A338
:10E3D000A3019201C701B6010F94962569A37AA300
:10E3E0008BA39CA380E1E1E6F2E08E010F5F1F4F5B
:10E3F000D80101900D928A95E1F70E940BFD2B0147
:10E400003C0128EC420E511C611C711C0DA31EA383
:10E4100081E0281A310809F460C00E940BFD8B01CD
:10E420009C01041915092609370937FD59C02B012C
:10E430003C0128EC420E511C611C711C80E00E94C2
:10E440001F5A2D893E894F89588D69817A818B8128
:10E450009C810F94002C69837A838B839C83298D04
:10E460003A8D4B8D5C8D6D817E818F8198850F9467
:10E47000002C6D837E838F8398872D8D3E8D4F8DED
:10E4800058A169857A858B859C850F94002C6987B6
:10E490007A878B879C8729A13AA14BA15CA16D85C6
:10E4A0007E858F8598890F94002C6D877E878F8756
:10E4B000988B750164018E010F5E1F4F9E01235FD3
:10E4C0003F4FAE01475F5F4FBE016B5F7F4F8DA136
:10E4D0009EA10E944EF481119BCF750164013CCE38
:10E4E0000E940BC2AECF8F929F92AF92BF92CF92FB
:10E4F000DF92EF92FF92CF93DF9380904102909052
:10E500004202A0904302B0904402FC01C080D1803E
:10E51000E280F38020E030E0A901C701B6010F944A
:10E520003025882341F0C0924102D0924202E0920D
:10E530004302F0924402C0917702D091780284E6BF
:10E5400090E09093780280937702C0907102D0900F
:10E550007202E0907302F090740280E090E0A0E814
:10E56000BFE38093710290937202A0937302B09301
:10E5700074020E94C06F8092410290924202A09267
:10E580004302B0924402D0937802C0937702C092C3
:10E590007102D0927202E0927302F0927402DF91E3
:10E5A000CF91FF90EF90DF90CF90BF90AF909F9072
:10E5B0008F9008950F931F93CF93DF9300D01F92F6
:10E5C000CDB7DEB79C010BE817E090E1E1E6F2E0A1
:10E5D000D80101900D929A95E1F7F90120813181DE
:10E5E00042815381F80160857185828593850F94FE
:10E5F000002CF801608771878287938780E090E024
:10E60000A0EAB0E489839A83AB83BC83CE010196F0
:10E610000E9473720F900F900F900F90DF91CF9127
:10E620001F910F9108952F923F924F925F926F9298
:10E630007F928F929F92AF92BF92CF92DF92EF9292
:10E64000FF921F93CF93DF93CDB7DEB72C970FB612
:10E65000F894DEBF0FBECDBF7A011901DC012D9108
:10E660003D914D915C912D833E834F835887FB01F3
:10E67000408051806280738080906102909062023D
:10E68000A0906302B0906402A50194016D817E8127
:10E690008F8198850F94302581110EC011E0A30160
:10E6A000920160916502709166028091670290917B
:10E6B00068020F943025811110E0D1012D913D9118
:10E6C0004D915C9129873A874B875C87F701C08021
:10E6D000D180E280F38020910B0230910C024091B6
:10E6E0000D0250910E02C701B6010F943025882308
:10E6F00009F44EC0C0920B02D0920C02E0920D02BF
:10E70000F0920E0280916D0290916E02A0916F02C4
:10E71000B09170024091650250916602609167026B
:10E720007091680280928B0790928C07A0928D075F
:10E73000B0928E0740938F07509390076093910794
:10E7400070939207C0929307D0929407E092950736
:10E75000F09296078093970790939807A093990754
:10E76000B0939A0720E030E040E05FE36091710CE5
:10E770007091720C8091730C9091740C0F9496258B
:10E7800069837A838B839C83CE0101960E94737286
:10E790002D813E814F81588520938B0730938C07C4
:10E7A00040938D0750938E0740928F0750929007A9
:10E7B0006092910770929207D1012D913D914D91F8
:10E7C0005C9160919707709198078091990790915B
:10E7D0009A070F94002C6093970770939807809383
:10E7E000990790939A0711112FC020E030E0A901FA
:10E7F00069857A858B859C850F943025811133C07E
:10E8000060E070E088EC92E469837A838B839C8378
:10E81000CE0101960E9473722C960FB6F894DEBF5B
:10E820000FBECDBFDF91CF911F91FF90EF90DF9092
:10E83000CF90BF90AF909F908F907F906F905F90A0
:10E840004F903F902F9008952AEF3EE74AE25FE312
:10E850006091750C7091760C8091770C9091780C8A
:10E860000F949625D1CF60E070E080EA91E4CCCFA0
:10E870000F931F93CF93DF9300D000D01F921F926E
:10E88000CDB7DEB78B01FC0123A5211102C00E9488
:10E8900056FB1D821E821F82188620E030E040E079
:10E8A0005FE36091690270916A0280916B029091BE
:10E8B0006C020F94002C69837A838B839C839E0166
:10E8C0002B5F3F4FAE014F5F5F4F65E672E081E621
:10E8D00092E00E9413731D821E821F82188620E020
:10E8E00030E040E05FE3F8016085718582859385C3
:10E8F0000F94002C69837A838B839C83B8016C5FAF
:10E900007F4F9E012B5F3F4FAE014F5F5F4FC801AE
:10E910000E94137328960FB6F894DEBF0FBECDBFCA
:10E92000DF91CF911F910F9108959B01AC01485F3A
:10E930005F4FBC016C5F7F4F0C9413732F923F921B
:10E940004F925F926F927F928F929F92AF92BF92FF
:10E95000CF92DF92EF92FF920F931F93CF93DF93AB
:10E96000CDB7DEB7A6970FB6F894DEBF0FBECDBF0A
:10E970008C011B015A8749874090610250906202C6
:10E9800060906302709064028090650290906602CD
:10E99000A0906702B0906802DB018D919D910D906F
:10E9A000BC91A02D8B8B9C8BAD8BBE8B9C01AD0144
:10E9B000C301B2010F94FF2B6B017C01D1011496AE
:10E9C0008D919D910D90BC91A02D8F8B988FA98FCB
:10E9D000BA8F9C01AD01C501B4010F94FF2B6B8F61
:10E9E0007C8F8D8F9E8FA985BA858D919D910D907D
:10E9F000BC91A02D8B879C87AD87BE879C01AD0104
:10EA0000C301B2010F94FF2B6F8F78A389A39AA340
:10EA1000A985BA8514968D919D910D90BC91A02DDC
:10EA20008F87988BA98BBA8B9C01AD01C501B4016E
:10EA30000F94FF2B6BA37CA38DA39EA3A70196012C
:10EA4000C701B6010F9496256B017C012B8D3C8D7F
:10EA50004D8D5E8DCA01B9010F9496259B01AC01C5
:10EA6000C701B6010F94002C4B015C012B893C8936
:10EA70004D895E896B857C858D859E850F94FF2BE6
:10EA80002B013C012F89388D498D5A8D6F857889EE
:10EA900089899A890F94FF2B6B017C01A301920154
:10EAA000C301B2010F9496252B013C01A7019601E9
:10EAB000C701B6010F9496259B01AC01C301B201B9
:10EAC0000F94002C0F94AE2E6B017C012F8D38A17A
:10EAD00049A15AA1CA01B9010F9496252B013C0105
:10EAE0002BA13CA14DA15EA1CA01B9010F949625AD
:10EAF0009B01AC01C301B2010F94002C9B01AC013E
:10EB0000C501B4010F94602E1816B4F520E030E072
:10EB1000A901C701B6010F94602E87FF2AC0C70163
:10EB2000B601905820E030E040EA50E40F94602EA7
:10EB3000181614F5A10169857A85C8010E949E7492
:10EB4000A6960FB6F894DEBF0FBECDBFDF91CF9172
:10EB50001F910F91FF90EF90DF90CF90BF90AF90FB
:10EB60009F908F907F906F905F904F903F902F90ED
:10EB70000895C701B601D6CF20E030E040E050E470
:10EB8000C501B4010F94602E181624F4B101C80118
:10EB90000E94387419821A821B821C82BE016F5F28
:10EBA0007F4FC1010E9495742DEC3CEC4CEC5CE372
:10EBB000C701B6010F9496259B01AC01F801608155
:10EBC0007181828193810F9496256D837E838F83DB
:10EBD0009887D8019B968C919B978823C9F02AE946
:10EBE00039E949E95FE314966D917D918D919C918E
:10EBF00017970F94962569837A838B839C83BE0134
:10EC00006F5F7F4F8BE897E00E949574F80113A621
:10EC1000BE016B5F7F4F89859A850E94957490CF66
:10EC20003F924F925F926F927F928F929F92AF929C
:10EC3000BF92CF92DF92EF92FF920F931F93CF93E9
:10EC4000DF93CDB7DEB76C970FB6F894DEBF0FBE7B
:10EC5000CDBFDB010C91142F100F153008F067C1E8
:10EC60001196DC90C22ECD0CB4E0BC1508F45FC147
:10EC7000ED2DF0E0EE5EFA4F8080912CB12CA12CAE
:10EC8000002E04C0B694A794979487940A94D2F760
:10EC900080FE4DC1EC2DF0E0EE5EFA4F8080912CAD
:10ECA000B12CA12C012E04C0B694A79497948794FC
:10ECB0000A94D2F780FE3BC1322E642F7C01409033
:10ECC000E5055090E6056090E7057090E8058091B5
:10ECD000ED059091EE05A091EF05B091F005898FBB
:10ECE0009A8FAB8FBC8F660F770B072E000C880BAB
:10ECF000990B0F9437254B015C01602F000F770BA8
:10ED0000880B990B0F943725298D3A8D4B8D5C8D8F
:10ED10000F949625A30192010F94002CA501940154
:10ED20000F94002C6D877E878F87988B612F110F32
:10ED3000770B880B990B0F943725298D3A8D4B8DC6
:10ED40005C8D0F949625A30192010F94002CA501D0
:10ED500094010F94FF2B69837A838B839C8340906B
:10ED6000E9055090EA056090EB057090EC05809104
:10ED7000F1059091F205A091F305B091F405898F0A
:10ED80009A8FAB8FBC8F632D660F770B072E000C0D
:10ED9000880B990B0F9437254B015C016D2DDD0C11
:10EDA000770B880B990B0F943725298D3A8D4B8D56
:10EDB0005C8D0F949625A30192010F94002CA50160
:10EDC00094010F94002C698B7A8B8B8B9C8B6C2D10
:10EDD000CC0C770B880B990B0F943725298D3A8D26
:10EDE0004B8D5C8D0F949625A30192010F94002CFE
:10EDF000A50194010F94FF2B6D837E838F839887E9
:10EE0000F70180859185A285B38589879A87AB872D
:10EE1000BC878D8B9E8BAF8BB88F47E651E061E04E
:10EE200070E0CE0141960E94C9C147E651E061E021
:10EE300070E0CE0105960E94C9C147E651E061E04D
:10EE400070E0CE010D960E94C9C147E651E061E035
:10EE500070E0CE0101960E94C9C189889A88AB886A
:10EE6000BC8827E137EB41ED58EBC501B4010F94A5
:10EE7000602E87FD5CC023E030E044EB53E4C50125
:10EE8000B4010F94302518160CF451C08D849E8463
:10EE9000AF84B88827E137EB41ED58EBC501B401E9
:10EEA0000F94602E87FD43C023E030E044EB53E431
:10EEB000C501B4010F9430251816CCF18D809E80C9
:10EEC000AF80B88427E137EB41ED58EBC501B401C1
:10EED0000F94602E87FD2BC023E030E044EB53E419
:10EEE000C501B4010F94302518160CF189809A8061
:10EEF000AB80BC8027E137EB41ED58EBC501B40195
:10EF00000F94602E87FD13C023E030E044EB53E400
:10EF1000C501B4010F94302518164CF0AE014F5FB7
:10EF20005F4FBE01635F7F4FC7010E949E746C9666
:10EF30000FB6F894DEBF0FBECDBFDF91CF911F910A
:10EF40000F91FF90EF90DF90CF90BF90AF909F9088
:10EF50008F907F906F905F904F903F9008952F9289
:10EF60003F924F925F926F927F928F929F92AF9259
:10EF7000BF92CF92DF92EF92FF920F931F93CF93A6
:10EF8000DF93CDB7DEB7CC58D1090FB6F894DEBF0A
:10EF90000FBECDBF80E19CE00E94443887E00E9414
:10EFA000274E81116EC084E50E947B1E882329F0C4
:10EFB0000E946E2481110E9439BA80E090E0A0E89E
:10EFC000BFE389839A83AB83BC838D839E83AF83A6
:10EFD000B8878DEC9CECACE4BEE389879A87AB875D
:10EFE000BC8780E090E0A0E2B1E48D879E87AF8788
:10EFF000B88B8CE390E09A8B898B8DEC90E09C8BA6
:10F000008B8B8DEC9CECACECBEE38D8B9E8BAF8B35
:10F01000B88F80E090E0A0EEBFE3898F9A8FAB8F2E
:10F02000BC8F1BA61CA64AE959E969E97EE38FE477
:10F030000E94AB246D8F7E8F8F8F98A360E083E456
:10F040000E94592489A360E08BE40E9459248AA37A
:10F0500082E40E947B1E882381F10E946E24009727
:10F0600061F19C01285231092536310520F16CE807
:10F0700070E082EE9BE00E9442418DED9BE00E9499
:10F080004438C457DF4F0FB6F894DEBF0FBECDBF74
:10F09000DF91CF911F910F91FF90EF90DF90CF9074
:10F0A000BF90AF909F908F907F906F905F904F90A8
:10F0B0003F902F9008959A8B898B8CE40E947B1E41
:10F0C0008823E1F00E9481246B017C01C986DA86E5
:10F0D000EB86FC8620E030E0A9010F94602E87FDCE
:10F0E0000AC020E030E040E050E4C701B6010F94D0
:10F0F000302518161CF485EB9BE0C1CF81E50E94FA
:10F100002D1E882331F180911B0590911C05892BC0
:10F11000E9F00E9481246B017C01CD82DE82EF82C6
:10F12000F8862DEC3CEC4CE45DE30F94602E87FDFB
:10F130000AC020E030E040E751E4C701B6010F9477
:10F140003025181634F484E89BE099CF89E59BE0DC
:10F1500096CF83E50E947B1E8823E9F00E948124DC
:10F160006B017C01CD8ADE8AEF8AF88E2DEC3CECB7
:10F170004CEC5DE30F94602E87FD0AC020E030E088
:10F1800040E050E4C701B6010F94302518161CF476
:10F1900082E39BE074CF80E50E942D1E882341F11D
:10F1A00080911B0590911C05892B19F48AEF9AE038
:10F1B00066CF8BA58F5F8BA70E9481246B017C019A
:10F1C000CD86DE86EF86F88A20E030E0A9010F9434
:10F1D000602E87FD0AC020E030E048EC51E4C70112
:10F1E000B6010F94302518161CF482ED9AE047CF33
:10F1F00086E40E947B1E8823E9F00E9481246B0133
:10F200007C01C98EDA8EEB8EFC8E20E030E040E887
:10F210005FE30F94602E87FD0AC020E030E040E8F5
:10F2200050E4C701B6010F94302518161CF489EA82
:10F230009AE025CFC98CDA8CEB8CFC8C8D889E886B
:10F24000AF88B88CA7019601C701B6010F94962527
:10F250009B01AC0160E070E084E490E40F94FA2C30
:10F2600029813A814B815C810F9496252B013C01C9
:10F27000A5019401C501B4010F949625A70196013B
:10F280000F9496252CEE31E548EB5DE30F94FA2CB4
:10F290009B01AC01C301B2010F94962569837A8367
:10F2A0008B839C8388E40E947B1E882379F00E94D4
:10F2B0006E24009759F09C01255A31092F303140B6
:10F2C00018F08BE79AE0DBCE9C8B8B8B85E50E9458
:10F2D0002D1E8823C9F00E940BFD61157105810563
:10F2E000910511F00F94B62080911B0590911C059B
:10F2F000892B91F00E948124609317057093180563
:10F300008093190590931A0582E50E942D1E8111A4
:10F3100008C087E49AE0B3CE60E070E088E492E44D
:10F32000EBCF80911B0590911C05892B61F00E9409
:10F330006E24AD969FAF8EAFAD97181619064CF0A0
:10F3400083E19AE09CCE8AE190E0AD969FAF8EAFCC
:10F35000AD9789E50E947B1E882381F10E9481245C
:10F360002091EB083091EC084091ED085091EE08A7
:10F370000F94FF2B6B017C0188E50E947B1E882384
:10F3800031F10E9481242091E7083091E8084091F2
:10F39000E9085091EA080F94FF2B6BA37CA38DA37F
:10F3A0009EA3CFA2D8A6E9A6FAA6CE0183960E9474
:10F3B000EC1D811115C089EE99E061CEC090650207
:10F3C000D0906602E0906702F0906802D5CF60911D
:10F3D0006102709162028091630290916402DDCFBC
:10F3E00084E40E942D1E91E089270E941C6980E020
:10F3F00090E0A0EAB0E48DA79EA7AFA7B8AB60E00D
:10F40000CE018D960E94D66490911008CD57DF4FA3
:10F410009883C358D040109210080E94E61B88ECD5
:10F4200099E00E94443889899A898A3191050CF0C3
:10F4300044C08B899C890E94031F61E080E00E9488
:10F44000D9BC811142C06FEF8DED99E00E94B23FAF
:10F450008CA5811104C0CE0101960E9456FB80E06C
:10F4600090E0A0EAB0E48093930790939407A09370
:10F470009507B09396071DA61EA61FA618AABE0143
:10F48000635D7F4F8BE897E00E949574CD57DF4F07
:10F490005881C358D040509310080E94E61B8AA19F
:10F4A0008111EFCD10928A11109289110E9491BEA4
:10F4B00090E080E00E94031FE4CD0E94412281E0A1
:10F4C0000E9462BB8111B5CFBECF10926D02109227
:10F4D0006E0210926F02109270028DE692E00E940E
:10F4E00094618BA5882309F452C020E030E040E706
:10F4F00051E46091750C7091760C8091770C90912D
:10F50000780C0F94FA2C6DA77EA78FA798AB80E19B
:10F51000E1E6F2E0ABE8B7E001900D928A95E1F701
:10F520002D853E854F855889609197077091980782
:10F530008091990790919A070F94002C60939707F8
:10F54000709398078093990790939A07CE018D96B0
:10F550000E9473722D853E854F855889609197076B
:10F56000709198078091990790919A070F94FF2BBB
:10F5700060939707709398078093990790939A07E1
:10F580008CA5811104C0CE0101960E9456FBE2E1D8
:10F59000F5E085E0DF011D928A95E9F780E1E1E67B
:10F5A000F2E0ABE8B7E001900D928A95E1F789852A
:10F5B0009A85AB85BC858093930790939407A0931D
:10F5C0009507B09396071DA61EA61FA618AABE01F2
:10F5D000635D7F4F8BE897E00E949574BE01635E88
:10F5E0007F4F8BE897E00E94957489A1882309F4E6
:10F5F0001CC42091610230916202409163025091DB
:10F600006402E5962CAF3DAF4EAF5FAFE5978091BA
:10F61000650290916602A0916702B0916802E1963E
:10F620008CAF9DAFAEAFBFAFE197312C212C9FEFD8
:10F63000A4969FAFA497AFEFA896AFAFA897BFEFE0
:10F64000C158DF4FB883CF57D040EFE4C058DF4FE9
:10F65000E883C058D040F3ECCF57DF4FF883C15850
:10F66000D04027E4CE57DF4F2883C258D04081E0F6
:10F6700090E0A0E0B0E0022C04C0880F991FAA1F00
:10F68000BB1F0A94D2F7CC57DF4F88839983AA8394
:10F69000BB83C458D040A2E1B5E0E796BFAFAEAFA0
:10F6A000E79710E000E09101032C000C440B550B90
:10F6B000C857DF4F288339834A835B83C858D040BB
:10F6C000C457DF4F2882CC58D040E796AEADBFADCF
:10F6D000E7978D91E796BFAFAEAFE79790E0B0E0C8
:10F6E000A0E0CC57DF4F288139814A815B81C45823
:10F6F000D04082239323A423B523892B8A2B8B2BE1
:10F7000009F024C1C857DF4F688179818A819B81C4
:10F71000C858D0400F9437252091ED053091EE0563
:10F720004091EF055091F0050F9496252091E50545
:10F730003091E6054091E7055091E8050F94002CC3
:10F74000EB966CAF7DAF8EAF9FAFEB97B801012EFC
:10F75000000C880B990B0F9437252091F1053091FF
:10F76000F2054091F3055091F4050F9496252091F0
:10F77000E9053091EA054091EB055091EC050F94B5
:10F78000002C6B017C01EB962CAD3DAD4EAD5FAD19
:10F79000EB97E5966CAD7DAD8EAD9FADE5970F9483
:10F7A000FF2B2B013C01A7019601E1966CAD7DADCD
:10F7B0008EAD9FADE1970F94FF2B4B015C01A30130
:10F7C0009201C301B2010F9496252B013C01A501C2
:10F7D0009401C501B4010F9496259B01AC01C301AE
:10F7E000B2010F94002C0F94AE2E4B015C01EB96EE
:10F7F0002CAD3DAD4EAD5FADEB976BA17CA18DA166
:10F800009EA10F94FF2B2B013C01A70196016FA134
:10F8100078A589A59AA50F94FF2B6B017C01A30104
:10F820009201C301B2010F9496252B013C01A7015F
:10F830009601C701B6010F9496259B01AC01C30147
:10F84000B2010F94002C0F94AE2E20E030E040E780
:10F8500051E40F94FA2CA50194010F94002C6B0134
:10F860007C018090170590901805A0901905B09024
:10F870001A0520E030E040E85FE3C501B4010F94D1
:10F88000602E1816F4F4C501B4010F946C2D4B01D1
:10F890005C0160E070E0CB01181419041A041B0429
:10F8A00034F40F946720A50194010F94962B0F94C4
:10F8B00037259B01AC01B601C7010F94002C6B01E9
:10F8C0007C01C158DF4F2881CF57D040C058DF4F4F
:10F8D0003881C058D040CF57DF4F4881C158D04001
:10F8E000CE57DF4F5881C258D040B601C7010F94A0
:10F8F000302587FF2BC0A4960FAFA497C457DF4FC6
:10F900003881CC58D040A8963FAFA897EC96CFAEA0
:10F91000EC97ED96DFAEED97EE96EFAEEE97EF96A5
:10F92000FFAEEF97C158DF4FC882CF57D040C058C5
:10F93000DF4FD882C058D040CF57DF4FE882C15840
:10F94000D040CE57DF4FF882C258D0400F5F1F4FD4
:10F950000530110509F0B9CE4FEF241A340A55E0ED
:10F960002516310409F083CEA4968FADA497E82F15
:10F97000F0E0EE5EFA4F208181E090E0A0E0B0E0A0
:10F98000A8960FACA89704C0880F991FAA1FBB1F89
:10F990000A94D2F7822B8083A8969FADA8976A9687
:10F9A0009FAF6A97A496AFADA4976B96AFAF6B97D6
:10F9B000EC968FADEC97ED969FADED97EE96AFADD3
:10F9C000EE97EF96BFADEF976F968CAF9DAFAEAF52
:10F9D000BFAF6F97A896BFADA897BF3F09F409C204
:10F9E000A496EFADA497EF3F09F403C26B2FBB0FB2
:10F9F000770B880B990B0F9437252091ED053091EB
:10FA0000EE054091EF055091F0050F949625209159
:10FA1000E5053091E6054091E7055091E8050F9422
:10FA2000002C162F072F382E292E862F902FA32D2E
:10FA3000B22D65968CAF9DAFAEAFBFAF6597A49664
:10FA4000FFADA4976F2FFF0F770B880B990B0F94C7
:10FA500037252091F1053091F2054091F305509141
:10FA6000F4050F9496252091E9053091EA0540911F
:10FA7000EB055091EC050F94002C6B017C0169960D
:10FA8000CCAEDDAEEEAEFFAE6997CE018F5A9F4F82
:10FA90000E94EC1D882309F4B0C120E030E040EA68
:10FAA00050E4612F702F832D922D0F94002C4B0169
:10FAB0005C01CB01D50121968CAF9DAFAEAFBFAF3E
:10FAC00021972596CCAEDDAEEEAEFFAE2597A8967B
:10FAD0002FADA8972111E3C1A4963FADA497311192
:10FAE000B3C120E030E040EA50E4C701B6010F9412
:10FAF000002C6B017C01A4964FADA497442309F41C
:10FB0000C5C1A4968FADA49784300CF0BFC122ED7F
:10FB1000422E23E5522E2BE7622E21E4722E2196EF
:10FB20008CAC9DACAEACBFAC219725968CAD9DAD99
:10FB3000AEADBFAD2597A7968CAF9DAFAEAFBFAFB3
:10FB4000A7979C01AD0169966CAD7DAD8EAD9FAD63
:10FB500069970F94FF2BAB966CAF7DAF8EAF9FAFC5
:10FB6000AB97A501940165966CAD7DAD8EAD9FAD53
:10FB700065970F94FF2B2D966CAF7DAF8EAF9FAF27
:10FB80002D97AB962CAD3DAD4EAD5FADAB9761966D
:10FB90002CAF3DAF4EAF5FAF6197A501940160916F
:10FBA00061027091620280916302909164020F94ED
:10FBB000FF2B4B015C01A7962CAD3DAD4EAD5FAD6B
:10FBC000A79760916502709166028091670290919B
:10FBD00068020F94FF2BA7966CAF7DAF8EAF9FAFDF
:10FBE000A797812F902FA32DB22D8DA79EA7AFA7EA
:10FBF000B8ABC9AADAAAEBAAFCAAC984DA84EB8456
:10FC0000FC84CDAADEAAEFAAF8AE2DEC3CEC4CECBD
:10FC10005CE3C301B2010F94962529813A814B819F
:10FC20005C810F94962520916D0230916E02409177
:10FC30006F02509170020F94002C69AF7AAF8BAFB6
:10FC40009CAFA5019401C501B4010F9496254B0109
:10FC50005C01A7962CAD3DAD4EAD5FADA797CA0137
:10FC6000B9010F9496259B01AC01C501B4010F9415
:10FC7000002C20E030E040E050E40F94602E181695
:10FC8000ACF420E030E040E05FE3C701B6010F9440
:10FC9000002C29966CAF7DAF8EAF9FAF2997BE0128
:10FCA000635C7F4FCE0101960E94387489859A85E6
:10FCB000AB85BC8529968CAF9DAFAEAFBFAF299702
:10FCC000A3961CAE1DAE1EAE1FAEA397BE01615A19
:10FCD0007F4FCE01CD960E9495748CA58823C1F0EC
:10FCE0002AE939E949E95FE36D817E818F81988551
:10FCF0000F949625A3966CAF7DAF8EAF9FAFA39761
:10FD0000BE01615A7F4F8BE897E00E9495741CA654
:10FD1000E0906D0CF0906E0C00916F0C1091700CD7
:10FD2000A090690CB0906A0CC0906B0CD0906C0CD9
:10FD30009501A601B701C8010F94602E181614F49E
:10FD4000750186018090410290904202A09043028A
:10FD5000B09044022DEC3CEC4CEC5DE3B701C801E3
:10FD60000F94962560934102709342028093430260
:10FD70009093440240E0BE01675B7F4FCE018D96B9
:10FD80000F94691480E1E1E6F2E0ABE8B7E001909E
:10FD90000D928A95E1F78092410290924202A092E0
:10FDA0004302B092440220E04FEFBE01675A7F4FFA
:10FDB000CE0101960E94107620E041E0BE01675A14
:10FDC0007F4FCE0101960E9410762FEF40E0BE01DA
:10FDD000675A7F4FCE0101960E94107621E040E0E5
:10FDE000BE01675A7F4FCE0101960E9410760E9495
:10FDF00083618091AB0C8093AC0CAD964EAD5FAD42
:10FE0000AD9741505109AD965FAF4EAFAD97452BC1
:10FE100009F419CB6A968FAD6A9787FD14CB6B9660
:10FE20008FAD6B9787FFE1CB0ECB2BA13CA14DA1F2
:10FE30005EA1E5962CAF3DAF4EAF5FAFE5978FA1CA
:10FE400098A5A9A5BAA5EBCB812F902FA32DB22DF4
:10FE500021968CAF9DAFAEAFBFAF219720E030E0D1
:10FE600040EA50E4C701B6010F94FF2B25966CAF12
:10FE70007DAF8EAF9FAF2597A4965FADA49754300A
:10FE80000CF42FCE182D092D3A2C2B2C92ED492E47
:10FE900093E5592E9BEF692E90E4792E40CEA896DB
:10FEA0009FADA89794300CF452C0A496AFADA49720
:10FEB000A4300CF120E030E040EA50E4612F702FD4
:10FEC000832D922D0F94FF2B21966CAF7DAF8EAFBB
:10FED0009FAF219720E030E040EA50E4C701B6012F
:10FEE0000F94FF2B6B017C01A496EFADA497E43037
:10FEF0000CF40DCECBCF812F902FA32DB22D2196B8
:10FF00008CAF9DAFAEAFBFAF219720E030E040EAAD
:10FF100050E4C701B6010F94002C25966CAF7DAF5D
:10FF20008EAF9FAF2597A496BFADA497B111D2CF46
:10FF300020E030E040EA50E4612F702F832D922DB5
:10FF40000F94FF2B162F072F382E292E9FCFA49604
:10FF5000FFADA497F1110DC020E030E040E251E484
:10FF6000B401C5010F94FF2B162F072F382E292E11
:10FF7000CECDA4962FADA49724309CF020E030E0A5
:10FF800040E251E4B401C5010F94FF2B21966CAF00
:10FF90007DAF8EAF9FAF2197182D092D3A2C2B2CBA
:10FFA000B6CD182D092D3A2C2B2C82ED482E83E549
:10FFB000582E8BEF682E81E4782EB1CD2F923F9290
:10FFC0004F925F926F927F928F929F92AF92BF9269
:10FFD000CF92DF92EF92FF920F931F93CF93DF9315
:10FFE000CDB7DEB7EE970FB6F894DEBF0FBECDBF2C
:10FFF0008091400C888B87E50E942D1E882309F490
:020000021000EC
:1000000023C120E030E0A9016091ED057091EE057B
:100010008091EF059091F0050F943025811108C073
:100020000E94134E8DE09DE00E94443810E01FC1F5
:100030008AE50E947B1E882339F10E948124209149
:10004000EF083091F0084091F1085091F2080F94B8
:10005000FF2B6B017C0120E030E040E251ECC70156
:10006000B6010F94602E87FD0AC020E030E040E228
:1000700051E4C701B6010F943025181674F40E949C
:10008000134E80E09DE0D0CFC0906902D0906A020C
:10009000E0906B02F0906C02DECF40E050E060EC4C
:1000A0007FE788E50E94AB242091E7083091E808BB
:1000B0004091E9085091EA080F94FF2B2B013C0175
:1000C00040E050E060EC7FE789E50E94AB2420919E
:1000D000EB083091EC084091ED085091EE080F9438
:1000E000FF2B4B015C016FEF89E40E943D24182F28
:1000F0006FEF8AE40E943D24082FA3019201C301FF
:10010000B2010F94F22E81116EC0A5019401C501B8
:10011000B4010F94F22E811166C08BA19CA1ADA1F8
:10012000BEA18BAB9CABADABBEAB2091E5053091D6
:10013000E6054091E7055091E805C301B2010F942F
:10014000FF2B2B013C0120E030E040E05FE36BA996
:100150007CA98DA99EA90F9496259B01AC01C30192
:10016000B2010F94002C2BA93CA94DA95EA90F94B4
:10017000FA2C0F946C2D162F4FA058A469A47AA4C2
:100180002091E9053091EA054091EB055091EC058D
:10019000C501B4010F94FF2B4B015C0120E030E05E
:1001A00040E05FE3C301B2010F9496259B01AC01CF
:1001B000C501B4010F94002CA30192010F94FA2CF5
:1001C0000F946C2D062F812F012E000C990B97FD9B
:1001D00033C005979CF5802F002E000C990B97FDDE
:1001E0002FC005977CF5153008F020CF053008F0BA
:1001F0001DCF80E00E941C6995E01902F0011124D6
:10020000E00FF11D07FDFA95EE0FFF1FEE0FFF1F28
:10021000E955F84FC082D182E282F382602F812FAC
:100220000E94CDF788890E941C698889882309F477
:10023000FDCE0E949930FACE10E0CDCF14E0CBCFA6
:1002400000E0D1CF04E0CFCF8AE40E942D1E182F0A
:10025000811127C070E060E086E50E9472249A83D5
:100260008983059708F18BED9CE00E944438812F2B
:10027000EE960FB6F894DEBF0FBECDBFDF91CF91E3
:100280001F910F91FF90EF90DF90CF90BF90AF90B4
:100290009F908F907F906F905F904F903F902F90A6
:1002A00008950E94FA6EC2CE60E084E40E94592450
:1002B0008F8740E050E0BA018AE50E94AB246BA72B
:1002C0007CA78DA79EA740E050E86BE376E483E52A
:1002D0000E94AB2420E030E040E752E40F94FA2C77
:1002E00060933D0270933E0280933F0290934002E0
:1002F000E0908B12F0908C12D7018D909D90AD9074
:10030000BC9020E030E0A901C501B4010F94002C9D
:100310006BAF7CAF8DAF9EAF20E030E040E450E4A7
:100320000F94302587FF06C01BAE1CAEB0E4BDAFF6
:10033000E0E4EEAF20E030E044EB53E4C501B4016B
:100340000F94002C662E7BAB8FAB98AF20E030E88B
:1003500042EB53E40F94602E18163CF4612CF0E845
:10036000FBAB22EB2FAB33E438AFD70114968D9063
:100370009D90AD90BC90179720E030E0A901C50199
:10038000B4010F94002CD62EE72EF82E092F20E072
:1003900030E040EE51E40F94302587FF05C0D12CAA
:1003A000E12CF0EEFF2E01E420E030E044EB53E4DA
:1003B000C501B4010F94002CB62EC72E89AF9AAF99
:1003C00020E030E046EA53E40F94602E181634F42F
:1003D000B12CC12CB6EAB9AFE3E4EAAF88E40E94DD
:1003E0002D1E882309F416C20E9481240F946C2DBF
:1003F0001B0177FF02C06F5F7F4F75956795719501
:10040000619571096C547F4F072E000C880B990B76
:100410000F943725762E872E982EA92E2D2D3E2D22
:100420004F2D502F0F94602E18161CF4D72C7401EA
:100430000A2D2BAD3CAD4DAD5EAD672D782D892DD0
:100440009A2D0F94602E181624F07BAC8CAC9DACCA
:10045000AEAC872D982DA92DBA2D8B8B9C8BAD8B97
:10046000BE8B8D2D9E2DAF2DB02F8F8B988FA98F8A
:10047000BA8FB101330C880B990B0F9437251B01F0
:100480002C01AC019B016D2D7E2D8F2D902F0F9493
:10049000002CD62EE72EF82E092F2B2D3C2D49AD02
:1004A0005AAD0F94302587FF04C0BD2CCE2CF9AE79
:1004B0000AAFA2019101672D782D892D9A2D0F94F5
:1004C000002CD62EE72EF82E092F262D3BA94FA95A
:1004D00058AD0F94302587FF04C06D2CEBAAFFAAFE
:1004E00008AF862D9BA9AFA9B8AD8B8F9C8FAD8F20
:1004F000BE8F8B2D9C2DA9ADBAAD8F8F98A3A9A3CC
:10050000BAA3BE01695E7F4FCE0143960E94392E89
:10051000882309F4B0C1BE01615E7F4FCE014B96C6
:100520000E94392EE82E882309F4A5C12F89388D21
:10053000498D5A8D6F8D78A189A19AA10F94FF2BB7
:1005400020E030E040E85EE30F9496254B015C012B
:100550002B893C894D895E896B8D7C8D8D8D9E8D1F
:100560000F94FF2B20E030E040E85EE30F949625E7
:100570006BA37CA38DA39EA38FA298A6A9A6BAA6BF
:1005800089819A811816190674F489EA9CE00E9400
:1005900044388F85882321F08FE99CE00E944438FD
:1005A0008AE00E940B380E9483610E94C21C80E096
:1005B0000E941C6980E090E0A0E2B1E48FA798ABB4
:1005C000A9ABBAAB60E0CE018F960E94D6642091B1
:1005D000ED053091EE054091EF055091F0056BA1CE
:1005E0007CA18DA19EA10F943025811130C0209156
:1005F000F1053091F2054091F3055091F4056FA19A
:1006000078A589A59AA50F943025811120C0209145
:10061000E5053091E6054091E7055091E8056B89C5
:100620007C898D899E890F943025811110C020917D
:10063000E9053091EA054091EB055091EC056F8991
:10064000788D898D9A8D0F9430258823A9F00E948A
:10065000FA6E88E0FE01B396ADEEB5E001900D9222
:100660008A95E1F788E0FE017396A5EEB5E001906A
:100670000D928A95E1F7188A60E085E40E9459247A
:10068000882309F4FBC0F1E0FBAB1B861C861D86AA
:100690001E861A8A9E2C4FE6C42E4CE0D42E5DE7AF
:1006A000A52E5CE0B52E1A8915300CF0F7C06B85CD
:1006B0007C858D859E859B01AC010F94F22E811166
:1006C000EDC0992009F4DDC031E03FAB35E0232EC9
:1006D00091E09926F12EFF0CFF0CF10EF394898B1B
:1006E00019896A89121509F4D5C0062E000C770BFA
:1006F000880B990B0F9437252FA138A549A55AA52A
:100700000F9496252F89388D498D5A8D0F94002C82
:100710002B013C01612F110F770B880B990B0F9464
:1007200037252BA13CA14DA15EA10F9496252B89C5
:100730003C894D895E890F94002C6B837C838D836B
:100740009E834F82588669867A8689819A81892B11
:1007500079F06F2D8BE89CE00E94184169E170E010
:1007600089E89CE00E94424186E89CE00E9444386F
:100770001F9299E19F931F92FF92DF92CF92BF92B7
:10078000AF921F920E94F8F829814BA9BE01695FC0
:100790007F4FCE0103960E9469F92B013C014B86E5
:1007A0005C866D867E860FB6F894DEBF0FBECDBF29
:1007B000AC019B010F94F22E811169C089883A889F
:1007C00025E0382D320380011124030D111D37FC63
:1007D0001A95000F111F000F111F0955184FA30183
:1007E00092016BA57CA58DA59EA50F94002CD80128
:1007F0006D937D938D939C931397632D882D0E9409
:10080000CDF7188A81E00E941F5AF3948989BFA905
:100810008B0F65CF4D2D5E2D6F2D702F86E40E94BE
:10082000AB241B012C014BAD5CAD6DAD7EAD8CE4FA
:100830000E94AB246B8B7C8B8D8B9E8B2F8A388E8A
:10084000498E5A8E4B2D5C2D69AD7AAD82E40E94A3
:10085000AB246B017C01462D5BA96FA978AD82E5C5
:100860000E94AB246B8F7C8F8D8F9E8FCF8ED8A2F2
:10087000E9A2FAA246CE8FEB9CE0F7CC22E02BABAC
:1008800004CF8FEF8FAB22242A9484E021CF888974
:100890000E941C698A898F5F8A8B05CF0E9463E45E
:1008A0000E94AC65882359F088890E941C6980E009
:1008B00090E0A0ECBFE78B879C87AD87BE876B85F8
:1008C0007C858D859E859B01AC010F94F22E811154
:1008D00059C08F85811126C082E0F82E02E094E095
:1008E000C92E12E0DC2CD11A21E041E0612F802FCB
:1008F0000E945A2221E04FEF612F8F2D0E945A2231
:100900002FEF41E06D2D802F0E945A222FEF4FEFE5
:100910006D2D8F2D0E945A22115020F70150F39413
:100920000F3FF9F60E9489400E94881E8F85811131
:1009300024C089E692E00E94721D4B015C0181E6B1
:1009400092E00E94181F9B01AC01C501B4010F94F5
:1009500096259B01AC016091690270916A028091B9
:100960006B0290916C020F94FF2B6093690270935D
:100970006A0280936B0290936C028F858111E888E4
:10098000E092400C0E94A91C8091400C81110E94B1
:10099000E52A0E9496670E9499306B857C858D853B
:1009A0009E8511E09B01AC010F94F22E81115FCC6A
:1009B0003DCB8F929F92AF92BF92CF92DF92EF92F8
:1009C000FF920F931F93CF93DF9300D01F92CDB769
:1009D000DEB75C016B017A01122F0023E1F10E9466
:1009E000174E88E999E00E94443861E0812F0E9407
:1009F000383A90902C0583E080932C0581E0809319
:100A00003E0C0E942F4082E08093981140E368E8FA
:100A100079E084E799E00E94344040E069E171E1C7
:100A20008DE699E00E94344061E088E699E00E94FA
:100A300016408AE799E00E94162280913E0C882396
:100A400041F060E0812F0E94383A81E00E941F5AF5
:100A5000F4CF90922C0520E030E0A901F5016081EF
:100A60007181828193810F943025882371F080E019
:100A700090E0A0ECB0E489839A83AB83BC83BE0191
:100A80006F5F7F4FC5010E945C6820E030E0A901E4
:100A9000F60160817181828193810F9430258823D2
:100AA00051F180907D0C90907E0CA0907F0CB090C6
:100AB000800C80E090E0A0E7B1E480937D0C9093FF
:100AC0007E0CA0937F0CB093800C80E090E0A0EAB5
:100AD000B1E489839A83AB83BC83BE016F5F7F4F90
:100AE000C6010E945C6880927D0C90927E0CA09260
:100AF0007F0CB092800C20E030E0A901F70160810A
:100B00007181828193810F94602E181674F480E0B5
:100B100090E0A0E4B0E489839A83AB83BC83BE01F8
:100B20006F5F7F4FC7010E945C688091010529E1DA
:100B300031E1882311F029E439E047E559E061E625
:100B400079E081E00E9457400E942F4081E00F90A1
:100B50000F900F900F90DF91CF911F910F91FF9009
:100B6000EF90DF90CF90BF90AF909F908F900895BF
:100B7000CF93C82F8091FD0B83FD14C080911A097B
:100B8000811110C080915F02909160029C01215000
:100B900031094091F4115091F5114217530714F4A3
:100BA0000E94031FCC2329F061E080E0CF910C94D8
:100BB000D9BC80911A0991E0892780933C028091E9
:100BC0003C02882389F08091F2119091F3112091D9
:100BD000F4113091F511821B930B97FF03C091958F
:100BE00081959109029744F410923C028091FD0B8B
:100BF00083FF06C0C1E01AC080E00E941F5ADFCF09
:100C0000C0911A09C11112C080915F0290916002D7
:100C100001972091F4113091F5112817390754F7F5
:100C20000E94174E8BE299E00E9444388C2FCF919E
:100C30000895AF92BF92CF92DF92EF92FF920F93FF
:100C40001F93CF93DF93CDB7DEB764970FB6F894B9
:100C5000DEBF0FBECDBF0E94164F87FDAFC08AE535
:100C60000E947B1E882309F4BAC040E050E0BA011C
:100C70008AE50E94AB247B018C01209169023091AE
:100C80006A0240916B0250916C0260E070E088EC67
:100C900093E40F94FF2B5B016C019701A8010F9463
:100CA000602E181614F07501860120E030E0A901CD
:100CB000B701C8010F94602E181624F4E12CF12C12
:100CC00000E010E0B701C8010F946C2D072E000C56
:100CD000880B990B0F943725698B7A8B8B8B9C8BA8
:100CE00020E030E0A9010F943025882321F0CE01C7
:100CF00041960E94DA7280E090E0A0EAB1E48D872C
:100D00009E87AF87B88B19861A861B861C868CE453
:100D10000E942D1E882309F467C00E9481246B0164
:100D20007C0120E030E0A901C701B6010F94602EDC
:100D300087FF04C0F7FAF094F7F8F094CD82DE82D2
:100D4000EF82F8862091F4113091F51124303105AD
:100D500074F08091F2119091F311821B930B97FF25
:100D600003C091958195910901E004970CF400E08E
:100D700080E00E94B885882359F022E0AE01435FED
:100D80005F4FBE016B5F7F4FCE0109960E94D984F1
:100D900069897A898B899C898B019C0130580983E8
:100DA0001A832B833C8320E030E0A9010F94302587
:100DB000882321F0CE0101960E94DA7264960FB664
:100DC000F894DEBF0FBECDBFDF91CF911F910F9181
:100DD000FF90EF90DF90CF90BF90AF900895E12CFF
:100DE000F12C00E211E449CFC090E005D090E1057C
:100DF000E090E205F090E30594CF7F928F929F926E
:100E0000AF92BF92CF92DF92EF92FF920F931F9318
:100E1000CF93DF9300D000D01F921F92CDB7DEB7E3
:100E20006C015B014A01722E780100912D060E942F
:100E30000F1F8091F4119091F5118E159F051CF4F0
:100E4000C7010E94031F80E00E94B885882331F00B
:100E5000272DA401B501C6010E94D9841E141F04C8
:100E60003CF4C7010E94031F60E080E00E94D9BCEF
:100E700081E00E94B88580E090E0A0E7B2E4898339
:100E80009A83AB83BC8380E090E0A0E8B0EC8D83D4
:100E90009E83AF83B887BE016F5F7F4FCE010596FB
:100EA0000E945C6887E00E94FC29811158C08091F3
:100EB000690290916A02A0916B02B0916C0240911C
:100EC0000605509107056091080570910905C090CD
:100ED0000205D0900305E0900405F0900505C0924E
:100EE0008B07D0928C07E0928D07F0928E0740938B
:100EF0008F075093900760939107709392078093A8
:100F0000930790939407A0939507B093960780E07A
:100F100090E0A8E4B2E489839A83AB83BC83CE01DA
:100F200001960E94737280910A0590910B05A09121
:100F30000C05B0910D058093930790939407A093AF
:100F40009507B093960780E090E0A0EAB0E489832B
:100F50009A83AB83BC83CE0101960E947372C12C2D
:100F6000D12C80E7E82E82E4F82EC982DA82EB8267
:100F7000FC8280E090E0A0E8B0E48D839E83AF83A4
:100F8000B887BE016F5F7F4FCE0105960E945C68F7
:100F900020E030E0A90160910E0570910F0580916D
:100FA0001005909111050F94302587FF0BC0C98261
:100FB000DA82EB82FC82BE016F5F7F4F8EE095E0AC
:100FC0000E945C6880910E0590910F05A09110051C
:100FD000B091110580936D0290936E02A0936F0201
:100FE000B09370028093970790939807A093990706
:100FF000B0939A0787E997E00E9494618091E40595
:1010000081110E9413F761E087EB99E00E947F3F16
:1010100080912A11815080932A114EE658E16FEB9E
:1010200079E085E00E94E8E280912A11882339F076
:101030000E9412AB80912A11815080932A1180E086
:101040000E94DAF80E94933180912B11823011F4C2
:101050000E9452380E9463E428960FB6F894DEBFCF
:101060000FBECDBFDF91CF911F910F91FF90EF90F9
:10107000DF90CF90BF90AF909F908F907F9008951A
:10108000CF92DF92EF92FF920F931F93CF93DF9354
:1010900000D01F92CDB7DEB77C016B018A0161E001
:1010A0008CE399E00E947F3F4EE658E163E479E0EB
:1010B00085E00E94E8E290912A1181E0890F8093F7
:1010C0002A118091381482FF06C08B7F80933814D8
:1010D0009E5F90932A110E94443980E1E1E6F2E09C
:1010E000A2E0B5E001900D928A95E1F70E9483613C
:1010F00081E00E94DAF820E030E0A901F701608188
:101100007181828193810F9430258823F1F0809141
:101110001A0981110CC080915F02909160020197C1
:101120002091F2113091F3112817390774F080E003
:1011300090E0A0E7B2E489839A83AB83BC83BE01CD
:101140006F5F7F4FC7010E945C6887E00E94FC29A7
:10115000811103C0B6010E94B06720E030E0A90110
:10116000F80160817181828193810F9430258823F9
:1011700041F080E00E94B885882319F0C8010E94E0
:101180008C68129A64E670E080E090E00E94EF259F
:1011900081E00F900F900F900F90DF91CF911F91F2
:1011A0000F91FF90EF90DF90CF900895CF92DF9254
:1011B000EF92FF92CF93DF936B017C01D42FC0910C
:1011C0002C0583E080932C0581E080933E0CC114B4
:1011D000D104E104F10431F00E940BFDC60ED71ECC
:1011E000E81EF91E80913E0C882389F0C114D104B9
:1011F000E104F10421F48D2F0E941F5AF3CF0E94C5
:101200000BFD6C197D098E099F0997FDF4CF109293
:101210003E0CC0932C05DF91CF91FF90EF90DF90B3
:10122000CF9008950F931F93CF93DF93C82F162F5E
:101230000E94174EC11194C0CFE8D8E0CE010E94A1
:10124000443861E0812F0E94383A0E940BFD6853B8
:1012500070458F4F9F4F6093290670932A068093A5
:101260002B0690932C0610922D0600912C0583E0FE
:1012700080932C0530E020E049E151E16DE179E017
:1012800082E00E9457408DE199E00E94162281E0A1
:1012900080933E0C80913E0C882309F464C060E08A
:1012A000812F0E94383A80912D06882309F454C07A
:1012B0000E94174E83E099E00E94443830E020E01D
:1012C0004DEE58E064EF78E082E00E94574084EFF2
:1012D00098E00E94162241E060E070E0CB010E949D
:1012E000D68830E020E050E040E060EE78E085E035
:1012F0000E94574080EE98E00E949A350E940F1F8E
:1013000080E00E94B8850E94174ECE010E944438AA
:101310000E940BFD685370458F4F9F4F60932906C5
:1013200070932A0680932B0690932C0610922D061C
:1013300030E020E049E151E164ED78E082E00E9494
:10134000574083EC98E00E94162281E080933E0C87
:1013500061E0812F0E94383A81E00E941F5A9ACFA3
:10136000C4EAD8E06BCF00932C05DF91CF911F9199
:101370000F910895CF92DF92EF92FF920F931F93F8
:10138000CF93DF93CDB7DEB7A0970FB6F894DEBF4B
:101390000FBECDBF0E94164F87FDCCC085E40E94D2
:1013A0002D1E882309F4D5C00E9481246B017C0185
:1013B00020E030E0A9010F94602E87FF04C0F7FA07
:1013C000F094F7F8F094F7FAF094F7F8F094CD8EE3
:1013D000DE8EEF8EF8A28CE0E6EDF2E0DE011196F3
:1013E00001900D928A95E1F78AE50E947B1E882381
:1013F00051F040E050E0BA018AE50E94AB246987D1
:101400007A878B879C8788E50E947B1E882351F012
:1014100040E050E0BA0188E50E94AB2469837A83FA
:101420008B839C8389E50E947B1E882351F040E0DA
:1014300050E0BA0189E50E94AB246D837E838F83DF
:10144000988785E50E942D1E882309F489C00E9493
:1014500081246B017C0120E030E0A901C701B601C5
:101460000F94602E87FF04C0F7FAF094F7F8F09419
:10147000F7FAF094F7F8F094C98EDA8EEB8EFC8EC2
:101480001D8A1E8A1F8A188E8CE40E942D1E8823B6
:1014900009F46FC00E9481246B017C0120E030E0E0
:1014A000A901C701B6010F94602E87FF04C0F7FAA7
:1014B000F094F7F8F094C98ADA8AEB8AFC8A62E041
:1014C00070E082E40E947224F82E80912A1181112A
:1014D00031C021E0AE01475E5F4FBE016F5F7F4FBD
:1014E000CE014D960E944088882321F16F2D81E026
:1014F0000E94128982E50E947B1E882309F442C063
:101500000E946E2440E050E060EA71E44D875E87FF
:101510006F87788B20912A11222361F08C012F2D67
:10152000AE01435F5F4FBE016F5E7F4FCE014596B8
:101530000E94FD86A0960FB6F894DEBF0FBECDBF09
:10154000DF91CF911F910F91FF90EF90DF90CF909F
:101550000895C12CD12C80E8E82E80E4F82E33CFFA
:10156000C090DC05D090DD05E090DE05F090DF0551
:1015700072CFC090E005D090E105E090E205F090D8
:10158000E3058CCF90E080E0BDCFCF92DF92EF9269
:10159000FF920F931F93CF93DF93CDB7DEB76C9776
:1015A0000FB6F894DEBF0FBECDBF8CE40E942D1E97
:1015B000882309F4B0C00E9481246B017C0120E0E3
:1015C00030E0A9010F94602E87FF04C0F7FAF09471
:1015D000F7F8F094F7FAF094F7F8F094C98EDA8EF1
:1015E000EB8EFC8E8CE0E6EDF2E0DE0111960190D0
:1015F0000D928A95E1F788E50E947B1E8823A1F071
:1016000040E050E0BA0188E50E94AB242091E70851
:101610003091E8084091E9085091EA080F94FF2BB7
:1016200069837A838B839C8389E50E947B1E882350
:10163000A1F040E050E0BA0189E50E94AB2420917E
:10164000E7083091E8084091E9085091EA080F94C2
:10165000FF2B6D837E838F8398878AE50E947B1E94
:10166000882351F040E050E0BA018AE50E94AB24A3
:1016700069877A878B879C871D861E861F86188AB6
:1016800080912A11811138C020E0AE01435F5F4F85
:10169000BE016F5F7F4FCE0149960E94408888232C
:1016A00059F18091E40581110E9413F760E080E018
:1016B0000E941289898D9A8DAB8DBC8DB0588D8B0F
:1016C0009E8BAF8BB88F198A1A8A1B8A1C8A1D863B
:1016D0001E861F86188A80912A11882369F010E0DF
:1016E00000E020E0AE014B5E5F4FBE016F5E7F4FBA
:1016F000CE010D960E94FD866C960FB6F894DEBF63
:101700000FBECDBFDF91CF911F910F91FF90EF9052
:10171000DF90CF900895C12CD12C80E8E82E80E492
:10172000F82E58CF2F923F924F925F926F927F92F6
:101730008F929F92AF92BF92CF92DF92EF92FF92E1
:101740000F931F93CF93DF93CDB7DEB7E5970FB617
:10175000F894DEBF0FBECDBF8DAB20912C052CAB16
:1017600021E020932C0580914A058D3409F403C6AD
:10177000843511F40C94E3A0873409F091C1809171
:101780004805909149058B31910509F4DDC108F0B8
:1017900079C18430910508F030C120910007823072
:1017A000910508F48EC1213009F091C111E0029732
:1017B00009F010E00E94C22419821A821B821C8246
:1017C0001D821E821F82188682E50E947B1E88234E
:1017D00009F490C10E9481246B017C0120E030E07B
:1017E000A9010F943025882309F4EAC040906102D2
:1017F0005090620260906302709064028091650272
:1018000090916602A0916702B09168028CA79DA793
:10181000AEA7BFA780908B0790908C07A0908D07F4
:10182000B0908E0780918F0790919007A0919107BB
:10183000B091920788AB99ABAAABBBABA501940161
:10184000C301B2010F94302581110DC028A939A917
:101850004AA95BA96CA57DA58EA59FA50F943025EF
:10186000882309F4ADC0A3019201C501B4010F940E
:10187000FF2B20E030E040E05FE30F94962568A75F
:1018800079A78AA79BA72CA53DA54EA55FA568A90A
:1018900079A98AA99BA90F94FF2B20E030E040E0B2
:1018A0005FE30F9496252B013C0120E030E0A90175
:1018B000C701B6010F943025881F8827881F181785
:1018C00009F40FC180E090E0A0E8BFEB8CA79DA7D2
:1018D000AEA7BFA728A539A54AA55BA5CA01B9012E
:1018E0000F9496254B015C01A3019201C301B20143
:1018F0000F9496259B01AC01C501B4010F94002CF7
:101900000F94AE2E4B015C01AC019B01C701B601E7
:101910000F94FF2B68AB79AB8AAB9BABA50194010D
:10192000C701B6010F94002C9B01AC0168A979A9ED
:101930008AA99BA90F9496256B017C0120E030E0D9
:10194000A9010F94602E87FDD1C0C701B6010F9485
:10195000AE2E6B017C01C301B2019058A501940128
:101960000F94FA2C2CA53DA54EA55FA50F949625A6
:10197000A70196010F94962528A539A54AA55BA530
:101980000F94002C69837A838B839C83A501940137
:1019900068A579A58AA59BA50F94FA2C2CA53DA531
:1019A0004EA55FA50F949625A70196010F94962545
:1019B000A30192010F94002C6D837E838F839887FF
:1019C00020E030E0A90169817A818B819C810F94AC
:1019D00030258111A3C020E030E0A9016D817E8116
:1019E0008F8198850F943025811198C00E94134EE5
:1019F0008BEB9FE00E9444386AC08531910509F461
:101A000066C08A31910509F49CC0049709F048C06A
:101A100080E50E947B1EC12CD12C7601882321F009
:101A20000E94FB236B017C0183E50E947B1E8823BF
:101A300061F00E94812420E030E04AE754E40F94F2
:101A400096250F94732D6B017C010E948361809118
:101A50002C11811105C060E081ED9FE00E94B23F32
:101A60000E940BFDC60ED71EE81EF91E0E940BFD3C
:101A70006C197D098E099F0997FF29C080E00E949B
:101A80001F5AF4CF8A32910509F4EAC260F48D310D
:101A9000910509F413C208F470C04E9709F466C2A8
:101AA0000E942CF914C08B35910509F4BCC38C3508
:101AB000910509F4BCC38A35910591F710920B0882
:101AC00006C0213021F40E94C2240E94C06F3DA9AB
:101AD000311102C00F9416148CA980932C050C941C
:101AE000449980E090E0A0E8BFE3F0CEC12CD12C77
:101AF000760131CF89E40E947B1E882331F00E9459
:101B0000812469837A838B839C838AE40E947B1E71
:101B1000882309F455CF0E9481244ECF412FBE0166
:101B20006F5F7F4F8BE897E00F9469140E940BFD65
:101B300060937D1170937E1180937F11909380113B
:101B4000C6CF0E94AF77C3CF87E00E94274E811196
:101B5000BECF8CE0E2EEF2E0DE01119601900D9234
:101B60008A95E1F770E060E080E50E941B24BE01E9
:101B70006F5F7F4F0E94B067AACF87E00E94FC2969
:101B8000811106C060E08FE40E94592481119FCF2B
:101B90000E948361109246026091400C8CE40E9486
:101BA0005924E82E80E00E941C690E940BFD60937E
:101BB0007D1170937E1180937F11909380110E940C
:101BC000C21C81E08093BC060E946D2B8AE50E94B6
:101BD0002D1EF82E882369F081E00E94FC29182F21
:101BE00082E00E94FC2911110C9406A111E08111E0
:101BF00001C010E088E50E942D1E81110C94F8A010
:101C0000111143C189E50E942D1E082F811307C0C1
